:020000040000fa
:080000000002040000000000f2
:020000040000fa
:10040000af152100007f24000001880000000000db
:100410000a00070011000700000020000000e000b3
:10042000020032000000020000000000386c0200f0
:10043000000000000040da000000fe004440a90077
:10044000a0d420000000e0000300320000002000e3
:10045000a00188004440a80000000600c041270019
:10046000010020001500370062004000e0804800d5
:10047000910188009001ba0062004000e0804800cd
:10048000910188009002ba0062004000e0804800bc
:100490000002eb006028e10004003a000059eb0084
:1004a0008301e900fdff3e00040037006128e10000
:1004b000010032000082eb00050007009101880076
:1004c0001001ba000200e000e7ff3a00000005005a
:1004d000910188008002780062004000e0804800be
:1004e0003559ba008301e900080032002559ba00e5
:1004f0008301e900050032000400e000f4ff32004f
:1005000015d9ba008301e900f1ff3a0000000600a6
:10051000f2840400000000003885040000000000a0
:10052000549704000000000028830400000000002d
:100530007e85040000000000226904000000000025
:100540009a6a040000000000086c0400000000002b
:100550009e6a040000000000b26b0400000000006e
:1005600088980400000000002c86040000000000b1
:10057000c088040000000000e088040000000000c3
:10058000dc88040000000000de8804000000000099
:10059000248a0400000000002c8a040000000000ef
:1005a0004c8a040000000000a68a0400000000003d
:1005b000188b040000000000588b040000000000ad
:1005c000e288040000000000ea8804000000000047
:1005d0000a89040000000000648904000000000093
:1005e000d689040000000000168a04000000000004
:1005f000545c0400000000002e5c040000000000b9
:100600009096040000000000d8970400000000004d
:100610002e960400000000009a97040000000000dd
:100620001403040000000000881f78000204780012
:10063000ba000700080040004f04780000000600e0
:100640000000fa00881f7800000478003fb9970086
:10065000ea8157008000780040312000b600070092
:10066000800078000000e000020035000040eb0050
:1006700000f47800010078004f0478000080fa0050
:10068000000006008001eb00020037008171780055
:100690008301e800828f5100fcff3a000000060051
:1006a00080007800010037000000e8001004e0003e
:1006b000fdff3a000100500000000600889fbe00c8
:1006c000e30440000900a100808f54004a00360076
:1006d000e38f540001003e0049002000027a8000b0
:1006e0000200e00002003200820078000c003700b7
:1006f00021f4200003003700908f540023003600bf
:100700008080e800110078000000e000faff3a0065
:100710000f003700908f54001c0036008080e800e6
:10072000110078000000e000faff3a0012017800a2
:1007300021f4200003003700908f5400130036008e
:100740008080e80011007800820f5000faff3a0024
:10075000f8798000890f5400010031000904780005
:10076000080078002d0107000000e00004003a00b6
:10077000890f5400200032000804d100f5ff370033
:100780000818780031000700d4ff37001101780005
:100790009201780064805100890f500003003100fd
:1007a000120090008008780007003700090041001f
:1007b00080087800920190001300980011007800e2
:1007c0001288140009097800910078000100e00007
:1007d00005003200110090000000e000020032002d
:1007e0000180e800010037000000eb00007a88007b
:1007f0000280e800010037000000eb004f04be005b
:100800000000060000047800060037008200410066
:10081000307a8000e10078000200e800207a880049
:1008200001000100227a8000407a8000800f510090
:10083000f6ff3900e0e82000307a8800200220002e
:10084000407a880008007800d80307000000e00024
:10085000310032008080e90091027800e38f52007d
:100860002d0036000508a3002b003a00127a800004
:100870000200e00002003200828f500004003100cc
:1008800002087800117a880016003700030178000a
:10089000920190000300e00002003200818f5100bd
:1008a000faff39001202780004004100808f5000e6
:1008b00019003900810f500003003a000509420079
:1008c00082007800070037000300e00003003200d8
:1008d00005804000808f51000f0039009300980080
:1008e00011019800110190000200e0000a0032009e
:1008f00011804000820f500007003a0000f42000f1
:100900000008eb00110090001101780090084100f0
:100910001000900090009800000006008001eb009d
:100920000200370061f079008301e800828f5100f6
:10093000fcff3a00000006006200fa00889fbe003b
:100940008a9fbe000004be00020578008300780084
:1009500060f92f000f004000b700070088979f0044
:1009600099979f000000eb00a09f9f009a45780098
:100970000b80fb000000ea00cf04de0050c2b30091
:1009800080cf5500020032000904780001003700d2
:100990000904e9000800e0000b0034001f909700f4
:1009a000080178008a0078008f9197000300010009
:1009b00090979f000000e000930032002f9897006e
:1009c00000004400a09f9f000905450050c2b300ed
:1009d00080cf5500040032000b04e000e3ff3a0032
:1009e0002f989700890037000000eb00809f9f0040
:1009f000f0979f00e0979f00d0979f00c0979f00bf
:100a0000b0979f00c09f9f000900370080f1200031
:100a10000080500000004000c1f02000e10078009c
:100a20004f98970001007000c09f9f000a05e800e2
:100a30001a4478008800fb0080f120008300070042
:100a4000800078000000e000f0ff3a00a0c2b30090
:100a5000804f54000e003a00bf8897000180e900e3
:100a6000b08f9f0010007800b09f9f000000e00052
:100a700005003d000000ea00b09f9f004f989700de
:100a80000020a000c09f9f000a05e800100037006a
:100a9000b19f9f0009003700bf989700f0ff270023
:100aa000808f5000040032006a08b9000000410045
:100ab00003004000b09f9f000a05e8001a01fb00f8
:100ac00003fd2f0003004100e90f5000f2ff360044
:100ad000e0c2b3009a4f1000040032000080eb0027
:100ae000909f9f008a0478001c0037008a04e80069
:100af000a0c2b300994f100007003a00bf889700ca
:100b00000180e900b08f9f0010007800909f9f0047
:100b10008a84e800110037000000eb00909f9f00de
:100b2000090037009f989700f0ff2700808f500042
:100b3000040032006a08b9000000410003004000d0
:100b4000909f9f008904e8001901fb0003fd2f001e
:100b500003004100e90f5000f2ff3600194478000d
:100b60008800fb0000f32000380007000000e000d0
:100b700002003a0000447800010037008904e800d0
:100b8000a87f9f0080c6b300804f540004003a0045
:100b9000994f14000a003a006640500006003700e2
:100ba000c0c6b300804f540005003a00994f1400ae
:100bb00003003a0065404000a07f9f008904e800e0
:100bc0000905e800cbfb2f008f8545001901fb00cc
:100bd00060f92f000f0040000084e8008b017800ce
:100be0008000780008007800210007000000e00085
:100bf00005003a008b007800080078005f010700cc
:100c00000000e00059ff3d000080eb004f05be00f2
:100c10004f04be000080fa00000006000000e00063
:100c200003003400e9020700e10f400001003a0030
:100c30000000eb00000006000200fa00f1bf9f0078
:100c4000010878000080fa00000006000400370068
:100c50000204e00001003a00000005000000e80086
:100c600010417800814f5100f9ff3a000000060062
:100c7000889fbe008a1f7800000478000102780077
:100c80008244780003057800e0c6b300804f51002d
:100c9000d200320015003c006b405000804f5100e4
:100ca000240032000a003c0070405000804f510088
:100cb0000f01320065404000804f51007400320047
:100cc00050c2b300804f510020013a001c01370090
:100cd00040c6b300804f51001b0032006540400009
:100ce000804f510019013a001700370030c7b30098
:100cf000804f5100fe00320007003c00644050006d
:100d0000804f5100620032000040e800804f5100e7
:100d10000e013a00e700370050c7b300804f510082
:100d20005b00320063404000804f510007013a00f1
:100d3000570037009180e900010a780078009000a0
:100d40009171780007013700a8609000c0c6b30019
:100d500080cf50000a003a00940078006480500070
:100d6000000a78001000be004f89de00cf91de003f
:100d70000002be00020378008203780013003700ef
:100d800010c7b30080cf500003003200a0c6b300ec
:100d900080cf500006003a00940078006880500030
:100da000000a78003002be002003be0007003700b2
:100db0001480e900000a7800100078000002780032
:100dc000cfa2de000503780086037800049cbe00f5
:100dd0000694be00a860900080c6b30080cf50008b
:100de0000e00320020c6b30080cf500005003a004c
:100df0000400fb00cf80de00010178008201780052
:100e00000a00370040c7b30080cf50000300320013
:100e10006640400080cf500006003a000400780091
:100e2000cf80de000101780082017800009cbe00c6
:100e30000294be003800be002801be00e00f500042
:100e4000e08f5800e00f5900e08f590003003d008b
:100e500078009000d1c2b3000a003700081090005b
:100e60000018a3000300320078009000b1c2b30064
:100e7000040037000008a3005300320078009000ff
:100e800001c2b300017578000000e8004d00370092
:100e9000a8609000c0c6b30080cf500006003a00a2
:100ea0009400780064805000000a78001002be00b0
:100eb0006033b8001300370010c7b30080cf500074
:100ec00003003200a0c6b30080cf500006003a00f5
:100ed0009400780068805000000a78003002be005c
:100ee0002003be00070037001480e900000a7800e4
:100ef00010007800000278000500200006002000a5
:100f000007002000049cbe000694be00a86090006c
:100f100080c6b30080cf50000e00320020c6b30060
:100f200080cf500005003a000480fb000100200043
:100f300002002000030020000a00370040c7b30071
:100f400080cf5000030032006640400080cf500048
:100f500006003a0004007800010020000200200092
:100f600003002000009cbe000294be000810900008
:100f70000038a300140032003800be002801be0073
:100f8000e00f5000e08f5800e00f5900e08f59004b
:100f90000d00320080c7b30080cf54000300320040
:100fa00080c5b30080cf540007003a00780090005d
:100fb00001c3b300017578008000e80009f57800ee
:100fc0000080e80070049800780090000000450060
:100fd000600498008940780042003700a8609000c3
:100fe000c0c6b30080cf5000250032000a003c008c
:100ff0006440500080cf50002800320000c0e8005c
:1010000080cf5000140032006840500080cf500064
:1010100022003a000a00370040c7b30080cf5000da
:101020001e0032006640400080cf50001b0032009e
:101030006940500080cf500018003a000600370089
:101040001480e900000a780010007800485c9000e5
:1010500008487800450037001480e900000a78004d
:101060001002780068089000cf80de00010178004f
:1010700082017800009abe000292be003b00370059
:101080001480e900000a78001001780068089000d8
:10109000cf80de000089be00340037001480e900f4
:1010a000000a780010007800680c900008087800aa
:1010b0002e0037001180e9008008780010007800c9
:1010c000cf80de000101780082017800009cbe0024
:1010d0000294be0078009000000045006004980073
:1010e00081c7b30008007800ee0007001f0037003a
:1010f0001480e900000a780010007800600498006d
:10110000580990000200e00002003d0064fd070065
:10111000090037008000eb009a010700800078008a
:101120000000e000030032006800900000805000e2
:101130000100370058089000100c98000b00370091
:101140007800900002757800060037007800900063
:10115000800045000904e00001003a0059c2b300d4
:10116000894878000000e800700498000000eb0057
:101170004f0578004f04be00000006000400fa008e
:10118000889fbe008a9fbe008c1f780000047800f4
:101190000106780070089000f800900001005000ef
:1011a000880890000100500098089000010050004d
:1011b000a808900001005000b808900001005000fd
:1011c000c8089000810550000002220090bf9f00d7
:1011d00000032300a0bf9f00081090000028a30078
:1011e00018003a000b00e000160034008b04780071
:1011f00009057800e28f5400020036002a00200022
:10120000020037000900e0000b0034005800900095
:10121000c80190000a017800ee8057000300010029
:10122000500498000000e00096003200680890002a
:1012300000004500600c98008a8454004240a900d8
:10124000ebff3c00780190000200e0000b0034004e
:1012500058009000c80190008c0078000300010045
:10126000500498000000e0008600320068089000fa
:10127000f800900001004000600c9800880c90007d
:101280000900e0001500340009057800e28f5400e1
:10129000020036002a002000020037000900e000aa
:1012a0000b00340058009000c80190000a0178003b
:1012b000ec80570003000100500498000000e0009b
:1012c000700032006808900000004500600c980033
:1012d0008a8454004240a900ebff3c0018099000aa
:1012e0000200e0000b003400e8009000580090007d
:1012f000c801900003000100500498000000e000c5
:1013000060003200680890009808900001004000da
:10131000600c9800a80c90000900e0001500340053
:1013200009057800e28f5400020036002a002000f0
:10133000020037000900e0000b0034005800900064
:10134000c80190000a017800ec80570003000100fa
:10135000500498000000e0004a0032006808900045
:1013600000004500600c98008a8454004240a900a7
:10137000ebff3c00380990000200e0000d00340053
:10138000e80090001808900080804000580090000d
:10139000c801900003000100500498000000e00024
:1013a0003800320068089000b80890000100400042
:1013b000600c9800c80c90000900e0001500340093
:1013c00009057800e28f5400020036002a00200050
:1013d000020037000900e0000b00340058009000c4
:1013e000c80190000a017800ec805700030001005a
:1013f000500498000000e0002200320068089000cd
:1014000000004500600c98008a8454004240a90006
:10141000ebff3c00081090000028a3001b003200e6
:101420000b00e000190034008b04780009057800f7
:10143000e28f5400020036002a002000020037002c
:101440000900e0000b00340058009000c801900033
:101450000a017800ee805700030001005004980054
:101460000000e0000700320068089000000045001e
:10147000600c98008a8454004240a90003003400a4
:10148000eaff37000080eb00010037000000eb00ae
:101490004f0678004f05be004f04be000080fa00e2
:1014a00000000600ef02b000889fbe008a9fbe00c9
:1014b0008c9fbe008e1f78000006780030ee200062
:1014c000c0b79f0080c5b30080cf50000800320035
:1014d00022ed2000c2b79f007740400080cf50002f
:1014e00003003a0083002000b3b79f000a003700d2
:1014f00080c7b30080cf500005003200a400200058
:10150000b4b79f0080c5b30080cf500002003a00fe
:1015100000012000b0b79f003c04be002c05be00b7
:1015200040c6b30080cf5000030032006540400049
:1015300080cf50000b003a00e00f5400e08f5c00b9
:10154000e00f5d00e08f5d0006003d006000b80028
:101550006011b80008045000898458000a05590039
:101560008b855900e00f5400e08f5c00e00f5d00b8
:10157000e08f5d0004003a005c0890008d012000bf
:101580000000e0000c003200bfb0970001027800bc
:10159000cfa2de0005037800860378000800be00b5
:1015a0000a01be006e0207004fb297006440780047
:1015b000d0df9f007d0120003fb09700000278003f
:1015c000cfa2de0005037800860378000800be0085
:1015d0000a01be005b020700009ebe000296be002c
:1015e0000d00e90061fc2f008f8040000087400063
:1015f0001e0037003fb1970002047800cfc4de0020
:10160000090578008a0578000802be000a03be00ba
:101610007fa897008fb097001fb19700afb19700d8
:1016200053020700d0b79f00e1b79f00f2b79f00b9
:1016300083bf9f008d06e9000802be000a03be00ba
:10164000d10207007faa970000005200cfb0970098
:10165000615778005fb09700efb097007fb19700b7
:101660008fb99700009ebe000296be003c00be00ef
:101670002c01be00f0af9f0081b79f0092b79f0082
:10168000a3b79f00e00f5000e08f5800e00f590013
:10169000e08f5900020034000d00e000d5ff3c004f
:1016a000bfb09700e88f500010003a000c10900077
:1016b0000038a3000d003200f78f560006003e00f0
:1016c00062fc2f000f0141008d00410000c3b300f8
:1016d000914f1000050032008d06e90000c3b300f1
:1016e00063fc2f008f81410080f17e00788116001d
:1016f000120e98006c00900063fc2f008f81410057
:101700008d80410085fc07001c0990005c0890005a
:10171000800f510006003d0002005000000e9800ae
:101720000c1090000040a100001698000f00370038
:101730000000e0000d003d000c10900074006000ff
:10174000f00f500009003a007c089000fc00900067
:10175000010050008c089000010050000200500071
:101760004240a90001003400000e98004f077800a5
:101770004f06be004f05be004f04be00ef02b10091
:10178000000006008001eb00040037008301e80040
:1017900090cf1000040032000000e800828f51005a
:1017a000faff3a000000eb00000006002002e20011
:1017b00004003d002342ab00020032002302ab00d4
:1017c000feff32000040da00feff3700889fbe00b7
:1017d00080047800e40ce20004003a000000eb0012
:1017e000100007000000e0000a00350020678000bc
:1017f0000900e00002003a0000047800060037000b
:101800000004780009004000060007000000e00026
:1018100001003d000084eb00080078004f04be008a
:1018200000000600800078000000e00004003a009c
:10183000a0f520002067880001017800060037002d
:101840000081eb00a0152100808f500002003e00b7
:10185000216788000001eb0002007800000006000c
:101860000001be00760207000470a70003f0a1008b
:1018700003f8a30013003a006509b100100032001c
:10188000090035006928e100020035000100280048
:101890000000050000004000818048008502e9004a
:1018a000fcff3a0000000600f88f420005003500fa
:1018b0008100d1000080d3008502e800fcff3a00df
:1018c000000006008000eb0000000500889fbe00bd
:1018d0008a9fbe00010578000100e0000400350089
:1018e00008003c000000e000200032000500370046
:1018f00060001000e080180002003b0001f02c00a6
:101900001a0037000004be006011b8006b09200007
:101910000982cf00020039000882cf000441b000e4
:10192000694252000e00320008003b0082817100c3
:10193000610164008904d1000884d3008b05e800ac
:101940000442e800f9ff3a000500370008044400ab
:1019500089844c008b05e9000442e900fbff3a0052
:101960004c0207000af0a70001f0a0004f05be00de
:101970004f04be0000000600889fbe008a9fbe0084
:101980008c1f7800690207007002330003866c0028
:101990006450e1002e0032006420e1003300320088
:1019a0006150e1002f0032006120e100310032007f
:1019b00085855500eb07b0000900200008042000d1
:1019c000050037000804440089844c000a003100f7
:1019d0000603430087834b000001530081815b00b5
:1019e000f8ff33000203be000800a0000804440012
:1019f00089844c00f6ff3900c639dd00830173008d
:101a000001003200130020008904d1000884d300b3
:101a10000998a300050032000800a7000300a000f9
:101a20008904d1000884d3008b05e8008904d10023
:101a30000884d3000001eb000281d20015020700e8
:101a400001f0a1000cf0a70001f0a000480237004f
:101a50006420e1004a0232000801be000200be001c
:101a6000f7ff37006120e100450232006000b80056
:101a7000f3ff37000000200001f82700f0ff3700d7
:101a8000889fbe008a9fbe008c1f78002702070037
:101a90002e02330003866c006450e1002400320003
:101aa0006420e100270032006150e1002200320092
:101ab0006120e100210032008b854200eb07b1007c
:101ac0000134b800003ab8000804420089844a0092
:101ad000013ab8000030b8008880400009014a008f
:101ae00004003300000040008180480002014900ea
:101af0008b05e900c909dd00830170000100320097
:101b000013002000c814de004814dd004709de0081
:101b10001200b200c808de0008847000dd01070072
:101b200001f0a1000cf0a70001f0a00010023700a6
:101b30006120e100120232000801be000200be0076
:101b4000f7ff37006150e100fcff3a000c0237005c
:101b500003f0a200889fbe008a9fbe008c1f780001
:101b6000f2010700f90133006450e1004f00320038
:101b70006420e1005200320003826c0007003b0049
:101b80000905d0000306d000820f54000c065d004a
:101b90000200390002003200890178000306780053
:101ba0008582550004003d000003fd008103fd0017
:101bb0008502ea008b854200840f720002003b0020
:101bc00060001000e08018006011b8000005eb0014
:101bd0007a28e1000a00390006007800c75ddd00c0
:101be000f707b200878075002d00370082817100f1
:101bf0000a017800610560008180d1000080d30077
:101c00008502e900f9ff3b00060440008784480094
:101c100002003b0060041400e0841c000988a3005b
:101c2000070032008a8171008281710061016400c5
:101c30008904d1000884d3008b05e8001700370021
:101c40000978a30013003a000b00e00013003400f1
:101c50008b05e9000804440089844c000a447400a0
:101c60000978a3000d003a000b00e00007003400e3
:101c70008b05e9000804440089844c0001003a0007
:101c80000b0020000978a300f7ff32000001eb00f1
:101c900002003700828171000a0178007d0107008f
:101ca0000cf0a70001f0a000b10137006420e100b2
:101cb00002003a00838f6c00b10133000801be00be
:101cc0000200be00aa013700f4ff2f00af01370069
:101cd00014002000ad0137000001be0058010700cc
:101ce0000470a70003f0a1006509b10016003200de
:101cf0000d0035006828e10006003500f0ff2f00d8
:101d0000f1ff27000300e00013003b000100280062
:101d10000000050000004000818048008502e900c5
:101d2000fcff3a0008003700f88f420002003c0038
:101d30008000eb00000005008100d1000080d3008e
:101d40008502e800fcff3a000300e00002003b00cf
:101d500060001000e080180000000600881f780076
:101d6000000478005001be004000be0004004000a6
:101d7000858048000601490087814900009cbe001b
:101d80000294be000400e1000588e1000690e10035
:101d90000798e10002003100680044001008e800e4
:101da0004f04780000000600f4874700889fbe00bb
:101db0008a9fbe008c9fbe008e1f78000205be0069
:101dc0000004be00d4b79f00e5b79f00f6b79f00a0
:101dd00087bf9f000000eb00c0b79f00b0b79f0017
:101de000a0b79f0090b79f0080b79f000d04200010
:101df000bfb097004fb09700000140000000e00026
:101e00000f003d004f08de0000007100c0b79f00ca
:101e10009e00070001003d0012002000a100070005
:101e200001003d0012002000a6000700b1000700dd
:101e3000b60007000f004000c8ff0700220037006f
:101e40004f08de0000067100ccb79f008f0007002e
:101e500001003d00120020009200070001003d003b
:101e60001200200097000700a20007000fb29700a1
:101e70009fb297002fb39700bfb39700a900070048
:101e80000000520081805a0002015b0083815b00e8
:101e900080b79f0091b79f00a2b79f00b3b79f0084
:101ea0000007eb009f0007000020e10001a8e1000f
:101eb00002b0e10003b8e100010031001e00200083
:101ec0000e005600c0b79f004fb297000400e0001c
:101ed0000700350010002000010020006011b8004c
:101ee00008047000898470000a0571008b857100f8
:101ef0008d06e900beff3a000400e00003003d004b
:101f0000820007000f00400094ff07004fa89700d1
:101f10000000e00004003a000fb497009fb497005f
:101f20002fb59700bfb59700940007004f077800c2
:101f30004f06be004f05be004f04be004f01b1006a
:101f400000000600881f780018002000881f780015
:101f500095ff07008f87e9004f0478000000060016
:101f6000801feb0090ff07008f87e900000006004c
:101f7000889fbe008a9fbe008c1f78006e000700fd
:101f800007003d0073000700e00f5b00e08f5b007f
:101f900007003d00320007000006eb000400370098
:101fa0003400070002003d002a0007001c0020004a
:101fb00072000700e3ff07000203be000002be003c
:101fc0000c00e00001003200220007000400be0007
:101fd0000601be004f0678004f05be004f04be004c
:101fe00000000600889fbe008a9fbe008c1f7800fc
:101ff0005100070005003d0056000700e00f5b00a0
:10200000e08f5b0006003d00040037001900070068
:1020100003003d006000b8006011b8001000070028
:1020200056000700ceff07000203be000002be00fc
:102030000c00e00001003200060007000400be00b2
:102040000601be004f0678004f05be004f04be00db
:10205000000006006000b8006011b8000000370002
:1020600004025000858258000603590087835900f6
:10207000000006000006eb00e00f5200e08f5a005f
:10208000e00f5b00e08f5b00000006000180400075
:1020900090b79f000001eb008fb097000100e000b7
:1020a000000006000200700090b79f000180400011
:1020b00080b79f000001eb00ffa897000100e0003f
:1020c000000006000200700080b79f000180400001
:1020d0006faa9700cf20de0001007000f0af9f00d4
:1020e00004024200250007004f18de0000027200c3
:1020f00000000600e4af9f000804440089844c00ff
:102100000a054d008b854d00000006003fb2970088
:10211000cfb297005fb39700efb3970000fe2f0098
:10212000000006003fb09700cfb097005fb1970066
:10213000efb19700000006000205be000004be00db
:10214000e00f5000e08f5800e00f5900e08f590079
:10215000000006006000b8006011b80008045000dc
:10216000898458000a0559008b8559001c002000fd
:10217000e00f5200e08f5a00000006000800be0089
:102180000a01be0000000600889fbe008a9fbe00b4
:102190008c1f78000205be000004be000006eb00a4
:1021a000e00f5000e08f5800e00f5900e08f590019
:1021b00007003d006000b8006011b800080450003e
:1021c000898458000a0559008b8559001c0020009d
:1021d000e00f5200e08f5a00e00f5b00e08f5b00e1
:1021e00002003d000f0007000c00a2000800be0026
:1021f0000a01be00800007000203be000002be000c
:102200000c00e00001003200060007000400be00e0
:102210000601be004f0678004f05be004f04be0009
:10222000000006006000b8006011b8000402500011
:102230008582580006035900878359000000060074
:10224000c70ade00f107b200f50fb2000800320045
:10225000e1cf4200020032000170a000240005001e
:10226000810f7000010032000408050044000500e1
:10227000810f700002003a00140005008502e90099
:102280000000400081c04800fcff3b000170a0003e
:102290002400050081002000618055000b003d00f6
:1022a0000b00200061fe2f000100e1001d00340042
:1022b00082817100610164008904d1000884d30027
:1022c0000000e800faff3a0071002000610064009d
:1022d0000300700002006000090032006104440045
:1022e000e0844c000988a500050032008b05e80059
:1022f0006808e10002003a008904d1000884d30094
:10230000f20f20000258e10005003d00c75ddd002e
:10231000f907b20089807500080078000000060007
:102320000bf827008b007800000005000004be00b9
:10233000c3ff07000003be000405be000200be008c
:10234000bfff0700844f7500000006000200be00ba
:102350006450e100050036006420e1000200360010
:102360000968a30001003a000800be000160a00057
:102370004f0678004f05be004f04be000000060067
:10238000f0ff2f00f1ff2700f9ff3700889fbe0004
:102390008a9fbe00841f7800e4ff07004f0078008a
:1023a00011003300f0ff2f00838f6c0006003b000c
:1023b000040565000a00a7000800370009f0a60020
:1023c0001000200008003700820f5400838f5c004b
:1023d000030039001000200001003e000000200032
:1023e00009f0a7000000ea004f05be004f04be0040
:1023f0000000e00000000600889fbe008a9fbe002b
:102400008c9fbe000404b8000506b800890446008d
:1024100060854e000606b8000a054600e0854e00bd
:102420000706b8008b054600040eb8008904460074
:102430000a854e00e0854d00050eb8000a054600ed
:102440008b854e00060eb8008b0546000416b800ba
:102450000a0546008b854e000516b8008b05460020
:10246000041eb8008b0546000800be000a01be002d
:102470004f06be004f05be004f04be000000060020
:102480000000fa0023c2bf000004a2000000fb000d
:10249000610060000080fa00000006000000fa0001
:1024a00033c2bf000004a2000000fb006100600016
:1024b0000080fa00000006000000fa0021e2a900f6
:1024c0009560a9009580a9008560a9008580a90074
:1024d0000080fa00000006000000fa0031e2a900c6
:1024e00097c0a90097e0a90087c0a90087e0a900cc
:1024f0000080fa00000006000200fa00000f7800d9
:102500008560a9008580a9001e00780067406000f2
:102510006740600067406000674060004401dd0084
:10252000910a200091407800f0c8b30000c060001c
:1025300002407000a9e0b700000720001e00600004
:102540004400de006740600067416000a10a20008f
:102550009140780080cfb30000c06000024070005e
:10256000aae0b7009e007800688060004300de00ab
:1025700061406000614060004301dd0051092000be
:102580009140780070cfb30000c06000024070003e
:1025900095e0b700000820001e0060004700de0044
:1025a00061406000614060004401dd00510920008d
:1025b00091407800f0ceb30000c06000024070008f
:1025c00095e0b7000080fa00000006000200fa0063
:1025d000000f780087c0a90087e0a9001e007800de
:1025e00067406000674060006740600067416000ce
:1025f000310b20009140780080cfb30000c0600014
:1026000002407000b3e0b700000720001e00600029
:102610004400de0067406000674060004401dd0068
:10262000310b200091407800f0c8b30000c060007a
:1026300002407000b3e0b7009e0078006880600040
:102640004300de0061406000614060004601dd0043
:102650007109200091407800f0cbb30000c0600009
:102660000240700097e0b700000820001e006000e4
:102670004700de0061406000c700dd0097c0bf007a
:102680000074a1000140700097e0b7000080fa00dc
:10269000000006000000fa0022c2bf006140600096
:1026a0000080fb000080fa00000006000000fa0035
:1026b00032c2bf00614060000080fb000080fa0071
:1026c000000006000c00fa0020079800310798006f
:1026d000420798000000eb00100798003e009000b1
:1026e000000f7800230037009e0090004e009000fd
:1026f000808f5000040031001e0090000000e800b0
:1027000010079800030037002e0090005007980033
:102710001d003700dfff07000004e000f2ff320079
:102720000000eb001007980020c2bf006640600068
:10273000e64f500007003a00311180003e00900043
:10274000010878003e0090000080e8003007980003
:102750000500370030118000804078001e007800ae
:10276000014878001e0fe8002e0090000000e900ec
:10277000200798002e0090000000e000e5ff3a00de
:102780002e009000500798005e0090000080fa0034
:10279000000006000c00fa0020079800310798009e
:1027a000420798000000eb00100798003e009000e0
:1027b000000f7800230037009e0090004e0090002c
:1027c000808f5000040031001e0090000000e800df
:1027d00010079800030037002e0090005007980063
:1027e0001d003700b1ff07000004e000f2ff3200d7
:1027f0000000eb001007980030c2bf006640600088
:10280000e64f500007003a00b11180003e009000f2
:10281000010878003e0090000080e8003007980032
:1028200005003700b0118000804078001e0078005d
:10283000014878001e0fe8002e0090000000e9001b
:10284000200798002e0090000000e000e5ff3a000d
:102850002e009000500798005e0090000080fa0063
:10286000000006000600fa00000f7800110798002b
:10287000220798002e009000401188001e0078006a
:10288000001188001e009000101188000080fa00de
:10289000000006000600fa00000f780011079800fb
:1028a000220798002e009000c01188001e007800ba
:1028b000801188001e009000901188000080fa00ae
:1028c000000006000400fa00100798001e009000a7
:1028d000000f780023c2bf00624060000004e000e7
:1028e000fcff3a0020c2bf0066406000e64f500087
:1028f00019003a000a0037001e009000100078000e
:10290000201188001e0090000080e8001007980049
:1029100023c2bf00624060000004e000fcff3a00f8
:102920001e009000100078000000e000f2ff3a0066
:102930000d0037001e007800104078000000fb00fa
:10294000201188001e0fe80023c2bf006240600013
:102950000004e000fcff3a001e0078001040780000
:102960000004e000f3ff3a000080fa0000000600d7
:102970000400fa00100798001e009000000f780075
:1029800033c2bf00624060000004e000fcff3a0078
:1029900030c2bf0066406000e64f500019003a00a8
:1029a0000a0037001e00900010007800a011880077
:1029b0001e0090000080e8001007980033c2bf009e
:1029c000624060000004e000fcff3a001e0090003e
:1029d000100078000000e000f2ff3a000d00370020
:1029e0001e007800104078000000fb00a011880055
:1029f0001e0fe80033c2bf00624060000004e00028
:102a0000fcff3a001e007800104078000004e0004f
:102a1000f3ff3a000080fa00000006000200fa000e
:102a200020c2bf0066406000e64f500003003a003d
:102a300030118000000f7800040037003111800051
:102a4000f00f200080806000010f78001e007800e9
:102a50000080fa00000006000200fa0030c2bf0049
:102a600066406000e64f500003003a00b01180005d
:102a7000000f780004003700b1118000f00f200033
:102a800080806000010f78001e0078000080fa004e
:102a9000000006000200fa00000f780023c2bf0009
:102aa000624060000004e000fcff3a0020c2bf006a
:102ab00066406000e64f500003003a001e007800b8
:102ac0002011880003003700f00f20001e00600076
:102ad000201188000080fa00000006000200fa00c1
:102ae000000f780033c2bf00624060000004e000c5
:102af000fcff3a0030c2bf0066406000e64f500065
:102b000003003a001e007800a0118800030037007f
:102b1000f00f20001e006000a01188000080fa0065
:042b200000000600ab
:020000040000fa
:0200000401f009
:04000000ffff0000fe
:020000040000fa
:0200000401f009
:04000400ffff0000fa
:020000040000fa
:0200000401f009
:04000c00faff0000f7
:020000040000fa
:0200000401f009
:040010007eff00006f
:020000040000fa
:0200000401f009
:040014007fff00006a
:020000040000fa
:0200000401f009
:04001800ffff0000e6
:020000040000fa
:100008008c980000d26d0000346e0000966e0000df
:10001800f86e00008c9800008c9800008c98000006
:100028008c9800008c9800008c98000064400000b8
:100038008c9800008c9800008c980000128d0000ad
:10004800529000008c9800008c980000d89700000f
:10005800909600008c9800008c9800008c98000006
:100068008c980000b88200008c9800008c980000e2
:100078008c9800008c9800008c9800008c980000e8
:100088008c9800008c9800008c980000e04a0000d2
:100098008c9800008c9800009a9700002e9600001b
:1000a8008c9800008c9800008c9800008c980000b8
:1000b8008c9800008c9800008c9800008c980000a8
:1000c8008c9800008c9800008c9800008c98000098
:1000d8008c9800008c9800008c9800008c98000088
:1000e8008c9800008c9800008c9800008c98000078
:1000f8008c9800008c9800008c9800008c98000068
:100108008c9800008c9800008c9800008c98000057
:100118008c9800008c9800008c9800008c98000047
:100128008c9800008c9800008c9800008c98000037
:100138008c9800008c9800008c9800008c98000027
:100148008c9800008c9800008c9800008c98000017
:100158008c9800008c9800008c9800008c98000007
:100168008c9800008c9800008c9800008c980000f7
:100178008c9800008c9800008c9800008c980000e7
:100188008c9800008c9800008c9800008c980000d7
:100198008c9800008c9800008c9800008c980000c7
:1001a8008c9800008c9800008c9800008c980000b7
:1001b8008c9800008c9800008c9800008c980000a7
:1001c8008c9800008c9800008c9800008c98000097
:1001d8008c9800008c9800008c9800008c98000087
:1001e8008c9800008c9800008c9800008c98000077
:0801f8008c9800008c980000b7
:020000040000fa
:100208008c980000d26d0000346e0000966e0000dd
:10021800f86e00008c9800008c9800008c98000004
:100228008c9800008c9800008c98000064400000b6
:100238008c9800008c9800008c980000128d0000ab
:10024800529000008c9800008c980000d89700000d
:10025800909600008c9800008c9800008c98000004
:100268008c980000b88200008c9800008c980000e0
:100278008c9800008c9800008c9800008c980000e6
:100288008c9800008c9800008c980000e04a0000d0
:100298008c9800008c9800009a9700002e96000019
:1002a8008c9800008c9800008c9800008c980000b6
:1002b8008c9800008c9800008c9800008c980000a6
:1002c8008c9800008c9800008c9800008c98000096
:1002d8008c9800008c9800008c9800008c98000086
:1002e8008c9800008c9800008c9800008c98000076
:1002f8008c9800008c9800008c9800008c98000066
:100308008c9800008c9800008c9800008c98000055
:100318008c9800008c9800008c9800008c98000045
:100328008c9800008c9800008c9800008c98000035
:100338008c9800008c9800008c9800008c98000025
:100348008c9800008c9800008c9800008c98000015
:100358008c9800008c9800008c9800008c98000005
:100368008c9800008c9800008c9800008c980000f5
:100378008c9800008c9800008c9800008c980000e5
:100388008c9800008c9800008c9800008c980000d5
:100398008c9800008c9800008c9800008c980000c5
:1003a8008c9800008c9800008c9800008c980000b5
:1003b8008c9800008c9800008c9800008c980000a5
:1003c8008c9800008c9800008c9800008c98000095
:1003d8008c9800008c9800008c9800008c98000085
:1003e8008c9800008c9800008c9800008c98000075
:0803f8008c9800008c980000b5
:020000040000fa
:102b2400436f00006d6d0000206c00006f6f0000ab
:102b340070200000697300002073000074610000bd
:102b440072740000656400000a000000497300000c
:102b540020740000686500007265000020610000b8
:102b6400206d00006573000073610000676500005c
:102b7400206600006f720000206d0000653f0000b9
:102b84000a00000025730000202d00003e200000f4
:102b9400257300000a00000053300000002a0000e2
:102ba400005300003100000054680000657200000a
:102bb4006520000069730000206400006174000057
:102bc4006120000055410000525400000a0000003a
:102bd40046610000696c0000656400002074000018
:102be4006f2000007265000061640000206d000029
:102bf4006573000073610000676500000a0000004f
:102c040049200000676f0000742000007468000011
:102c1400652000006d6500007373000061670000ab
:102c2400650a000000540000686500007265000039
:102c340020690000732000006461000074610000da
:102c4400206f00006e200000425400000a000000c3
:102c54005b25000030320000585d00000043000096
:102c6400464700005f4300004f4d00004d4c0000fc
:102c74004f4f0000503a00002073000062430000f0
:102c840066670000436f00006d6d00004c6f00002c
:102c94006f70000044650000636f0000646500000d
:102ca4000a0000005365000074200000436f000018
:102cb4006d6d00004c6f00006f7000002056000026
:102cc40065720000626f000073690000747900008f
:102cd4000a000000537400006f700000706500006b
:102ce40064200000436f00006d6d00004c6f000015
:102cf4006f7000002056000065720000626f0000d3
:102d040073690000747900000a0000004346000063
:102d1400475f0000434f00004d4d00004c4f000042
:102d24004f5000003a20000073620000426100002e
:102d34007369000063520000657000006c79000044
:102d4400456e0000636f0000646500000a00000027
:102d540043460000475f0000434f00004d4d000014
:102d64004c4f00004f5000003a20000073620000f6
:102d7400536500006e6400004d650000737300002d
:102d840061670000650000004b45000045500000ed
:102d94005f4100004c490000564500003a20000005
:102da4007362000042610000736900006352000016
:102db400657000006c790000456e0000636f0000d0
:102dc40064650000004b000045450000505f0000b2
:102dd400414c000049560000453a000020730000b1
:102de40062530000656e0000644d000065730000ce
:102df4007361000067650000004b0000656500001a
:102e040070200000416c000069760000650a000033
:102e140000430000464700005f4300004f4d0000a0
:102e24004d3a000020730000624300006667000012
:102e3400436f00006d6d000044650000636f000087
:102e440064650000005300007461000072740000a7
:102e540065640000206300006f6e00007469000068
:102e64006e7500006f75000073200000636f000032
:102e74006d6d0000756e00006963000061740000f0
:102e8400696f00006e0a00000053000074610000c6
:102e94007274000065640000206f00006e2d000055
:102ea400646500006d6100006e6400002063000032
:102eb4006f6d00006d7500006e69000063610000b5
:102ec400746900006f6e00000a00000043460000b1
:102ed400475f0000434f00004d4d00003a200000c2
:102ee40073620000426100007369000063520000d5
:102ef400657000006c790000456e0000636f00008f
:102f04006465000000430000464700005f43000082
:102f14004f4d00004d3a0000207300006253000042
:102f2400656e0000644d000065730000736100006d
:102f34006765000000530000544100005445000040
:102f44003a200000736200005265000071530000d3
:102f5400746100007465000044650000636f000044
:102f64006465000000530000544100005445000013
:102f74003a20000046610000696c000065640000ae
:102f8400207400006f200000656e0000636f000075
:102f94006465000020680000656c00006920000082
:102fa4007374000061740000650a0000005300009f
:102fb40054410000544500003a20000073620000b0
:102fc400536500006e6400004d65000073730000db
:102fd4006167000065000000416300006365000054
:102fe40070740000656400002073000074610000c8
:102ff40074650000207200006571000075650000b2
:1030040073740000202500003034000058200000b4
:1030140025300000345800000a0000004745000035
:10302400545f00005645000052530000494f000011
:103034004e3a0000207300006256000065720000e2
:10304400736900006f6e00004d7300006745000057
:103054006e6300006f640000650a00000047000012
:10306400455400005f5600004552000053490000db
:103074004f4e00003a2000007362000053650000c8
:103084006e6400004d65000073730000616700000a
:103094006500000052650000636500006976000069
:1030a400656400002076000065720000736900000a
:1030b4006f6e0000207200006571000075650000ed
:1030c400737400000a000000534500004e530000d2
:1030d4004f5200004c490000535400003a200000b5
:1030e40073620000536500006e7300006f7200008d
:1030f4004c69000073740000456e0000636f0000ab
:10310400646500000a000000534500004e530000af
:103114004f5200004c490000535400003a20000074
:1031240073620000536500006e6400004d6500008a
:1031340073730000616700006500000052650000c1
:103144006365000069760000656400002073000078
:10315400656e0000736f0000722000006c6900004f
:103164007374000020720000657100007565000032
:10317400737400000a000000436f00006e6e0000cc
:1031840065630000746900006f6e00002061000038
:10319400636300006570000074650000640a000049
:1031a400004300004f4e00004e4500004354000011
:1031b4003a2000007362000042610000736900005d
:1031c40063520000657000006c790000456e0000d9
:1031d400636f0000646500000a000000434f0000b4
:1031e4004e4e000045430000543a00002073000096
:1031f40062530000656e0000644d000065730000ba
:10320400736100006765000000440000495300003a
:10321400434f00004e4e000045430000543a000066
:1032240020730000624200006173000069630000c3
:1032340052650000706c0000794500006e63000068
:103244006f640000650a0000004400004953000058
:10325400434f00004e4e000045430000543a000026
:103264002073000062530000656e0000644d00008e
:10327400657300007361000067650000004400008e
:1032840069730000636f00006e6e000065630000e8
:10329400746900006f6e0000206100006363000029
:1032a4006570000074650000640a000000520000ac
:1032b40045530000455400003a20000073620000aa
:1032c40042610000736900006352000065700000f1
:1032d4006c790000456e0000636f000064650000b7
:1032e4000a0000005245000053450000542000002d
:1032f40052650000636500006976000065640000a3
:103304000a00000043460000475f0000424c0000f2
:1033140055450000544f00004f540000483a000047
:1033240020730000624300006f6e000066690000b5
:103334006775000072650000426c0000756500004e
:10334400746f00006f74000068440000656300003f
:103354006f640000650a0000004300004647000057
:103364005f4200004c550000455400004f4f0000e0
:10337400544800003a2000007362000042610000db
:103384007369000063520000657000006c790000ee
:10339400456e0000636f0000646500000a000000d1
:1033a40043460000475f0000424c000055450000c2
:1033b400544f00004f540000483a000020730000ae
:1033c40062530000656e0000644d000065730000e8
:1033d4007361000067650000004300006f6e000029
:1033e40066690000677500007265000064200000d3
:1033f400426c000075650000746f00006f7400007b
:1034040068200000287300007567000067650000ed
:10341400737400002072000065730000657400007e
:10342400290a000000430000464700005f4f0000e7
:10343400415600004f490000443a00002073000048
:1034440062430000666700004f41000044650000cd
:10345400636f0000646500000a000000434600003a
:10346400475f00004f410000564f000049440000f0
:103474003a2000007362000042610000736900009a
:1034840063520000657000006c790000456e000016
:10349400636f0000646500000a00000043460000fa
:1034a400475f00004f410000564f000049440000b0
:1034b4003a20000073620000536500006e6400004f
:1034c4004d65000073730000616700006500000033
:1034d400436f00006e6600006967000075720000ab
:1034e40065640000204f00006273000074610000f6
:1034f400636c000065200000417600006f690000e5
:10350400646100006e630000650a0000004300006f
:10351400464700005f540000494d0000454f00003d
:10352400555400003a200000736200004366000016
:1035340067540000696d0000656f00007574000039
:1035440044650000636f0000646500000a00000029
:10355400436f00006e66000069670000757200002a
:103564006564000020540000696d0000656f000070
:10357400757400003a200000256400002026000035
:1035840020250000640a00000043000046470000b4
:103594005f540000494d0000454f000055540000a1
:1035a4003a20000073620000426100007369000069
:1035b40063520000657000006c790000456e0000e5
:1035c400636f0000646500000a00000043460000c9
:1035d400475f0000544900004d4500004f5500006e
:1035e400543a00002073000062530000656e00002e
:1035f400644d00006573000073610000676500009e
:1036040000490000676e00006f72000065640000ee
:1036140020540000726900006d2000004d6f00000e
:1036240064650000202800004e6f00002068000040
:10363400616e0000646c000065720000290a0000dd
:1036440000540000524900004d5f00004d4f00003f
:10365400444500003a2000007362000054720000e8
:10366400696d00004d6f000064650000456e000048
:10367400636f0000646500000a00000054520000fb
:10368400494d00005f4d00004f440000453a0000e2
:103694002073000062530000656e0000644d00005a
:1036a400657300007361000067650000005400004a
:1036b400524900004d5f00004d4f0000444500009a
:1036c4003a2000007362000054720000696d00002b
:1036d4004d6f00006465000044650000636f0000e6
:1036e400646500000a000000496700006e6f000076
:1036f400726500006420000054720000696d0000cf
:10370400204d00006f640000650a000000430000c3
:103714006f6e000066690000677500007265000046
:103724006420000054720000696d0000204d000008
:103734006f640000650a0000005400005249000054
:103744004d5f00004d4f0000444500003a2000004a
:10375400736200004261000073690000635200005c
:10376400657000006c790000456e0000636f000016
:10377400646500000a000000496700006e6f0000e5
:103784007265000064200000436f00006e74000046
:10379400726f00006c200000506100007261000034
:1037a4006d6500007465000072730000202800003d
:1037b4004e6f000020680000616e0000646c000021
:1037c40065720000290a0000004300005452000002
:1037d4004c5f000050410000524d00003a200000b0
:1037e4007362000054720000696d00004d6f0000a8
:1037f40064650000456e0000636f000064650000ae
:103804000a00000043540000524c00005f500000c6
:10381400415200004d3a0000207300006253000042
:10382400656e0000644d0000657300007361000064
:103834006765000000430000545200004c5f000024
:1038440050410000524d00003a2000007362000015
:1038540043740000726c000050610000726100004b
:103864006d6500007465000072730000446500001b
:10387400636f0000646500000a00000049670000ef
:103884006e6f00007265000064200000436f00004a
:103894006e740000726f00006c2000005061000024
:1038a400726100006d6500007465000072730000b1
:1038b4000a000000436f00006e66000069670000a4
:1038c4007572000065640000204300006f6e000004
:1038d400747200006f6c00002050000061720000e0
:1038e400616d00006574000065720000730a0000d9
:1038f40000430000545200004c5f0000504100009f
:10390400524d00003a200000736200004261000042
:103914007369000063520000657000006c79000058
:10392400456e0000636f0000646500000a0000003b
:1039340043460000475f000052410000575f00000b
:10394400434d0000443a000020730000624300002d
:103954006667000052610000774300006f6e00004c
:10396400747200006f6c000044650000636f000017
:10397400646500000a000000436f00006e660000ea
:103984006967000075720000656400002052000041
:1039940061770000204300006f6d00006d6100003e
:1039a4006e6400000a00000043460000475f000008
:1039b40052410000575f0000434d0000443a0000ac
:1039c400207300006242000061730000696300001c
:1039d40052650000706c0000794500006e630000c1
:1039e4006f640000650a00000043000046470000c1
:1039f4005f520000415700005f4300004d44000047
:103a04003a20000073620000536500006e640000f9
:103a14004d650000737300006167000065000000dd
:103a240043460000475f0000434f00004e5400002f
:103a3400524f00004c3a0000207300006243000023
:103a440066670000436f00006e740000726f000030
:103a54006c440000656300006f640000650a0000a8
:103a6400004300006f6e0000666900006775000087
:103a74007265000064200000436f00006e74000053
:103a8400726f00006c200000436f00006d6d000039
:103a9400616e0000640a0000004300004647000015
:103aa4005f4300004f4e0000545200004f4c000092
:103ab4003a20000073620000426100007369000054
:103ac40063520000657000006c790000456e0000d0
:103ad400636f0000646500000a00000043460000b4
:103ae400475f0000434f00004e540000524f000057
:103af4004c3a00002073000062530000656e000021
:103b0400644d000065730000736100006765000088
:103b140000530000455400005f4300004f4e000076
:103b2400545200004f4c00003a2000007362000021
:103b340053650000744300006f6e0000747200004f
:103b44006f6c000044650000636f00006465000052
:103b54000a00000041630000636500007074000007
:103b640065640000204300006f6e00007472000062
:103b74006f6c0000204300006f6d00006d61000059
:103b84006e6400000a00000053450000545f00000a
:103b9400434f00004e540000524f00004c3a0000c6
:103ba400207300006242000061730000696300003a
:103bb40052650000706c0000794500006e630000df
:103bc4006f640000650a00000053000045540000c3
:103bd4005f4300004f4e0000545200004f4c000061
:103be4003a20000073620000536500006e64000018
:103bf4004d650000737300006167000065000000fc
:103c040053450000545f0000434f00004e54000031
:103c1400524f00004c3a0000207300006253000031
:103c240065740000436f00006e740000726f000042
:103c34006c5700006974000068540000696d00004e
:103c440065730000746100006d700000446500003d
:103c5400636f0000646500000a0000005241000028
:103c6400575f0000434f00004d4d0000414e0000df
:103c7400443a0000207300006252000061770000a3
:103c8400436f00006e740000726f00006c4400000b
:103c9400656300006f640000650a000000410000d5
:103ca4006363000065700000746500006420000018
:103cb4005261000077200000436f00006d6d00002a
:103cc400616e0000640a00000052000041570000c9
:103cd4005f4300004f4d00004d4100004e44000082
:103ce4003a20000073620000426100007369000022
:103cf40063520000657000006c790000456e00009e
:103d0400636f0000646500000a0000005241000077
:103d1400575f0000434f00004d4d0000414e00002e
:103d2400443a00002073000062530000656e0000f6
:103d3400644d000065730000736100006765000056
:103d440000530000455400005f4e0000415600003f
:103d54004d4f0000444500003a200000736200000b
:103d640053650000744e0000617600004465000055
:103d7400636f0000646500000a0000005345000002
:103d8400545f00004e410000564d00004f440000b7
:103d9400453a000020730000624200006173000095
:103da4006963000052650000706c000079450000f2
:103db4006e6300006f640000650a00000053000099
:103dc400455400005f4e0000415600004d4f000076
:103dd400444500003a20000073620000536500006f
:103de4006e6400004d65000073730000616700009d
:103df400650000004163000063650000707400000a
:103e040065640000204e000061760000204d000033
:103e14006f64000065200000257300000a000000a4
:103e2400496700006e6f00007265000064200000a6
:103e34004e610000762000004d6f000064650000b4
:103e440020250000730a0000005500006e6b00007e
:103e54006e6f0000776e0000206300006f6d00003d
:103e64006d6100006e6400000a000000556e0000e1
:103e74006b6e00006f7700006e200000636f00001f
:103e84006d6d0000616e0000643a00002073000054
:103e94006242000061730000696300005265000023
:103ea400706c0000794500006e6300006f640000d0
:103eb400650a000000530000425f000058580000eb
:103ec400585800003a200000736200005365000057
:103ed4006e6400004d6500007373000061670000ac
:103ee400650000000a0d0000556e000068610000c6
:103ef4006e6400006c650000642000006d650000c5
:103f04007373000061670000652000003c25000019
:103f140030320000583e00000a0000004d730000db
:103f24006720000025300000325800003a200000cd
:103f340045720000726f000072200000636f000081
:103f44006465000020250000640a0000004d0000a4
:103f5400736700002025000030320000583a00004a
:103f64002073000075630000636500007373000034
:103f74000a000000256c0000642d000000450000cc
:103f8400727200006f7200002077000072690000f6
:103f940074740000696e000067200000504900003e
:103fa4004e0a00000d00000045720000726f000010
:103fb40072200000777200006974000074690000c8
:103fc4006e670000204e0000616d0000650a00006d
:103fd4000d000000000000000000000000000000d0
:103fe40000000000000a00000a0d000048650000ff
:103ff4006c6c00006f2c000020490000276d00004d
:104004002068000061700000707900002028000022
:1040140053450000522000004a7500006c20000047
:10402400313200002032000030310000302900001d
:104034000a0000000a0a00000d480000656c000038
:104044006c6f00002c200000492700006d20000048
:1040540068610000707000007920000028420000b0
:10406400542000004a7500006c200000313200002a
:104074002032000030310000302900000a00000026
:10408400446500006275000067200000667500004a
:104094006e630000746900006f6e00002069000008
:1040a4007320000061630000746900007661000001
:1040b40074650000642000006f6e0000207400002e
:1040c400686900007320000063680000616e0000ee
:1040d4006e6500006c0a0000004900004d550000a8
:1040e400206e00006f740000206900006e690000fb
:1040f40074690000616c000069730000656400006d
:10410400004900004d550000205200006561000088
:10411400647900003a200000626f000061720000c0
:104124006420000025380000730a0000000a000023
:104134004f730000636900006c6c00006174000040
:104144006f72000020450000727200006f72000060
:104154000a0a0000000a00004164000064720000c2
:10416400657300007320000045720000726f000048
:10417400720a00000a0000000a5300007461000083
:10418400636b000020450000727200006f72000033
:104194000a0a0000000a00004d6100007468000073
:1041a40020450000727200006f7200000a0a0000cd
:1041b40000000000204d0000616e00002e20000071
:1041c400466f00007263000065000000204d00008f
:1041d400616e00002e2000004e6f00006e6500002e
:1041e40020000000204d0000616e00002e20000021
:1041f400506f00007320000020000000204d0000dc
:10420400616e00002e200000566500006c20000046
:1042140020000000204d0000616e00002e200000f0
:10422400526500006c2000002000000020410000c6
:10423400757400006f200000466f00007263000078
:104244006500000020410000757400006f2000002c
:104254004e6f00006e650000200000002041000049
:10426400757400006f200000506f00007320000080
:104274002000000020410000757400006f20000041
:10428400566500006c200000200000002041000062
:10429400757400006f200000526500006c2000005f
:1042a40020000000436f00006e740000696e00007f
:1042b400756f000075730000004f00006e20000051
:1042c40072650000717500006573000074000000e1
:1042d400566500007274000069630000616c0000a0
:1042e400264800006f720000697a00006f6e0000bb
:1042f400746100006c0000004e6f00006e650000e9
:1043040000560000657200007469000063610000db
:104314006c000000486f0000726900007a6f0000b2
:104324006e740000616c00000052000061770000b0
:10433400204300006f6e0000747200006f6c000078
:10434400004900006e6300006f7200007265000097
:1043540063740000204e000061760000204d0000d0
:104364006f64000065000000537400006f7000006b
:1043740000490000646c0000650000005461000006
:104384006b650000204f000066660000004c0000d2
:10439400616e000064000000486f00007665000054
:1043a40072000000436f00006e740000726f000022
:1043b4006c6c00006564000000530000696e00002e
:1043c4006b6900006e670000000000004661000099
:1043d400696c000065640000207400006f20000018
:1043e400656e0000636f00006465000020680000d3
:1043f400656c0000692000007374000061740000a3
:1044040065200000300a00000046000061690000d9
:104414006c65000064200000746f000020650000db
:104424006e6300006f640000652000006865000092
:104434006c69000020730000746100007465000062
:10444400203100000a000000496e0000766100007f
:104454006c69000064200000736f00007572000036
:1044640063650000206600006f7200002073000086
:104474006574000050650000726900006f640000fc
:10448400696300005374000061740000650a000051
:1044940000000000536f00006674000077610000a4
:1044a40072650000004900006e760000616c000037
:1044b4006964000000460000726f00006d20000077
:1044c40052430000004d000065730000736100005a
:1044d400676500003a2000006964000020250000a0
:1044e40030320000582f0000253000003258000000
:1044f40020680000616e0000646c0000652000000c
:10450400256400002f250000642000006c65000075
:104514006e200000256400002f25000064200000a8
:104524005b0000002530000032580000200000002d
:104534005d200000435200004320000025300000ad
:10454400325800000a000000ac410000c43f0000e3
:10455400969e000039bc00009ebd0000e63f0000ae
:104564004e0900001a400000000000000000000096
:1045740000240000743f0000001c000022400000e2
:1045840033d700000d4000004d6100007220000090
:1045940033300000203200003031000030000000d1
:1045a40002000000100000004000000000000000b5
:0445b4000c040000f3
:020000040000fa
:1045b800881f78000004780001007800723907002d
:1045c8000001eb00428498003284980062849800cd
:1045d80052849800321498004214980080382100c0
:1045e80010149800803e2000201498006000b80045
:1045f800600c9800710c980002149800400b200081
:10460800400c980000192000300c9800a0002000f1
:10461800500c980010c0b30060449800020c780059
:10462800028c9800128c9800228c9800328c98008a
:10463800428c98004f04780000000600cf26b00096
:10464800889fbe008a9fbe008c9fbe008e1f780088
:1046580080047800010578000004eb004880980089
:104668003880980068809800588098003810980022
:10467800481098008038210090149800803e20004f
:10468800a01498006000b800e00c9800f10c9800a5
:104698008814980062082000880078000a007800d2
:1046a800f6ef07001910900060059800a910900017
:1046b80051059800085598001855980028559800f5
:1046c80038559800485598005855980068559800ee
:1046d800085d9800185d9800285d9800385d98007e
:1046e800680d9800780d980008159800181598001e
:1046f8006815980078159800081d9800181d9800ee
:1047080078059800688744000e007800c5380700cf
:10471800ee8644000d007800c23807000989900031
:104728000200e00003003200215929001000200097
:10473800020001000081eb008081eb00e2b79f00de
:10474800f3b79f00a30220008381440083bf9f002a
:1047580069099000f90990006fb29700ffb29700bd
:104768000400510085805900753e2000850f5000d7
:10477800e08f580008003600e2b79f00f3b79f00ab
:10478800098990000200e00003003200815a2900e4
:1047980010002000020001000a5190008280fb00f6
:1047a80000678000808f50001700320002407800b8
:1047b800ff27070000047800e0ccbf00fc270700b3
:1047c800881f7800801f7800405c2900801f7800cf
:1047d80000ee2f000f00400097ef070009899000b6
:1047e800e68757000200e0000400320061ee2f0067
:1047f8008f80400010002000020001000a50900045
:104808000080fb0000678800e94090000104e00098
:1048180021003200398090000000e0001e003200c4
:10482800598090000000e0001b00320009899000c8
:104838000200e00003003200e15c290020002000b3
:1048480002000100820c20008fb897000e0078004b
:10485800201807000000e0000800320009899000d5
:104868000200e00003003200115d29001000200062
:10487800020001000e0078006a3807005980900095
:104888008000e900d18498000000eb00b084980013
:1048980066033200e9409000e1cf50002100320069
:1048a800498090000000e0001e00320069809000fe
:1048b8000000e0001b003200098990000200e000bf
:1048c80003003200315d29002000200002000100b1
:1048d800820c20008fb897000d007800fd170700a4
:1048e8000000e00008003200098990000200e000a2
:1048f80003003200115d29001000200002000100b1
:104908000d00780047380700698090008000e900b2
:10491800e18498000000eb00c08498003c0332005a
:10492800e94090000104e0003a003a008085eb007d
:10493800e1cf5000550032000b00e0005600350072
:10494800ef6894000180fb00801f7800a2622900b4
:10495800821f780020ee2f000f00400036ef07007e
:1049680009899000e48757000200e0000400320043
:1049780061ee2f008f80400010002000020001002f
:104988006f689400000678000c04b200f043b2008f
:10499800e06f9c000042eb0083d82f0084f17f0079
:1049a8000080fb000100200061005000e0805800fa
:1049b800f40f5000e08f5800da023e00006001005a
:1049c80050003700d600370080003700ac003700b1
:1049d800eb0037000c0137002c0137008d0237003f
:1049e800fd013700b4023700680137004402370080
:1049f8007101370091013700460137005b0237002b
:104a080025023700920237009c013700b6013700b3
:104a1800ca013700110020000e007800fd3707009a
:104a28000000e000e8023a00098990000200e00076
:104a380003003200615d290020002000020001000f
:104a4800830c2000e2e22f000f0141008080eb0080
:104a58000e0078004d170700000478000000e00001
:104a6800fa023a00098990000200e000f4023200dc
:104a7800216029002000200002000100880578003c
:104a8800e9409000e1cf5000abff3a000b00e00096
:104a9800abff3d002eff3700110020000d0078000d
:104aa800dc3707000000e00029ff3a000989900080
:104ab8000200e000030032005161290020002000bc
:104ac80002000100830c2000e2e22f000f014100e8
:104ad8008080eb000d0078002c1707000000e00034
:104ae800e5023a00098990001b0020000200e0005e
:104af80093ff3200216029002000200002000100fd
:104b08008fff37008042eb0084d82f0005f27f002a
:104b18000004eb00b8149800098990000200e00036
:104b280003003200e18b2900100020000200010080
:104b38006f6994000274a00083d82f008f81410010
:104b480088407800a0e82f000f00400004160700f6
:104b58000000e0004e063200098990000200e000e3
:104b680003003200318d29000008200002000100f6
:104b780084d82f0064c07f000004e0002f003200ba
:104b88000080fb00801f7800cf6a94000580fb003e
:104b9800801f780000f92900801f780000ee2f00a0
:104ba8000f004000a4ee070009899000e68757002f
:104bb8000200e000e6fe320061ee2f008f80400028
:104bc8000001200002000100e1fe370019019000f9
:104bd800a28f9d00a9019000b38f9d0042d92f009c
:104be8000f0141008040eb00a0e82f000f004000bb
:104bf800311607000000e000b70232000989900072
:104c08000200e000daff3200618629000008200077
:104c180002000100098990000200e000d4ff320080
:104c2800018a2900100020000200010084d82f000a
:104c380064c07f000004e000d1ff3a00ef689400f0
:104c48000180fb00801f780092fa2900821f7800fb
:104c580020ee2f000f00400077ee07000989900032
:104c6800e48757000200e000b9fe320061ee2f0031
:104c78008f8040001000200002000100b4fe3700c1
:104c880091d82f008f804000e0e22f000f004000f5
:104c98001b130700800078000000e000ac0232001f
:104ca800098990000200e0000300320051a12900a8
:104cb8000008200002000100c0cfb30081d82f00f7
:104cc80080f07f006f6994000274a00083d82f00e1
:104cd8008f8141008040eb00a0e82f000f004000ca
:104ce8009f1507000000e000a90232000989900022
:104cf8000200e0009eff320001a329000008200006
:104d080002000100098990000200e00098ff3200cb
:104d1800a1a62900100020000200010094ff37001e
:104d28008040eb0080d82f0001f07f006f6994006d
:104d38000274a0008f014000a0e82f000f0040007f
:104d4800871507000000e00054023200098990002e
:104d58000200e00086ff3200719029000008200060
:104d680002000100098990000200e00080ff320083
:104d78001194290010002000020001007cff370078
:104d880061da2f008f804000e0e22f000f00400022
:104d9800e4120700000478000000e0000404320078
:104da800098990000200e00003003200b170290078
:104db8000008200002000100c0cfb30082d82f00f5
:104dc80000f17f006f6994000274a00083d82f005f
:104dd8008f8141008040eb00a0e82f000f004000c9
:104de8005f1507000000e000a60332000989900063
:104df8000200e0005eff32008176290000082000f2
:104e0800020001005aff3700c1d92f008f804000ef
:104e1800e0e22f000f004000d71207000000e0007a
:104e2800b6033200098990000200e0000300320056
:104e380021d129000008200002000100c0cfb300e2
:104e480085d82f0080f27f006f6994000274a0005b
:104e580083d82f008f8141008040eb00a0e82f000d
:104e68000f0040003e1507000000e000c1033200bb
:104e7800098990000200e0003dff3200f1d42900ca
:104e8800000820000200010039ff370081d92f00f7
:104e98008f804000e0e22f000f0040004913070018
:104ea800000478000000e0001e0532000989900027
:104eb8000200e0000300320091a829000008200049
:104ec80002000100c0cfb30081d82f0080f07f001e
:104ed8006f6994000274a00083d82f008f8141006d
:104ee8008040eb00a0e82f000f0040001c150700d1
:104ef8000000e00036053200098990000200e00059
:104f08001bff320071ac29000008200002000100dc
:104f180017ff37008041eb0082d82f0003f17f0094
:104f28006f6994000274a00083d82f008f8141001c
:104f38008040eb00a0e82f000f0040000815070094
:104f48000000e00030043200098990000200e0000f
:104f58000900320091952900000820000200010094
:104f6800098990000200e0000300320041972900ff
:104f78001000200002000100198890000000e000e5
:104f88000100320000000100ffff37000000eb00c5
:104f9800b01498000c00e0001c053a000989900044
:104fa8000200e000f2fe3200f16f2900100020003c
:104fb80002000100eefe3700d1d82f008f8040009c
:104fc800e0e22f000f004000f81207000000e000a8
:104fd80020053200098990000200e0000300320039
:104fe800a1c929000008200002000100c0cfb300b9
:104ff80084d82f0000f27f006f6994000274a0002b
:1050080083d82f008f8141008040eb00a0e82f005b
:105018000f004000d21407000000e000bd0132007c
:10502800098990000200e000d1fe320061cd29001c
:105038000008200002000100cdfe3700e1de2f004d
:105048008f804000e0e22f000f004000ec140700c2
:105058000000e000c6fe3a00d06f9c00098990006d
:105068000200e000c2fe3200e1de2f008f80400027
:105078001000200002000100bdfe37000a50900019
:10508800e54f500085033200d0cfb30081d82f0000
:1050980080f07f000000eb00b01498000c00e000e6
:1050a800b3fe32006f6994000274a00083d82f0009
:1050b8008f81410080407800a0e82f000f00400059
:1050c800a71407000000e000b1033200098990002e
:1050d8000200e000a6fe320061dc29000008200082
:1050e80002000100a2fe3700d83607000001780050
:1050f8008040eb00a0e82f000f004000c814070014
:105108000000e00000053200098990000200e0007c
:1051180097fe3200018129000008200002000100ea
:10512800098990000200e00091fe3200c184290044
:1051380010002000020001008dfe3700a1dd2f00c5
:105148008f804000e0e22f000f004000e7130700c7
:105158000000e0007c033200098990000200e000b2
:1051680003003200419829000008200002000100d5
:10517800c0cfb30084d82f0000f27f006f6994007d
:105188000274a00083d82f008f8141008040eb007b
:10519800a0e82f000f004000711407000000e00095
:1051a80099013200098990000200e00070fe320087
:1051b800f19a2900000820000200010009899000e6
:1051c8000200e0006afe3200f19e29001000200073
:1051d8000200010066fe37000a5490000042eb000e
:1051e80083d82f0084f17f00a1d82f008f80400042
:1051f800e0e22f000f004000f8110700800078005f
:105208000000e000c0013200098990000200e000bf
:105218000300320031ea29000008200002000100e2
:10522800c0cfb30085d82f0080f27f000000eb00cc
:10523800b01498000c00e00081023a0085d82f00d5
:10524800e5c27f000504e00024023a00a0d82f0040
:1052580060c07f000055980055250700801f780022
:10526800c2ef2900821f780020ee2f000f004000b7
:10527800f1ec070009899000e48757000200e0007c
:105288003bfe320061ee2f008f80400010002000ae
:105298000200010036fe3700398990000200e00064
:1052a800010432000f7494000804e000bd033a00c2
:1052b80001da2f008f8040000000eb00020001009f
:1052c8008001eb0002da2f000f01410088407800ce
:1052d800a0e82f000f004000471207000000e00080
:1052e800e2033200098990000200e00020fe32004b
:1052f80031b2290000082000020001001cfe37001e
:105308000a509000e74f500054013200d0cfb3004c
:1053180081d82f0080f07f000000eb00b0149800c7
:105328000c00e00012fe32006f6994000274a000c5
:1053380083d82f008f81410080407800a0e82f009b
:105348000f004000061407000000e000bf04320010
:10535800098990000200e00005fe320071e629008c
:10536800000820000200010001fe3700b1d82f001c
:105378008f804000e0e22f000f004000631107001b
:10538800800078000000e0001102320009899000d6
:105398000200e00004003200116329000008200028
:1053a8000200010009899000c0cfb30085d82f0002
:1053b80080f27f001900e000220132000200e000c4
:1053c800030032004165290010002000020001009e
:1053d8006f6994000274a00083d82f008f81410068
:1053e8008040eb00a0e82f000f004000dc1307000e
:1053f8000000e000f5003200098990000200e0009a
:10540800dbfd32008168290000082000020001004d
:10541800d7fd370001d92f008f804000e0e22f0030
:105428000f00400062110700000478000000e0004f
:1054380044043200098990000200e000ccfd3200eb
:10544800d17929000008200002000100c8fd3700ba
:10545800298990000200e000330332000f749400a1
:105468000804e000fe023a00a1dc2f008f80400013
:105478000000eb00020001008001eb00a2dc2f001d
:105488000f01410088407800a0e82f000f0040007d
:10549800241307000000e000e202320009899000ae
:1054a8000200e000b2fd320071be290000082000b1
:1054b80002000100aefd37000a509000e54f500091
:1054c80098013200d0cfb30081d82f0080f07f0040
:1054d8000000eb00b01498000c00e000a4fd3200be
:1054e8006f6994000274a00083d82f008f81410057
:1054f80080407800a0e82f000f00400098130700b4
:105508000000e000b1023200098990000200e000ca
:1055180097fd320061dc290000082000020001002c
:1055280093fd3700098990000200e0000300320073
:1055380071f229000008200002000100e0cfb3004a
:1055480085d82f0080f27f006f6994000274a00054
:105558008f8142008040eb00a0e82f000f00400040
:105568007f1307000000e0001a003200098990004c
:105578000200e0000300320081f329000008200047
:10558800020001006f6994000280fb00801f780010
:1055980043f72900831f780020ee2f000f004000fa
:1055a80025ec070009899000e48757000200e00015
:1055b8006ffd320061ee2f008f8040001000200048
:1055c800020001006afd3700e94090008085eb0089
:1055d800d7fc37006658b90000004700421f20007a
:1055e800a1e82f008f804000ba1407000000e000f7
:1055f800e4ff3200098990000200e000e1ff320078
:10560800d1f529000008200002000100ddff370065
:10561800798190001000200002000100e94090000c
:105628000104e000c1fc3200fafc370079819000e7
:105638000100780002000100e940900096fc370064
:1056480082057800e9409000b9fc37000e00780028
:10565800f4340700098990000200e000daff320004
:10566800a15e290000012000020001008085eb00f6
:10567800e9409000aefc37000d007800e9340700df
:10568800098990000200e00031fc3200a15e290087
:1056980000012000020001002dfc37006658b90007
:1056a80000004700820c2000a1e82f008f804000f6
:1056b800881407000000e000aafd32000989900064
:1056c8000200e0002afd3200719229000008200043
:1056d80002000100a3fd37006658b900000047002a
:1056e800820c2000a1e82f008f8040007914070069
:1056f8000000e00047fd3200098990000200e00048
:105708001bfd32006188290000082000020001000a
:1057180040fd37006658b90000004700820c2000a1
:10572800a1e82f008f8040006a1407000000e00005
:105738000ffd3200098990000200e0000cfd3200e4
:1057480071cf2900000820000200010008fd370081
:1057580093d82f0063c07f006340600020559800f5
:1057680084d82f0001f27f006f6994000274a000b2
:1057780083d82f008f8141008040eb00a0e82f00e4
:105788000f004000f61207000000e00057fd3a0045
:105798006658b90000004700820c2000a1e82f00dd
:1057a8008f8040004b1407000000e00055fd3200d8
:1057b800098990000200e000edfc320001a52900f3
:1057c80000082000020001004efd37006658b900ad
:1057d80000004700820c2000a1e82f008f804000c5
:1057e8003c1407000000e000e1fc32000989900049
:1057f8000200e000defc3200a16a29000008200057
:1058080002000100dafc37006658b90000004700c2
:10581800820c2000a1e82f008f8040002d14070083
:105828000000e00065fe3200098990000200e000f7
:10583800cffc3200219d2900000820000200010051
:105848005efe37000200e000e1fe3200c16629007a
:105858000001200002000100ddfe370061db2f009f
:105868008f804000e0e22f000f004000b6100700d4
:105878000000e0000e003200098990000200e000fc
:105888000300320001e329000008200002000100a3
:10589800c0cfb30083d82f0080f17f000000eb0059
:1058a800b01498000c00e000b1fc32009efe3700f6
:1058b800bf9a950025159800cf9895003115980046
:1058c8005f99950042159800ef9995005315980037
:1058d800c014980084d82f0000f27f000989900036
:1058e8000200e0008cfe320011e5290010002000c3
:1058f800020001000000eb00b01498000c00e0006a
:105908009bfc320088fe3700a2d82f0062c07f00bf
:10591800804f540048003200e34f50003a003200f4
:105928002c003e00e14f50001e00320013003600ec
:10593800e14f540005003200e44f540003003200e8
:10594800d0cfb30084d82f0000f27f0089109000d8
:10595800703e2000808f500034fe3e00a0cfb30080
:1059680081d82f0080f07f000000eb00b014980071
:105978000c00e00031fe3200b1003700e14f540066
:105988002afe3200d0cfb30083d82f0080f17f00e9
:105998000000eb00b01498000c00e00027fe320075
:1059a800a70037000804e00020fe3200e74f54004b
:1059b8001efe3200d0cfb30085d82f0080f27f00c2
:1059c8000000eb00b01498000c00e0001bfe320051
:1059d8009b003700e54f5000340032002b0039009f
:1059e800e74f50001b003200d0cfb30081d82f0002
:1059f80080f07f000000eb00b01498000c00e0007d
:105a08000efe32008e003700e74f5400ddff3e00e7
:105a18008800fb00100020000100dd00600fb200cc
:105a2800d8ff32000000eb00b01498000c00e00032
:105a380002fe32008200370083d82f0081f17f00f8
:105a48000000eb00b01498000c00e000fbfd3200f1
:105a58007b003700e14f540003003200d0cfb30081
:105a680082d82f0000f17f00211598003115980089
:105a780041159800511598000000eb00b0149800eb
:105a88000c00e000edfd32006d0037006540540069
:105a9800e14f5000c7ff3e000000eb00b014980033
:105aa8000c00e000e5fd320065003700e64f5400c9
:105ab8004f003200e44f54004d003200d0cfb30005
:105ac80082d82f0000f17f000000eb00b01498008e
:105ad8000c00e000d9fd320059003700a3d82f0090
:105ae80063c07f0032230700801f780024f129005b
:105af800841f780020ee2f000f004000ceea070038
:105b080009899000e48757000200e00018fc320081
:105b180061ee2f008f80400010002000020001007d
:105b280013fc3700e1da2f008f804000e0e22f00fd
:105b38000f004000eb0f07000000e0000e003200ed
:105b4800098990000200e00003003200b1d8290062
:105b58000008200002000100c0cfb30083d82f0046
:105b680080f17f000000eb00b01498000c00e0000a
:105b7800fffb32005afe3700ff929500650d980032
:105b88008f989500710d98001f999500021598003f
:105b9800af99950013159800c014980084d82f0069
:105ba80000f27f00098990000200e00048fe320000
:105bb800c1da290010002000020001000000eb00fb
:105bc800b01498000c00e000e9fb320044fe3700f6
:105bd800b2d82f0062c17f000280fb00800c7800e1
:105be80083d82f0081f17f0009899000f1fd3700eb
:105bf8008000eb00610d9800710d98000115980068
:105c0800111598002a589000e14f500002003a0000
:105c18004a1a9000041598003a589000e24f500034
:105c280002003a008a2a900015159800c1149800bd
:105c38000000eb00b01498000c00e0007ffd32007b
:105c48006f6994000274a00083d82f008f814100ef
:105c580080407800a0e82f000f004000c011070026
:105c68000000e00016003200098990000200e00000
:105c780072fd320001ec290000082000020001003a
:105c88006efd37006658b90000004700820c2000fe
:105c9800a1e82f008f8040000e1307000000e000ed
:105ca800b3fb3200098990000200e000b0fb32002b
:105cb800517829000008200002000100acfb3700e1
:105cc8006658b90000004700820c2000a1e82f00a8
:105cd8008f804000ff1207000000e00057fd3200ef
:105ce800098990000200e00054fd320011ee2900fd
:105cf800000820000200010050fd3700c2d92f0023
:105d080062c17f00025d9800d3d92f00e3c17f00f4
:105d1800135d9800e4d92f0064c27f00245d9800c9
:105d2800f5d92f00e5c27f00355d980081d82f0096
:105d380080f07f00098990000200e00042fc3200f8
:105d480031d3290010002000020001006f6994007f
:105d58000274a00083d82f008f8141008040eb009f
:105d6800a0e82f000f0040007d1107000000e000b0
:105d78003ffc3a006658b90000004700820c20003a
:105d8800a1e82f008f804000d21207000000e00039
:105d980077fb3200098990000200e00074fb3200b2
:105da80001d72900000820000200010070fb37001d
:105db80064da2f0064c07f006141600012559800ca
:105dc800e14f510024003a00990090005f9095003f
:105dd8000100600010059800a90090006f909500e0
:105de800010060002005980075da2f0065c07f006b
:105df8000004e00002003a000240780082f27f00ce
:105e08000081fb0072059800813e20001100090006
:105e18008200d8008000fd000b804500090040008a
:105e28004f91950052809800798190000b0078007e
:105e38000200010083d82f0088f17f0009899000b3
:105e48000200e000dffb3200517229001000200040
:105e580002000100dbfb37000b8045000900400011
:105e6800588098007805980079819000880078001b
:105e78000b0078000200010085d82f0088f27f000f
:105e8800098990000200e000cefb320071742900fd
:105e98001000200002000100cafb3700e1db2f00e0
:105ea8008f804000e0e22f000f004000ce0e070078
:105eb8000000e0000e003200098990000200e000b6
:105ec8000300320021e02900000820000200010040
:105ed800c0cfb30083d82f0080f17f000000eb0013
:105ee800b01498000c00e00021fb32006dfc370074
:105ef800ff9a9500650d98008fa09500710d980088
:105f08001fa1950002159800afa1950013159800e0
:105f1800c014980084d82f0000f27f0009899000ef
:105f28000200e0005bfc3200c1da2900100020000a
:105f3800020001000000eb00b01498000c00e00023
:105f48000bfb320057fc3700498990000200e00043
:105f58000c003200e0dd2f008f004000640050008c
:105f68000f0040000200010080c0eb000000e000cc
:105f780001003a008040780082d82f0001f17f00ac
:105f88007efc370084d82f0002f27f007bfc3700ac
:105f98006658b90000004700820c2000a1e82f00d5
:105fa8008f8040004b1207000000e000f0fa32003a
:105fb800098990000200e000edfa320071de290044
:105fc8000008200002000100e9fa37006658b9000d
:105fd80000004700820c2000a1e82f008f804000bd
:105fe8003c1207000000e000e1fa32000989900045
:105ff8000200e000defa320071de2900000820000d
:1060080002000100dafa37006658b90000004700bc
:10601800820c2000a1e82f008f8040002d1207007d
:10602800cffb37006658b90000004700820c2000fb
:10603800a1e82f008f804000261207000000e00032
:10604800cbfa3200098990000200e000c8fa320059
:1060580041c029000008200002000100c4fa3700ee
:10606800a1dc2f008f804000e0e22f000f004000ed
:106078008a1007000000e0001a0032000989900029
:106088000200e00003003200d1c12900000820000e
:1060980002000100c0cfb30084d82f0000f27f00b7
:1060a8006f6994000274a00083d82f008f8141008b
:1060b8008040eb00a0e82f000f004000a810070068
:1060c8000000e0001f003200098990000200e00093
:1060d800a7fa3200b1c72900000820000200010019
:1060e800a3fa370029899000a1dc2f008f80400097
:1060f80010002000020001000000e0002000320033
:1061080080c0eb0080d82f0001f07f000989900043
:106118000200e000e2ff320001c429000001200073
:1061280002000100deff3700098990000200e0004c
:106138008ffa3200e1bb29000001200002000100b3
:106148008bfa37006658b90000004700820c20001f
:10615800a1e82f008f804000de1107000000e0005a
:1061680083fa3200098990000200e00080fa3200c8
:1061780041c0290000082000020001007cfa370015
:1061880082d82f0000f17f00098990000200e0000a
:10619800c3ff3200c1c52900100020000200010021
:1061a800bfff370001da2f008f804000e0e22f00a8
:1061b8000f004000c20e07000000e0001a00320085
:1061c800098990000200e0000300320091b529001f
:1061d8000008200002000100c0cfb30084d82f00bf
:1061e80000f27f006f6994000274a00083d82f002a
:1061f8008f8141008040eb00a0e82f000f00400095
:10620800571007000000e0002e00320009899000b6
:106218000200e00056fa3200f1b929000008200017
:106228000200010052fa37003989900001da2f0084
:106238008f80400010002000020001000000e000f4
:106248002f00320080c0eb0080d82f0001f07f00c3
:10625800098990000200e000e2ff320061b72900de
:106268000001200002000100deff37006658b90077
:1062780000004700820c2000a1e82f008f8040001a
:10628800941107000000e00039fa320009899000f3
:106298000200e00036fa320001b4290000082000ac
:1062a8000200010032fa3700098990000200e0007c
:1062b8002ffa320031b0290000012000020001004d
:1062c8002bfa37006658b90000004700820c2000fe
:1062d800a1e82f008f8040007e1107000000e00039
:1062e80023fa3200098990000200e00020fa320007
:1062f80001b4290000082000020001001cfa370040
:1063080082d82f0000f17f00098990000200e00088
:10631800b4ff320091b829001000200002000100eb
:10632800b0ff37004f8895000000e0000100320000
:10633800a01498005f8895000000e000010032007a
:106348009014980099119000630598002912900004
:106358005405980085d82f0088f27f00ea00900045
:10636800811f78005a019000821f7800a3aa290093
:10637800831f780000ee2f000f004000aee80700f2
:1063880009899000e68757000200e0000400320007
:1063980061ee2f008f8040001000200002000100f5
:1063a800b8149800c81498006f6994000274a0008b
:1063b80083d82f008f8141008040eb00a0e82f0098
:1063c8000f004000e60f07000000e000cafa3a009c
:1063d8006658b90000004700820c2000a1e82f0091
:1063e8008f8040003b1107000000e000e0f9320018
:1063f800098990000200e000ddf9320081ae290031
:106408000008200002000100d9f937008040780018
:1064180085d82f0080f27f006f6994000274a00075
:106428008f814200a0e82f000f004000cc0f07002a
:106438000000e00025003200098990000200e00019
:10644800cbf93200616c290000082000020001002d
:10645800d2fa3700d1d82f00e1c07f00414599001a
:10646800e2d82f0062c17f005245990083d82f00df
:1064780080f17f00098990000200e000defa320016
:10648800e1cb29001000200002000100dafa3700f1
:106498006658b90000004700820c2000a1e82f00d0
:1064a8008f8040000b1107000000e000b0f93200b7
:1064b800098990000200e000adf93200018f29003f
:1064c8000008200002000100a9f937006658b90049
:1064d80000004700820c2000a1e82f008f804000b8
:1064e800fc1007000000e000acfa320009899000b7
:1064f8000200e0009ef93200516e290000082000d9
:1065080002000100a5fa37006658b90000004700ec
:10651800820c2000a1e82f008f804000ed100700ba
:106528000000e000fefa3200098990000200e00055
:106538008ff93200118329000008200002000100b1
:10654800f7fa3700990090000f8895000100600065
:10655800808f9d00a90090001f88950001006000b1
:10656800908f9d00290890000000010061f62f001f
:106578008f80400042000900ba1878006108b10015
:106588006a08b1008f899500c3379f001f8a95005c
:10659800d4379f000101780088407800a0e82f00d8
:1065a8000f004000991e07000000e00018003200ac
:1065b800098990000200e00003003200517b2900a5
:1065c80000082000020001009f8a9500851f7800be
:1065d8007f809500801f7800e17e2900811f780068
:1065e80000ee2f000f00400013e807000989900013
:1065f800e68757000200e0005df9320061ee2f00e7
:106608008f804000100020000200010058f9370078
:106618006658b90000004700820c2000a1e82f004e
:106628008f804000ab1007000000e000e6ff32005a
:10663800098990000200e000e3ff3200917d290003
:106648000008200002000100dfff37006658b9008b
:1066580000004700820c2000a1e82f008f80400036
:106668009c1007000000e00041f932000989900001
:106678000200e0003ef9320081e82900000820000d
:10668800020001003af93700889fbe008a9fbe00c9
:1066980080047800010478002008900000000100c0
:1066a800885190000382fb00e3cf51009300320031
:1066b8002a003600e5cf5100b20032008d003100cb
:1066c80099109000e18f40000300320039109000cb
:1066d800808f5000b10036000380fb00800f52000d
:1066e800030032000000eb008014980088519000ed
:1066f800285090008080fb000118a300240032007d
:10670800082890000000e900fa002000ed0f500072
:106718001f003e006180600020003a00800578007c
:1067280080027800e3cf51004b003200e3cf5100e4
:106738005b003e00e1cf510079003e000040eb00d5
:106748006054980030549800405498005054980071
:106758004f05be004f04be0000000600e1cf510007
:10676800af003200e2cf5100dbff3a008002eb00bd
:10677800b5149800390890002003b10088289000cb
:10678800808f5000be003c0088519000d2ff370037
:106798000085eb0061806000e0ff3200282a90004d
:1067a800382b9000c82b9000d82a90008400e9006c
:1067b8008005eb0040092000808f500006003e0055
:1067c80062092000040051007400b900110009009a
:1067d8000200d800800578000500e900440920007f
:1067e800840f500006003e00620920000500510099
:1067f8007400b900110009000200d8008085550016
:106808000600e9008002eb00840f500006003e00fd
:1068180062092000060051007400b9001100090047
:106828000200d8008002ea008700e9004009200041
:10683800808f5000bbff3e00620920000700510016
:106848007400b900110009000200d80080824200db
:10685800e3cf5100b5ff3a0020c0b3006054980060
:1068680010c0b30030549800405498005354980016
:1068780008289000d908900001005000101c9800ca
:106888000000eb006014980070149800001c980039
:106898004f05be004f04be0000000600afff3700e2
:1068a800e5cf5100400032002e00310010c0b30087
:1068b800305498004054980030c0b30050549800a9
:1068c8000a00e0009900340020c0b300605498002a
:1068d8001a1c9800651498007b1498000000eb00bf
:1068e800001c98004f05be004f04be0000000600c3
:1068f8009aff3700e6cf510077ff3a000000eb001f
:10690800b01498008828900049089000808f5000a3
:106918009dff3c0013c0b300035498006eff37007e
:1069280020c0b3006054980010c0b30030549800e1
:106938004054980030c0b30050549800b90c9000ef
:10694800191c98000000eb0060149800701498005f
:10695800001c98004f05be004f04be000000060052
:106968007eff3700e6cf510052003200e7cf5100da
:1069780072ff32004f05be004f04be000000060043
:1069880076ff370099109000e18f40002d0032000b
:1069980039109000808f50002a003e0063c0b30079
:1069a800035498004cff3700285890005054980022
:1069b80008109000001c98000a00e00064003400f1
:1069c80020c0b300605498001a1c98000858900022
:1069d80030549800e14f5000500032000500e000ac
:1069e80023003a0068089000601498001858900036
:1069f80040549800e14f5000410032000b00e00085
:106a08002600320010c0b300405498007b14980050
:106a18004f05be004f04be00000006004fff3700c0
:106a280099109000e18f40002bff32003910900040
:106a3800808f500028ff3e008041eb0003549800ef
:106a480025ff3700a9109000e18f400022ff320097
:106a580049109000808f50001fff3e0043c0b300d4
:106a68000354980008289000101498001aff370063
:106a780010c0b3003054980065149800dbff37004d
:106a8800335c98001114980043c0b3000354980075
:106a9800b5149800885190000fff370078089000cf
:106aa800701498004f05be004f04be000000060099
:106ab8002aff370020c0b3006054980010c0b3000c
:106ac800305498004054980030c0b3005054980097
:106ad80008289000d908900001005000101c980068
:106ae800651498007b1498000000eb00001c9800c7
:106af8004f05be004f04be000000060017ff370018
:106b08007808900000804500701498004f05be007a
:106b18004f04be000000060010ff37006808900010
:106b28000080420060149800b0ff370020c0b30016
:106b38006054980018109000101c98006514980074
:106b48007b1498000000eb00001c980065ff3700dc
:106b5800385890006054980018109000101c980045
:106b68009aff370080017800f008900060089000d4
:106b780002004000e0804800e0099800f109980010
:106b8800031090000000410080119800231090002d
:106b9800e10f400003003200c3109000810f500045
:106ba80009003e0093109000e18f4000050032007c
:106bb80033109000808f5000020036000000410022
:106bc800b01198000000060001004100c0119800b3
:106bd800f4ff37004000fa00881f780060738000d7
:106be800e20f500001003200c900370060e32000c6
:106bf800400490006140b90032eb0700601f980024
:106c0800711f98000800e00007003d000200200006
:106c1800037824006e189000fe189000cbeb070054
:106c2800601f9800711f9800a2702d0033b22300d6
:106c38006e189000fe1890008feb070042b62300f4
:106c480073fa2300c0eb0700707388008173880013
:106c580060e32000600490006140b90019eb070070
:106c6800401f9800511f98000800e00007003d00f1
:106c780002002000037824004e189000de189000cf
:106c8800b2eb0700401f9800511f9800229524007e
:106c9800d3b123004e189000de18900076eb070061
:106ca800228e2500f3f92300a7eb070090738800d4
:106cb800a173880060e32000100478006140b900e7
:106cc80000eb0700201f9800311f98000800e00023
:106cd80007003d0002002000037824002e189000d1
:106ce800be18900099eb0700201f9800311f9800ec
:106cf800324c2600a3aa23002e189000be1890003c
:106d08005deb0700f2482e0023df23008eeb07001f
:106d1800b0738800c173880060e3200020049000ed
:106d28006140b900e7ea0700001f9800111f9800aa
:106d38000800e00007003d0002002000037824005e
:106d48000e1890009e18900080eb0700001f980016
:106d5800111f9800a2702d0033b223000e18900066
:106d68009e18900044eb070082b72000c3fa230066
:106d780075eb0700d0738800e173880060e320009a
:106d8800500490006140b900ceea070060179800ef
:106d9800711798000800e00007003d00020020007d
:106da800037824006e109000fe10900067eb070037
:106db8006017980071179800324c2600a3b2230080
:106dc8006e109000fe1090002beb0700721b2d0038
:106dd80003fb23005ceb0700f07388000174880054
:106de80060e32000700490006140b900b5ea070034
:106df80040179800511798000800e00007003d0070
:106e080002002000037824004e109000de1090004d
:106e18004eeb07004017980051179800a2702d00fc
:106e280033b223004e109000de10900012eb0700e2
:106e380092e4220073fa230043eb070010748800e1
:106e48002174880060e32000100490006140b900bc
:106e58009cea070020179800311798000800e00006
:106e680007003d0002002000037824002e10900047
:106e7800be10900035eb07002017980031179800d6
:106e8800324c2600a3aa23002e109000be109000ba
:106e9800f9ea0700a24e200043e323002aeb07008b
:106ea800307488004174880060e32000300490004a
:106eb8006140b90083ea070000179800111798008d
:106ec8000800e00007003d000200200003782400cd
:106ed8000e1090009e1090001ceb07000017980001
:106ee80011179800324c2600a3b223000e10900010
:106ef8009e109000e0ea0700a29b2400c3fa23003a
:106f080011eb07005074880061748800c4003700d2
:106f180060e32000100478006140b90069ea0700c6
:106f2800600f9800710f98000800e00007003d000e
:106f380002002000037824006e089000fe089000ec
:106f480002eb0700600f9800710f9800a2702d00e7
:106f580033b223006e089000fe089000c6ea0700ce
:106f680042b6230073fa2300f7ea0700707388001b
:106f78008173880060e32000200490006140b9001c
:106f880050ea0700400f9800510f98000800e000f1
:106f980007003d0002002000037824004e089000fe
:106fa800de089000e9ea0700400f9800510f9800aa
:106fb80022952400d3b123004e089000de089000eb
:106fc800adea0700228e2500f3f92300deea070068
:106fd80090738800a173880060e32000400490004b
:106fe8006140b90037ea0700200f9800310f980078
:106ff8000800e00007003d0002002000037824009c
:107008002e089000be089000d0ea0700200f9800d4
:10701800310f9800324c2600a3aa23002e089000b6
:10702800be08900094ea0700f2482e0023df2300f0
:10703800c5ea0700b0738800c173880060e32000c8
:10704800600490006140b9001eea0700000f980034
:10705800110f98000800e00007003d000200200022
:10706800037824000e0890009e089000b7ea0700f5
:10707800000f9800110f9800a2702d0033b2230062
:107088000e0890009e0890007bea070082b7200057
:10709800c3fa2300acea0700d0738800e1738800c4
:1070a80060e32000100490006140b90005ea070081
:1070b80060079800710798000800e00007003d008d
:1070c80002002000037824006e009000fe0090006b
:1070d8009eea07006007980071079800324c260066
:1070e800a3b223006e009000fe00900062ea070041
:1070f800721b2d0003fb230093ea0700f07388003e
:107108000174880060e32000300490006140b900f9
:10711800ece9070040079800510798000800e000d4
:1071280007003d0002002000037824004e00900074
:10713800de00900085ea0700400798005107980094
:10714800a2702d0033b223004e009000de009000a4
:1071580049ea070092e4220073fa23007aea07005a
:10716800107488002174880060e3200050049000a7
:107178006140b900d3e9070020079800310798005b
:107188000800e00007003d0002002000037824000a
:107198002e009000be0090006cea070020079800bf
:1071a80031079800324c2600a3aa23002e00900035
:1071b800be00900030ea0700a24e200043e32300ff
:1071c80061ea0700307488004174880060e3200099
:1071d800700490006140b900bae90700008fbe0052
:1071e8000800e00005003d000200200003782400ac
:1071f8001e00be0055ea0700008fbe00324c260074
:10720800a3b223001e00be001bea0700a29b2400b5
:10721800c3fa23004cea07005074880061748800a0
:1072280070738000817380000200200003f823003f
:10723800a3ea07000000e00001003c000500370059
:107248000000200001f82300707388008173880013
:107258000c003700707380008173800002002000ea
:1072680003f82b0098ea07000000e0000100350051
:10727800040037000000200001f82b00707388001c
:107288008173880090738000a17380000200200041
:1072980003f823008aea07000000e00001003c0030
:1072a800050037000000200001f8230090738800d3
:1072b800a17388000c00370090738000a1738000d0
:1072c8000200200003f82b007fea07000000e0001e
:1072d80001003500040037000000200001f82b00f1
:1072e80090738800a1738800b0738000c173800018
:1072f8000200200003f8230071ea07000000e00004
:1073080001003c00050037000000200001f82300c0
:10731800b0738800c17388000a003700b07380001a
:10732800c17380006011b80067ea07000000e00040
:1073380001003500030037006000b800b073880012
:10734800c1738800d0738000e173800002002000c0
:1073580003f823005aea07000000e00001003c009f
:10736800050037000000200001f82300d0738800d2
:10737800e17388000c003700d0738000e17380004f
:107388000200200003f82b004fea07000000e0008d
:1073980001003500040037000000200001f82b0030
:1073a800d0738800e1738800f07380000174800056
:1073b8000200200003f8230041ea07000000e00073
:1073c80001003c00050037000000200001f8230000
:1073d800f0738800017488000c003700f073800097
:1073e800017480000200200003f82b0036ea070031
:1073f8000000e00001003500040037000000200014
:1074080001f82b00f0738800017488001074800064
:10741800217480000200200003f8230028ea0700f6
:107428000000e00001003c000500370000002000db
:1074380001f8230010748800217488000c003700bc
:1074480010748000217480000200200003f82b00d3
:107458001dea07000000e0000100350004003700c5
:107468000000200001f82b001074880021748800a7
:1074780030748000417480000200200003f823006b
:107488000fea07000000e00001003c00050037009b
:107498000000200001f8230030748800417488003f
:1074a8000a00370030748000417480006011b80011
:1074b80005ea07000000e00001003500030037007e
:1074c8006000b800307488004174880050748000ef
:1074d800617480000200200003f82300f8e9070027
:1074e8000000e00001003c0005003700000020001b
:1074f80001f8230050748800617488000c0037007c
:1075080050748000617480000200200003f82b0092
:10751800ede907000000e000010035000400370035
:107528000000200001f82b00507488006174880066
:107538004f0478000080fa00000006008400fa007a
:107548000040eb0010479800d702a80000c42900ab
:1075580001002000d92e0700d702a90000c4290085
:1075680001002000d52e070010c8b300204798005e
:1075780000c1b300104798009e4090002e40900034
:10758800d82a070020c8b300204798000040eb0025
:10759800104798009e4090002e409000d12a070086
:1075a80030c8b30020479800f0c2b30010479800d5
:1075b8009e4090002e409000ca2a070060c8b30081
:1075c80020479800a0c4b300104798009e40900040
:1075d8002e409000c32a070070c8b30020479800c7
:1075e8000040eb00104798009e4090002e4090000d
:1075f800bc2a0700b0c8b300204798000040eb0041
:10760800104798009e4090002e409000b52a070031
:10761800c0c8b3002047980040c0b3001047980086
:107628009e4090002e409000ae2a0700d0c8b300bc
:107638002047980010c4b300104798009e4090005f
:107648002e409000a72a0700e0c8b3002047980002
:107658000040eb00104798009e4090002e4090009c
:10766800a02a070000c9b30020479800e0ceb30065
:10767800104798009e4090002e409000992a0700dd
:10768800b0c9b3002047980050c5b3001047980010
:107698009e4090002e409000922a0700c0c9b30077
:1076a8002047980050c0b300104798009e409000b3
:1076b8002e4090008b2a0700d0c9b30020479800bd
:1076c80080c1b300104798009e4090002e40900063
:1076d800842a070020cbb30020479800c0c3b3001a
:1076e800104798009e4090002e4090007d2a070089
:1076f80050cbb3002047980040c1b3001047980012
:107708009e4090002e409000762a0700e0c9b30002
:107718002047980000c9b300104798009e40900089
:107728002e4090006f2a0700f0c9b3002047980048
:107738000040eb00104798009e4090002e409000bb
:10774800682a0700f0c8b30020479800c0c2b300f9
:10775800104798009e4090002e409000612a070034
:1077680080cab3002047980020c0b3001047980093
:107778009e4090002e4090005a2a070070cab3001d
:107788002047980020c0b300104798009e40900002
:107798002e409000532a070020cab30020479800c3
:1077a8008f87e80090c4b300e0ff9f0017ccb300b8
:1077b800f6cdb30025c6b30094c4b30003ccb30020
:1077c80012cbb300f1cdb3002e409000552a07002c
:1077d8008f87e900f0c8b30020479800c0c0b30005
:1077e800104798009e4090002e4090003d2a0700c8
:1077f80010c4b3002047980000c1b300004f7800c0
:10780800e30047001e4178002e409000882a0700b8
:10781800d0c5b3002047980030c0b300004f7800af
:10782800e30047001e4178002e409000802a0700a0
:1078380060c6b3002047980030c0b300004f7800fe
:10784800e30047001e4178002e409000782a070088
:1078580020c7b3002047980010c0b300004f78003d
:10786800e30047001e4178002e409000702a070070
:1078780050c7b3002047980010c0b300004f7800ed
:10788800e30047001e4178002e409000682a070058
:107898000000eb00507a88000000eb00607a880056
:1078a8000080fa00000006006800fa000040eb00c3
:1078b80030479800f0c4b300004f78000040eb0058
:1078c800104798000040eb00204798000040eb006c
:1078d80050479800a1c0b30060c8b300012a070050
:1078e8005b0037000040eb00104798000040eb00b9
:1078f8004047980053003700ce40900000c8b300be
:10790800f829070001c2b30090cab300f52907009f
:10791800c1c2b300f0c8b300f2290700e60047006f
:1079280012c0b30090c0b300412a07006e41900016
:10793800e800470010c2b3003d2a0700c1c0b300e9
:10794800f0c8b300e72907008040eb0090cab300f5
:10795800e4290700e700470012c0b30070c0b30075
:10796800332a070001c4b300d0c8b300dd290700db
:1079780001c8b30050c8b300da2907007106200017
:107988008e80400012c0b30070c0b300282a0700e0
:107998000b003700710620008e80400012c0b30033
:1079a80070c0b300222a070000fa2000010020005e
:1079b800c22d07003e4090000040e8003047980084
:1079c8007ee090000080fb004600de000000a20080
:1079d800610060000004a2000004e00004003a0016
:1079e800be40900060c9b30080cf5000e9ff360068
:1079f800e500470012c0b30030c1b3000c2a0700ed
:107a08000040eb00304798004e4090008080fb001b
:107a18005e4190007800470001004000024878006d
:107a28005e4090000004e00003003d001e4090000e
:107a38000040e800104798004e4090000040e800e1
:107a4800404798004e4090009e4f5000aaff3900d2
:107a58001e409000e24f5000a2ff3600a1c4b300c0
:107a680060c8b3009f2907007800470010407800dd
:107a7800704798000040eb0040479800140037001a
:107a88004e4090008080fb007800470001004000d5
:107a9800904078007e40900080cf50000900390067
:107aa8004e4090008080fb007800470001004000b5
:107ab800104078007047980080e62000ce40900083
:107ac800014878004e4090000040e8004047980088
:107ad8004e4090009e4f5000e9ff390080e620009c
:107ae800104078008080fb0078004700810040004b
:107af8000040eb008048780078004700104078008c
:107b0800704798000040eb00404798001400370089
:107b18004e4090008080fb00780047000100400044
:107b2800904078007e40900080cf500009003900d6
:107b38004e4090008080fb00780047000100400024
:107b4800104078007047980080e62000ce409000f2
:107b5800114098004e4090000040e80040479800cf
:107b68004e4090009e4f5000e9ff390080e620000b
:107b7800104090008080fb007800470081004000a2
:107b88000040eb00804878007800470010407800fb
:107b9800704798000040eb004047980014003700f9
:107ba8004e4090008080fb007800470001004000b4
:107bb800904078007e40900080cf50000900390046
:107bc8004e4090008080fb00780047000100400094
:107bd800104078007047980080e62000ce40900062
:107be800214098004e4090000040e800404798002f
:107bf8004e4090009e4f5000e9ff390080e620007b
:107c08009040780080e620001040900080cf50001f
:107c18000a00360080e6200010407800704798007f
:107c280080e620009040900080e62000014878001f
:107c3800fe40900080e620001140980080e6200079
:107c48009040900080e620002040900080cf5000b7
:107c58000a00360080e62000104090007047980027
:107c680080e62000a040900080e6200011409800a7
:107c7800fe40900080e620002140980080e6200029
:107c88009040780080e620001040900080cf50009f
:107c98000a00360080e620001040780070479800ff
:107ca80080e620009040900080e62000014878009f
:107cb800fe40900080e620001140980080e62000f9
:107cc8009040780000c8b3000629070001c2b3003d
:107cd80090cab30003290700c1c2b300f0c8b300bb
:107ce80000290700e600470012c0b30090c0b300a7
:107cf8004f2907006e419000e800470010c2b3000a
:107d08004b290700c1c0b300f0c8b300f52807002d
:107d18008040eb0090cab300f2280700e700470054
:107d280012c0b30070c0b3004129070001c4b300fa
:107d3800d0c8b300eb28070001c8b30050c8b3008f
:107d4800e82807000080fa00000006000800fa0092
:107d580060e22000404090000080fb00100798007f
:107d68001e009000000f780060e2200010407800ac
:107d78000080fb002007980060e22000104090007f
:107d88000080fb00300798009e009000000c200047
:107d9800008060004200dd0010079800000320000a
:107da8001e0060004400dd00000f78009e00900077
:107db8002e0090008080400060e3200001087800d9
:107dc8003e0090009e00400060e3200011009800f3
:107dd80060e22000404090000080fb0010079800ff
:107de8009e009000010f780060e220002040900083
:107df8000080fb002007980060e2200030409000df
:107e08000080fb00300798001e0090006c006000a6
:107e18004600dd00100798009e007800638060002f
:107e28004800dd00000f78009e0090002e009000b2
:107e38008080400060e32000210098003e00900010
:107e48009e00400060e320003100980060e22000be
:107e5800104890000080fb00100798001e0090005a
:107e6800000f780060e22000504090000080fb0086
:107e78002007980060e22000604090000080fb002e
:107e8800300798009e009000000c200000806000e1
:107e98004200dd0010079800000320001e0060006b
:107ea8004400dd00000f78009e0090002e00900036
:107eb8008080400060e32000410098003e00900070
:107ec8009e00400060e320005100980060e220001e
:107ed800104890000080fb00100798009e0090005a
:107ee800010f780060e22000704090000080fb00e5
:107ef8002007980060e22000004890000080fb0006
:107f0800300798001e0090006c0060004600dd00fd
:107f1800100798009e007800638060004800dd002c
:107f2800000f78009e0090002e0090008080400096
:107f380060e32000610098003e0090009e00400031
:107f480060e32000710098000080fa00000006003d
:107f58000800fa00881f78000040eb00004f780006
:107f6800440037001e80fb00300798001e80fb008d
:107f780061e3200000004000610478006140b9001e
:107f880050e6070010079800210798000800e00055
:107f980007003d0002002000037824001e00900026
:107fa800ae009000e9e60700100798002107980046
:107fb80002002000833424001e009000ae009000d0
:107fc800e1e60700020020006341240068e607009c
:107fd8000001be0061e420003e0290004220dd0066
:107fe800010040000288be001e80fb0061e4200002
:107ff8004200dd00008040001000be006011b800a3
:1080080031e707000000e0000100350006003700f6
:108018001e80fb0061e420004200dd0001014000f9
:108028006000b8000089be001e80fb0061e42000eb
:108038004200dd00008040001000be000200200069
:1080480003f823001ee707000000e00001003c00e1
:10805800070037001e80fb0061e420004200dd00bd
:10806800010140000000200001f823000089be0043
:108078001e4fe80070c0b3009e4f1000b9ff3600d5
:108088004f0478000080fa00000006000000fa00a3
:108098006d29070082290700d702a800e922a80055
:1080a8000000eb003073880024fd0700fefd070088
:1080b800762907000000eb000080fa0000000600a7
:1080c8003600f800809fbe00829fbe00849fbe00dd
:1080d800869fbe001200fa000040eb00004f7800b7
:1080e8000040eb00104798009460a9000040eb00a6
:1080f800104798000040eb00004f7800507a80004d
:108108000000e800507a8800607a80000000e800eb
:10811800607a880012c0b3008e00780070c0b30087
:10812800432807001e4078008080fb00500820008c
:10813800008060000000e0001a00320001c2b300b5
:1081480090cab300e7270700c1c2b300f0c8b30064
:10815800e42707008e00e80012c0b30090c0b30007
:10816800332807001e4190008e80e80010c2b3003b
:108178002f280700c1c0b300f0c8b300d9270700f3
:108188008040eb0090cab300d627070001c8b300af
:1081980070c8b300d327070021c8b30050c8b30084
:1081a800d02707009e407800a0c3b30080cf5000be
:1081b80022003a000000eb00507a88000000eb0033
:1081c800607a88008e00e80012c0b30090c0b30047
:1081d800172807001e41900061e2200010c2b3007a
:1081e8001328070060e22000404890000080fb0050
:1081f80063006000e30f50000d003a003073800008
:108208000000e8003073880030738000e30f5000ee
:1082180002003a000000eb003073880030738000e1
:1082280081e62000e140780000c8b300ad270700d0
:1082380021c8b30050c8b300aa270700517a8000ac
:10824800700c2000808f50001200360030738000c0
:108258000000e90030738800307380000000e000ff
:1082680002003d0020002000307388003173800038
:1082780080e62000e0c0780000c8b3009927070016
:1082880021c8b30050c8b300962707000000eb00d0
:10829800507a8800617a8000f07c2000808f50003e
:1082a80010003600d702a80000c4290001002000f1
:1082b800822b0700d702a80000c429000100200073
:1082c8007e2b07000000eb00307388009bfc070042
:1082d80075fd07000000eb00507a88000000eb00f5
:1082e800607a880099fe07003afa07008460a900be
:1082f8009460a8000080fa004f03be004f02be0041
:108308004f01be004f00be003600f90000400600d5
:108318000200fa00000f7800200020009e0f1000d5
:1083280002003e001e007800607388000080fa009a
:10833800000006000000fa00607380000080fa0068
:10834800000006000000fa0082ce20006000b8009d
:10835800602198007121980082ce20006000b8004a
:10836800002998001129980082ce20006000b800ea
:10837800402998005129980082ce20006000b8005a
:10838800003998001139980082ce20006000b800aa
:10839800203998003139980082ce20006000b8005a
:1083a80060399800713998000080fa0000000600d2
:1083b8000200fa00000f780081ce20001002200091
:1083c800a000980080ce2000a000900080ce200061
:1083d8003100980081ce20000000eb00c00098001a
:1083e80081ce20000000eb00e000980082ce200043
:1083f8006000b800401998005119980082ce2000fa
:108408006000b800601998007119980082ce2000a9
:108418006000b800002198001121980082ce200049
:108428006000b800202198003121980081ce2000fa
:108438000000eb00f000980081ce20000000eb0067
:108448008008980081ce20000080eb00800878002a
:1084580081ce20000080eb009000980081ce2000a3
:108468000000eb008088980081ce200010002000da
:108478009088980082ce20006000b800208998007b
:108488003189980081ce20000000eb00c088980058
:1084980081ce200010002000d088980082ce2000d5
:1084a8006000b800608998007189980081ce20002a
:1084b8000000eb008090980081ce20001000200082
:1084c8009090980082ce20006000b800209198001b
:1084d8003191980081ce20000000eb00c0909800f8
:1084e80081ce200010002000d090980082ce20007d
:1084f8006000b800609198007191980082ce2000c9
:10850800a0702d0031c2230010099800210998009d
:1085180082ce2000000020000112240030099800bb
:108528004109980082ce20006000b80050099800e8
:108538006109980082ce20006000b80010119800f0
:108548002111980082ce20006000b80030119800f8
:108558004111980082ce20000000200001fc230079
:10856800501198006111980082ce20000000200070
:1085780001082400701198000119980082ce20008b
:108588003033230031eb2300700998000111980063
:1085980081ce2000800c20009018980081ce200009
:1085a80040062000b018980081ce2000803e2000b0
:1085b800a018980082ce20006000b8000031980012
:1085c8001131980082ce20006000b8002031980058
:1085d8003131980082ce20006000b8004031980008
:1085e8005131980082ce20006000b80020819800a8
:1085f8003181980082ce20006000b8004081980048
:108608005181980082ce20006000b80060819800f7
:108618007181980081ce20000000eb0080989800be
:1086280081ce20000000eb009098980045ff0700dd
:108638001e00e000040032009e00780080ce20007a
:108648000100010001003700e4290700260d07009a
:108658000080fa00000006000e00fa0080ce20001c
:10866800a000900080ce200030009000808f500045
:1086780010003a0080ce2000100078008000e8004a
:1086880080ce20000108780080ce2000900078007d
:1086980080ce200020189000808f50000c003400fd
:1086a80080ce2000a018900080ce2000010878001d
:1086b8000700370081ce20000000eb00800878001a
:1086c80080ce2000a000900080ce200031009800cd
:1086d80080ce2000200090006f006000e20f500064
:1086e80010003a0080ce2000100090008000e800c2
:1086f80080ce20001100980080ce200090009000cd
:1087080080ce200020189000808f50000800340090
:1087180080ce2000a018900080ce20001100980084
:108728000300370081ce20000000eb009000980085
:108738002d0d07001007980080ce2000000890003b
:108748000000e000050032001e0090000000e0007c
:1087580002003a00100020001007980080ce200088
:10876800200090006f006000e20f500012003200fd
:108778001e00900060079800ee009000e18f500006
:10878800090032006e019000e20f51000100320032
:1087980009003700caa2a80081ce200010002000de
:1087a80080089800d4003700caa2a80081ce200013
:1087b80010002000800898000000eb00000f7800ef
:1087c80080ce2000a0009000000f20008080600074
:1087d8005107980000022000de009000808f5000b2
:1087e80008003200000420005e019000800f510054
:1087f800140032005e009000f00f5000310032008b
:108808003f0037003074800041748000d2cc2c00c7
:10881800c3f423002ae507000000e00001003c0043
:108828003700370080ce200020009000ef00600065
:10883800000420008080700080ce20002100980075
:108848002f00370080ce20009000780080ce2000d6
:1088580030189000808f500012003d003074800066
:1088680041748000d2cc2c00c3e4230016e5070035
:108878000000e000010035002100370080ce200014
:1088880020009000ef00600000022000808070004f
:1088980080ce20002100980010002000000f7800f2
:1088a8001700370080ce2000200090006f00600085
:1088b800800078000140a00080ce200021009800b0
:1088c8000f0037003074800041748000d2cc2c0037
:1088d800c3e42300fce407000000e00001003500c9
:1088e8000700370080ce200020009000ef006000d5
:1088f800000220008080700080ce200021009800b7
:108908001e00e0004400320080ce2000a00090004d
:10891800000f20008080600000022000808f50003f
:108928003d003a0080ce2000200090006f006000db
:1089380040079800ce009000e28f500012003200ed
:108948004e019000e20f510004003e004e009000de
:10895800e10f5000080032002f003700ce009000d1
:10896800e48f5000290032004e019000e80f5100ba
:10897800260032002800370081ce20002002200087
:10898800a00098002400370080ce200090009000be
:1089980080ce200010189000808f50001e003400f8
:1089a800b0738000c1738000d2cc2c00c3e42300d4
:1089b800c5e407000000e00001003500160037009c
:1089c80081ce200040022000a0009800d0738000d3
:1089d800e17380000001eb003207980002002000dc
:1089e80003f02300b6e407000000e00001003c00ab
:1089f80002003700100020003007980080ce2000c9
:108a0800be009000610098000300370081ce20006e
:108a180020022000a000980080ce2000a000900036
:108a280020022000808f500009003a0080ce2000ec
:108a38009000900080ce200020189000808f500079
:108a480003003a0081ce200010022000a000980008
:108a580080ce2000a0009000000f200080806000e1
:108a680021079800000220002e019000800f51007d
:108a78001500320000042000ae009000808f5000e6
:108a8800110032002e019000f00f51000100320059
:108a98001900370081ce200010002000808898003f
:108aa80081ce200010002000c088980081ce2000d0
:108ab800100020008090980081ce20001000200037
:108ac800c09098000c00370081ce20000000eb0019
:108ad8008088980081ce20000000eb00c0889800b4
:108ae80081ce20000000eb008090980081ce20000d
:108af8000000eb00c09098000080fa00000006001b
:108b08000c00fa00000f78001e0078006f0f60005c
:108b180080ce2000a0009000000f200000806000a0
:108b2800f00f5000030032000080eb00200798008f
:108b38008200370080ce2000200090006f00600087
:108b48009e0f500003003a000000eb002007980039
:108b58007a00370080ce2000000890000000e00076
:108b6800170032001e007800300798003e00900081
:108b7800e40f5000070032003e009000e80f50005c
:108b8800040032003e009000e20f50000400320062
:108b98000b0037000000eb00200798006700370043
:108ba80080ce2000200090006f006000e10f500090
:108bb80003003a000000eb00200798005f00370030
:108bc80080ce2000200090006f0060001007980001
:108bd8001e009000e20f50002c0032001e00900092
:108be800e20f500004003e001e009000e10f50000c
:108bf800120032004c0037001e009000e40f5000b5
:108c08003f0032001e009000e80f500001003200c3
:108c1800450037001e007800e10f500001003200c7
:108c28000300370081ce200010012000a00098002a
:108c38000080eb0020079800400037001e007800f5
:108c4800400798004e009000e20f500004003200e8
:108c58004e009000e80f5000050032000800370071
:108c680081ce200020012000a000980031003700ac
:108c780081ce200080012000a00098002d00370040
:108c88000080eb00200798002c0037001e007800b9
:108c9800500798005e009000e10f50000400320079
:108ca8005e009000e40f500005003200110037000c
:108cb80081ce200010012000a00098001d00370080
:108cc80080ce20009000900080ce200010189000e8
:108cd800808f50000400340081ce20004001200025
:108ce800a00098001300370010002000200798000b
:108cf800120037000080eb00200798000f003700b3
:108d08001e0078000000e900e10f500003003e005b
:108d180081ce200020012000a00098000080eb00f8
:108d280020079800050037000080eb002007980016
:108d3800020037000000eb00200798002e0090008a
:108d48000080fa00000006002000fa00881f780062
:108d58006000b80060079800710798006000b800cc
:108d680040079800510798006000b8002007980055
:108d78003107980080ce2000600090000000e000dd
:108d88002d00320082ce20006000b8000039980023
:108d98001139980082ce20006000b8002039980070
:108da8003139980082ce20006000b8006039980000
:108db8007139980080ce2000509090000000e000ab
:108dc80004003a0080ce2000409090000000e000af
:108dd80005003a00b0738000c173800082ce200085
:108de800609198007191980080ce20006091900069
:108df800f0919000220798003307980080ce200059
:108e080080109000700890002e019000be01900024
:108e1800abe307000000e00001003c00ee00370073
:108e280080ce2000700990008011900022079800e1
:108e380033079800e800370080ce2000509090005b
:108e48000000e00004003a0080ce2000409090002e
:108e58000000e0000c003a0081ce20000000eb008a
:108e6800c000980080ce2000e010900050109000c4
:108e7800b2738000c3738000ffe2070082ce200037
:108e8800609198007191980080ce200060929000c7
:108e9800f092900080ce200050119000e0119000d8
:108ea8000400be0086e307000000e00001003c006b
:108eb8000600370080ce2000e0109000501090008f
:108ec80082ce2000609198007191980080ce200099
:108ed80060929000f092900080ce200030119000b7
:108ee800c01190000400be0077e307000000e00016
:108ef800010035000600370080ce2000c010900029
:108f08003010900082ce20006091980071919800f6
:108f180080ce2000c000900080ce2000500090003d
:108f2800808f50001000320082ce20006000b80010
:108f3800003998001139980082ce20006000b800ee
:108f4800203998003139980082ce20006000b8009e
:108f5800603998007139980080ce2000c0009000d8
:108f680080ce20005100980080ce20004000900064
:108f78000000e00006003200e0d9200060119000f7
:108f8800f0119000620798007307980005003700f9
:108f9800e0d9200040119000d0119000620798009d
:108fa8007307980080ce2000801890007010900001
:108fb8006e019000fe01900043e307000000e0000e
:108fc800010035000500370080ce200070119000a8
:108fd80080199000620798007307980080ce2000df
:108fe800c0109000301090006e019000fe019000bb
:108ff80033e307000000e00001003c0005003700f3
:1090080080ce200030119000c011900062079800b7
:109018007307980080ce2000f09090006090900038
:109028006e019000fe019000c7e2070082ce20008a
:10903800603198007131980080ce2000100a9000ad
:10904800a00a900080ce200000399000903990004e
:1090580080ce2000f030900060309000d6cc2c00fc
:10906800c7dc2300ce19070082ce200060319800ab
:109078007131980022852b00e3e9230040d52000b8
:109088006f1b070080ce200010099000a0099000f7
:1090980040d52000371a070094c22500f5d82300d0
:1090a80092c22500f3d82b0040d52000401b0700b2
:1090b80080ce2000203a9000b03a900080ce200068
:1090c80050099000e00990000400be009fe20700ec
:1090d80082ce2000203998003139980080ce2000b7
:1090e800b038900020389000600f9800710f9800f9
:1090f80080ce2000209c90006140b900f1e107007b
:10910800400f9800510f98000800e00007003d004c
:1091180002002000037824004e089000de0890002a
:109128008ae20700400f9800510f98004e099000fe
:10913800de09900000002500316424000ce20700dd
:109148000001be006e089000fe0890004ae2070089
:1091580082ce2000203998003139980080ce200036
:10916800b0389000203890000200200003f8230057
:10917800d3e207000000e00001003c0005003700d2
:1091880082ce20000000200001f82300203998003a
:109198003139980080ce2000b038900020389000f7
:1091a8006011b800c8e207000000e00001003500c7
:1091b8000400370082ce20006000b80020399800f3
:1091c8003139980080ce200020399000b0399000c5
:1091d800220798003307980080ce20001090900056
:1091e8000000e00004003a0080ce200000909000cb
:1091f8000000e0001b003a00d0738000e17380009b
:1092080001f0a200008fbe00a299290093e12b0073
:109218001e00be00aae207000000e00001003c00ba
:1092280009003700a299290093e123001e00be001f
:10923800a5e207000000e000010035000200370049
:109248006000b800008fbe001e00be0002002000b3
:109258000304240008e2070082ce20002091980031
:1092680031919800e0d9200060199000f019900021
:109278004207980053079800020020006339240031
:109288004e009000de0090008de207000000e00034
:1092980001003c0004003700000020006139240070
:1092a80040079800510798000200200063392c00fd
:1092b8004e009000de00900083e207000000e0000e
:1092c80001003500040037000000200061392c003f
:1092d80040079800510798004e009000de0090006b
:1092e800850a0700400798005107980080ce2000a3
:1092f800b0909000209090004e019000de01900008
:1093080011e2070082ce20004021980051219800e8
:1093180080ce200010099000a009900000d3200002
:10932800291a0700f4282c0055df2300f2282c0006
:1093380053df2b0000d320009d1a070080ce2000a9
:109348009028900000289000200f9800310f980076
:1093580080ce2000209c90006140b90059e10700b0
:10936800000f9800110f98000800e00007003d006a
:1093780002002000037824000e0890009e08900048
:10938800f2e10700000f9800110f98000e099000f5
:109398009e099000000025003164240074e1070054
:1093a8000001be002e089000be089000b2e1070040
:1093b80082ce2000002998001129980080ce200034
:1093c8009028900000289000d2cc2c00c3ec2300f9
:1093d8003be207000000e00001003c000500370008
:1093e80082ce2000d0cc2c00c1ec230000299800ac
:1093f8001129980080ce2000902890000028900025
:10940800d2cc2c00c3ec2b002fe207000000e000b8
:10941800010035000500370082ce2000d0cc2c009a
:10942800c1ec2b00002998001129980080ce20005b
:10943800a0109000101090002e019000be01900026
:109448008de107000001be002e009000be009000d4
:10945800bde107000002be0080ce20000029900078
:10946800902990000400be00b8e1070082ce2000d9
:10947800401998005119980080ce20002e019000c4
:10948800be0190006218980073189800507480000c
:1094980061748000d2cc2c00c3f4230008e20700da
:1094a8000000e00001003c00050037006011b80032
:1094b8006000b80073220700a2fb0700070037000e
:1094c80080ce200060199000f019900080ce200016
:1094d800d0189000401890006a22070080ce200023
:1094e800108890000000e00004003a0080ce2000c0
:1094f800008890000000e0000e003a001074800020
:1095080021748000d2cc2c00c3e423005ae1070068
:109518000002be0090738000a17380000001be00ad
:109528000400be0089e1070082ce2000208998004f
:109538003189980080ce2000508890000000e0001b
:1095480004003a0080ce2000408890000000e0002f
:109558000f003a00f073800001748000d2cc2c0018
:10956800c3e4230044e107000002be0070738000da
:10957800817380000001be000400be0073e1070093
:1095880001f0a20082ce20006089980071899800bd
:1095980080ce200060899000f089900080ce200065
:1095a800b088900020889000772207004f04780048
:1095b8000080fa00000006003600f800809fbe0018
:1095c800829fbe00849fbe00869fbe003400f800c4
:1095d80000c0b300a00188000200fa00d5c2bf0095
:1095e800684060000004e00013003200306780002b
:1095f800212d2a0000004000e1007800d0168500e7
:1096080000807000980e0700306780000000e800b6
:109618003067880030678000212d2a000000400054
:10962800610078000000e00007003a000000eb004d
:10963800306788000400370081ce20001000200029
:10964800f0009800caa2a80003fc070080ce200002
:10965800009890000000e0000500320080ce200055
:109668008098900080ce20001098900001000100a2
:1096780080ce2000200090006f006000000f78006e
:109688001e007800e40f5000070032001e0078002a
:10969800e80f5000060032001e007800e20f50006c
:1096a8000b00320038003700a7fd07003e003700e6
:1096b80080ce2000a0009000000f200000806000f5
:1096c800f00f5000380032009ffd070036003700c9
:1096d8005074800061748000d2cc2c00c3f4230045
:1096e80077e107000000e00001003c0004003700bb
:1096f8006011b8006000b800e22107001e003700c2
:10970800907a80000000e0001200320080ce200035
:109718009000900080ce20001018900022002000b9
:10972800811f7800110009000200d80001017800ab
:10973800cf007800808f500006003d0080ce2000ca
:1097480080109000700890006011b800cd210700cb
:109758000900370080ce2000700990008011900029
:1097680080ce20008010900070089000c52107006e
:109778000000eb00907a88006011b8006000b80023
:10978800012207000800370010002000907a8800a6
:109798006011b8006000b800ba2107006011b80075
:1097a8006000b800f82107008760a9000080fa006f
:1097b8003400f9004f03be004f02be004f01be0047
:1097c8004f00be003600f90000400600a04090009f
:1097d8008180fb0063834000e303400020c4b300a2
:1097e800c049e300180032000600e00003003a0018
:1097f800064078000080fb00000006000041eb00f6
:109808000000eb0080007800059c2000674078008d
:10981800014068000080fb0060c07a000080fb0007
:10982800c808dd00810068000241e8000280fb00f2
:10983800860f5000f5ff3900014078000080fb00da
:1098480000000600edff37000001eb00059c20003a
:1098580083cdb3000410200002407800810020006e
:109868000004e0000a003500004040008100e900e3
:10987800fbff3a0000f17a000201e800840f510072
:10988800d9ff32000240780081002000f4ff370041
:109898000040d000034068008100e900f0ff3a0072
:1098a800f4ff370001487800124098008040eb0030
:1098b8002140980000000500889fbe0080047800c1
:1098c80010407800b044980019409000c0449800b7
:1098d80029409000d04498000084fb0063044400b1
:1098e80009007800b9ff0700b0dc980088804400c0
:1098f800b04098000000eb004f04be0000000600d6
:109908006040900080487800000005006300400037
:109918003041900082487800404090009040980084
:109928000000050063004000304190008248780044
:109938004041900092409800d04190008381fb0004
:10994800604190004811dd0082817100b3009800e9
:10995800704190000281fb00a2009800004990002d
:109968000281fb00104890004800dd0000017100f2
:1099780092009800000005006601400092417800be
:10998800efc861001281fb004411de00924098008c
:1099980067004000904178006fc16100a2409800c4
:1099a8001080fb004400de00b04098000000050075
:1099b80063004000b04190008381fb00404190006b
:1099c8004811dd008281710093009800504090009a
:1099d8000080fb00800878000000050060409000cf
:1099e800804878000000050063004000b041900006
:1099f8008381fb00404190004811dd00828871009e
:109a0800d04190008381fb00604190004811dd0047
:109a18008281710093009800f04190008381fb00df
:109a2800004990004811dd0082817100a300980070
:109a3800904990008381fb00204990004811dd0087
:109a480082817100b3009800604990000281fb0098
:109a580003002000c2009800d3009800c819dd0058
:109a68000280fd00824178000041eb00504a9000de
:109a78000482fb000500200004017100858171004b
:109a8800c2009800d3009800c819dd000280fd00cc
:109a9800824178000041eb00404a90000482fb00bc
:109aa800050020000401710085817100c200980042
:109ab800d3009800c819dd000280fd0082417800bb
:109ac8000041eb00304a90000482fb0005002000b2
:109ad8000401710085817100c2009800d3009800cc
:109ae8000000050063004000b04190008381fb0046
:109af800404190004811dd0082887100d0419000fb
:109b08008381fb00604190004811dd008281710073
:109b180093009800f04190008381fb000049900079
:109b28004811dd0082817100a3009800104990005f
:109b38000281fb00204890004800dd000001710010
:109b4800b20098000000050063004000b04190009a
:109b58008381fb00404190004811dd00828871003c
:109b6800d04190008381fb00604190004811dd00e6
:109b78008281710093009800f04190008381fb007e
:109b8800004990004811dd0082817100a30098000f
:109b9800104990000281fb00204890004800dd0039
:109ba80000017100b2009800000005006300400049
:109bb80030419000824878004040900090409800e2
:109bc8000000050063004000b04190008381fb0065
:109bd800404190004811dd0082887100504190009a
:109be8000281fb00604090004800dd000001710028
:109bf8009200980000000500889fbe008a9fbe0062
:109c0800000578000140780002047800e30445006c
:109c1800e605450011c5b3000300e000130032005b
:109c2800004178000a0078001eff0700984d780070
:109c380028409000c044980038409000d0449800d4
:109c480048409000e044980058449000f844980038
:109c580050c0b300204598000a00780016ff07009e
:109c68004f05be004f04be000000060011c9b30036
:109c7800004178000a0078000aff0700984d780034
:109c880028409000c044980038409000d044980084
:109c980048409000e044980058449000f8449800e8
:109ca80050c0b300204598000a00780002ff070062
:109cb8004f05be004f04be0000000600ebff370052
:109cc800630040003041900082487800c041900015
:109cd8008381fb00504190004811dd0082817100b2
:109ce80093009800604190000281fb007040900052
:109cf8004800dd0000017100a20098000000050086
:109d0800d1252a000004e00004003200c1242a0002
:109d1800e14f50000100320051252a00010078006f
:109d280000000600889fbe008a9fbe0000057800dc
:109d3800014078008204780063044500e605450088
:109d480051c9b3000300e0003c0032000041780034
:109d58000a007800d3fe07001900be00804d780085
:109d6800c809de00480add004801de000201720071
:109d7800424498004009de00030020005244980045
:109d88004808de006044980029009000b90090005f
:109d980070449800c809de00480add004801de006a
:109da80002017200024c98004009de000300200006
:109db800124c98004808de00204c9800490090009a
:109dc800d9009000304c9800c809de00480add0030
:109dd8004801de0002017200424c98004009de0092
:109de80003002000524c98004808de00604c9800a0
:109df80049489000704c9800594a900004549800c3
:109e08006948900010549800794a900024549800aa
:109e18000950900030549800995490004954980083
:109e280020c1b300204598000a007800a2fe070070
:109e38004f05be004f04be000000060051c1b3002c
:109e4800004178000a00780096fe07001900be005d
:109e5800804d7800c809de00480add004801de00b0
:109e680002017200424498004009de00030020000d
:109e7800524498004808de00604498002900900089
:109e8800b900900070449800c809de00480add0057
:109e98004801de0002017200024c98004009de0011
:109ea80003002000124c98004808de00204c98005f
:109eb80049009000d9009000304c9800c809de0095
:109ec800480add004801de0002017200424c980099
:109ed8004009de0003002000524c98004808de00cc
:109ee800604c980049489000704c9800594a90007e
:109ef800045498006948900010549800794a9000da
:109f080024549800095090003054980099549000b7
:109f18004954980020c1b300204598000a007800f1
:109f280065fe07004f05be004f04be000000060096
:109f3800c2ff370063004000304290000482fb00fb
:109f480005002000404190004811dd00030020007a
:109f58000202720083827200504190008281fb00ed
:109f680002002000020272008382720060419000a9
:109f7800c811dd0002002000821872008390720070
:109f8800704290000482fb00050020000049900008
:109f98004811dd0003002000020272008382720073
:109fa800104990008281fb0002002000020272002a
:109fb8008382720020499000c811dd000200200051
:109fc8000202720083827200a4009800b500980013
:109fd800304a90000482fb000500200040499000b0
:109fe8004811dd0003002000020272008382720023
:109ff800504990008281fb0002002000020272009a
:10a008008382720060499000c811dd0002002000c0
:10a018000202720083827200c4009800d500980082
:10a02800f04990008381fb00005190004811dd0049
:10a0380082817100e3009800905190008381fb00b9
:10a04800205190004811dd0082817100f3009800d2
:10a05800305190000281fb00405090004800dd0024
:10a06800000171008208980000000500889fbe006a
:10a078008a9fbe000004780001407800020578003d
:10a08800e3054400e604440051c5b3000300e000c2
:10a0980001003a0051c9b300004178000800780077
:10a0a80000fe0700e40045004000200021f07c008d
:10a0b8000000e900fdff3a0067814500f400450013
:10a0c80000012000217178000000e900fdff3a003e
:10a0d80040c1b3002044980008007800f6fd07004e
:10a0e8004f05be004f04be0000000600630240009a
:10a0f80066004000e481400042002000e051790001
:10a108000201e900fdff3a0067014200f4804000c7
:10a1180000012000e25078000000e900fdff3a004d
:10a1280000000600889fbe008a9fbe0000057800d8
:10a138000140780002047800e3044500e605450084
:10a1480021c5b3000300e000290032000041780077
:10a158000a007800d3fd0700984d78001840900059
:10a16800c044980028409000d0449800384090009f
:10a17800e044980048409000f0449800584090000f
:10a18800804c980068409000904c9800784090006f
:10a19800a04c980008489000b04c980018489000cf
:10a1a800c04c980028489000d04c9800384890003f
:10a1b800e04c980048489000f04c980058489000af
:10a1c800805498006848900090549800784c90000b
:10a1d800a854980000c1b300204598000a007800f0
:10a1e800b5fd07004f05be004f04be000000060085
:10a1f80021c9b300004178000a007800a9fd0700d2
:10a20800984d780018409000c0449800284090006d
:10a21800d044980038409000e044980048409000ae
:10a22800f044980058409000804c98006840900096
:10a23800904c980078409000a04c980008489000f6
:10a24800b04c980018489000c04c980028489000de
:10a25800d04c980038489000e04c9800484890004e
:10a26800f04c980058489000805498006848900036
:10a2780090549800784c9000a854980000c1b300fe
:10a28800204598000a0078008bfd07004f05be00a6
:10a298004f04be0000000600d5ff370063004000f1
:10a2a800b04190008381fb00404190004811dd00df
:10a2b80082887100d04190008381fb00604190004a
:10a2c8004811dd008281710093009800f0419000f0
:10a2d8008381fb00004990004811dd0082817100f4
:10a2e800a3009800904990008381fb0020499000ca
:10a2f8004811dd0082817100b3009800b0499000d8
:10a308008381fb00404990004811dd008281710083
:10a31800c3009800d04990008381fb0060499000f9
:10a328004811dd0082817100d3009800f049900047
:10a338008381fb00005190004811dd00828171008b
:10a34800e3009800105190000281fb00205090001b
:10a358004800dd0000017100f200980000000500cf
:10a36800889fbe00000478000240780083047800cb
:10a378000074a0000141780080407800080078004f
:10a3880048fd0700994478006944980010c0b3005c
:10a39800204498000800780047fd07004f04be00dd
:10a3a80000000600889fbe008a1f7800000578001c
:10a3b80002047800e604450001417800e1c0b300da
:10a3c8000a00780037fd0700080178000000eb005c
:10a3d8000104200032f07c000000e800810f5000ea
:10a3e800fcff3a0000042000204598000a0078008d
:10a3f80031fd07004f0578004f04be00000006003d
:10a40800660040000001eb0003042000e0587900da
:10a418000201e800830f5100fcff3a00000005002c
:10a42800889fbe008a1f7800000578000204780023
:10a43800e30445000141780041c9b3000a007800ef
:10a4480018fd070018407800b044980018409000a4
:10a45800c044980028409000d044980038409000ac
:10a46800e04498006a014500f40044000000eb0055
:10a47800317178000000e800f00f5000fcff3a004e
:10a4880077814400e40044000000eb00317178005b
:10a498000000e800f00f5000fcff3a007440400054
:10a4a800204598000a00780003fd07004f05780052
:10a4b8004f04be0000000600889fbe008a1f780077
:10a4c80000057800820478006304450001417800a3
:10a4d80031c8b3000a007800f2fc07002940900058
:10a4e8003044980039409000404498001940780062
:10a4f80050449800994490006944980040c0b300c3
:10a50800204598000a007800ebfc07004f0578000a
:10a518004f04be0000000600881f78000004780081
:10a52800aafc070080417800a8409000d2ff2f00c5
:10a5380040c5b30080cf5000030036000200780009
:10a548004f047800000006000180fb006400400012
:10a55800e2ff2f0071052000810f5000f7ff3c003b
:10a5680038d8900000c069000080fb000001ea00b4
:10a578004f91de00020078004f04780000000600ca
:10a58800f1ff370010417800e54f5100120032000a
:10a5980009003600e84f51001a0032000f0036005b
:10a5a800e94f510019003200ea4f510016003200fd
:10a5b8000080eb0000000600e24f51000c00320062
:10a5c80009003600e34f510009003200e44f510002
:10a5d800f7ff3a00cafc3700d2fc3700e64f5100bb
:10a5e800f3ff3a00e4fc3700e14f5100f0ff3a0076
:10a5f8005b000900b0587800c105b100c005b10082
:10a6080000000500eafc370036fd3700f3fc370090
:10a618008000fa00889fbe008a9fbe0080057800ef
:10a6280002047800420620000221070058409000ea
:10a638000080fb00801f7800284090000080fb000d
:10a64800801f7800484090000080fb00801f780041
:10a65800184090000080fb00801f78003840900070
:10a668000080fb00801f78001880fb00801f7800a6
:10a6780050262a00801f7800a0f62f000f00400007
:10a68800edd7070042062000a1f62f008f8040007a
:10a698000b007800e7200700ee875700284090005d
:10a6a8000004e00012003a0038d890000080fb0057
:10a6b800801f7800a0292a00801f780040f72f000b
:10a6c8000f004000dcd707004206200041f72f00aa
:10a6d8008f8040000b007800d6200700e4875700e1
:10a6e8004f05be004f04be000080fa0000000600bf
:10a6f800660544008004eb003a80fb00801f780068
:10a7080040292a00801f780040f72f000f004000e2
:10a71800c9d707004206200041f72f008f8040006c
:10a728000b007800c32007008904e8002840900047
:10a738000080fb00e4875700808f5400daff310067
:10a748003a80fb00801f780040292a00801f78008b
:10a7580040f72f000f004000b7d70700420620003f
:10a7680041f72f008f8040000b007800b1200700d0
:10a778008904e800284090000080fb00e487570027
:10a78800808f5400dcff3900c7ff3700889fbe0068
:10a798008a9fbe008c1f78000005780001067800ab
:10a7a80082047800830578006304410032002000a9
:10a7b80088007800932007008081eb000000e0000b
:10a7c80005003200030078004f0678004f05be00f0
:10a7d8004f04be0000000600984c780049409000e5
:10a7e80090449800d9409000a14498000141e800a5
:10a7f800b3ff2f0040c5b30080cf5000f1ff3e00eb
:10a808000281fb00e68044008b0178000a00780092
:10a818007c200700e3ff2f000000e000e9ff3a007a
:10a82800294090000080fb00090040006040900033
:10a83800b0dc98000900780037ff0700d3ff2f002d
:10a848000000e000dfff3a000c00e00004003500e3
:10a858001980fb00c3ff2f00800f5600d9ff3a0074
:10a86800000020004f0678004f05be004f04be00d0
:10a8780000000600d8ff37005c00fa00881f780047
:10a88800020478008180fb0022fa2f000f014100aa
:10a89800beff07008080eb000000e00004003200eb
:10a8a800010078004f0478000080fa0000000600dc
:10a8b8008800780020fa2f000f00400031ff0700c1
:10a8c800000078004f0478000080fa0000000600bd
:10a8d800f7ff370082017800214190000281fb00d8
:10a8e80064014100e3804000422037000400fa0080
:10a8f800204798000040eb00004f7800ae409000e1
:10a9080000c1b3007a1c0700004f78001e00fb004e
:10a918000080fa00000006000400fa0020479800b2
:10a92800314798000040eb00004f78003e4190000e
:10a93800ae40900000c1b300c51c0700004f78006e
:10a948001e00fb000080fa00000006000c00fa0060
:10a9580010079800210798000000eb00000f78000e
:10a968002e0090000000e00003003a00e0ff2f00f6
:10a97800500798001c00370010002000300798008e
:10a988000a0037003e009000800078001e0090000a
:10a9980000804000104078000080fb001e0f40003f
:10a9a8003e0090000000e80030079800be009000cc
:10a9b8002e009000808f5000f2ff3900f00f200029
:10a9c8001e0f60001e00e000030032000080eb0054
:10a9d80040079800020037000000eb00400798008d
:10a9e8004e009000500798005e0090000080fa002a
:10a9f800000006001800fa00200f9800e300470046
:10aa0800a3c0b30042c7b30000c1b3005c1c070079
:10aa1800204798002e4090000004e0000400320017
:10aa28002e4090000000fb00300f98001d003700fa
:10aa380063004700a1002000c4ff070020479800da
:10aa48002e4090000004e000040032002e409000e8
:10aa58000000fb00300f9800120037000000eb00e8
:10aa6800000f7800090037001e0078008000780089
:10aa78002e089000008140009e00e8006300470017
:10aa880060c07800004978001e0fe80070002000c0
:10aa98009e0f1000f4ff34002e4090000000fb00d1
:10aaa800300f98003e0890000080fa000000060071
:10aab8000600fa00100798000040eb00004f7800ed
:10aac800e3c0b300e2c0b3009e00900000c1b30031
:10aad8002b1c0700004f78001e04e0000300320022
:10aae8001e00fb00200798000b0037001e00900096
:10aaf800e100200095ff0700004f78001e04e000e9
:10ab0800030032001e00fb002007980002003700f7
:10ab18000000eb00200798002e0090000080fa004b
:10ab2800000006000600fa00100798000040eb003d
:10ab3800004f7800e3c0b3000041eb009e00900096
:10ab480000c1b3000e1c0700004f78001e04e0008f
:10ab5800030032001e00fb00200798000b0037009e
:10ab68001e009000e100200078ff0700004f7800e9
:10ab78001e04e000030032001e00fb0020079800be
:10ab8800020037000000eb00200798002e0090001c
:10ab98000080fa00000006000600fa00100798007e
:10aba8000040eb00004f7800e3c0b300c2c1b3001f
:10abb8009e00900000c1b300f11b0700004f780011
:10abc8001e04e000050032009e4078006ac0500074
:10abd8000000fb00200798000d0037001e009000c1
:10abe800e100200059ff0700004f78001e04e00034
:10abf80005003200e0ccb3001e4040000000fb001e
:10ac080020079800020037000000eb00200798009a
:10ac18002e0090000080fa00000006000600fa00ee
:10ac2800100798000040eb00004f7800e3c0b30025
:10ac3800a2c2b3009e00900000c1b300d01b070061
:10ac4800004f78001e04e000030032001e00fb00e5
:10ac5800200798000b0037001e009000e10020003c
:10ac68003aff0700004f78001e04e000030032009e
:10ac78001e00fb0020079800020037000000eb00d0
:10ac8800200798002e0090000080fa0000000600bf
:10ac98000600fa00100798000040eb00004f78000b
:10aca800e3c0b30082c3b3009e00900000c1b300ac
:10acb800b31b0700004f78001e04e00003003200b9
:10acc8001e00fb00200798000b0037001e009000b4
:10acd800e10020001dff0700004f78001e04e0007f
:10ace800030032001e00fb00200798000200370016
:10acf8000000eb00200798002e0090000080fa006a
:10ad0800000006000600fa00100798000040eb005b
:10ad1800004f780063c0b30062c4b3009e00900087
:10ad280000c1b300961b0700004f78001e04e00026
:10ad3800030032001e00fb00200798000b003700bc
:10ad48001e0090006100200000ff0700004f7800ff
:10ad58001e04e000030032001e00fb0020079800dc
:10ad6800020037000000eb00200798002e0090003a
:10ad78000080fa00000006000600fa00100798009c
:10ad88000040eb00004f780063c0b300c2c4b300ba
:10ad98009e00900000c1b300791b0700004f7800a7
:10ada8001e04e000030032001e00fb00200798008c
:10adb8000b0037001e00900061002000e3fe070032
:10adc800004f78001e04e000030032001e00fb0064
:10add80020079800020037000000eb0020079800c9
:10ade8002e0090000080fa00000006000600fa001d
:10adf800100798000040eb00004f780043c1b300f3
:10ae080002c6b3009e00900000c1b3005c1b07009f
:10ae1800004f78001e04e000050032009e407800d4
:10ae28006ac050000000fb00200798000d003700a2
:10ae38001e00900041012000c4fe0700004f78006a
:10ae48001e04e00005003200e0ccb3001e404000c4
:10ae58000000fb0020079800020037000000eb000c
:10ae6800200798002e0090000080fa0000000600dd
:10ae78000600fa00100798000040eb00004f780029
:10ae8800e3c0b30022c5b3009e00900000c1b30028
:10ae98003b1b0700004f78001e04e000030032004f
:10aea8001e00fb00200798000b0037001e009000d2
:10aeb800e1002000a5fe0700004f78001e04e00016
:10aec800030032001e00fb00200798000200370034
:10aed8000000eb00200798002e0090000080fa0088
:10aee800000006000600fa00100798000040eb007a
:10aef800004f780023c1b30062c6b3009e009000e3
:10af080000c1b3001e1b0700004f78001e04e000bc
:10af1800030032001e00fb00200798000b003700da
:10af28001e0090002101200088fe0700004f7800d5
:10af38001e04e000030032001e00fb0020079800fa
:10af4800020037000000eb00200798002e00900058
:10af58000080fa00000006000200fa00000f7800e6
:10af6800e0c0b30061fe0700804078001e00780052
:10af7800014878001e0fe800f0c0b3005bfe070030
:10af8800804078001e007800014878001e0fe80015
:10af980000c1b30055fe0700804078001e0078000d
:10afa800014878001e0fe80010c1b3004ffe0700eb
:10afb800804078001e007800014878001e0fe800e5
:10afc80020c1b30049fe0700804078001e007800c9
:10afd800014878001e0fe80030c1b30043fe0700a7
:10afe800804078001e007800014878001e0fe800b5
:10aff80040c1b3003dfe0700804078001e00780085
:10b00800014878001e0fe80050c1b30037fe070062
:10b01800804078001e007800014878001e0fe80084
:10b0280060c1b30031fe0700804078001e00780040
:10b03800014878001e0fe80070c1b3002bfe07001e
:10b04800804078001e007800014878001e0fe80054
:10b0580080c1b30025fe0700804078001e007800fc
:10b06800014878001e0fe80090c1b3001ffe0700da
:10b07800804078001e007800014878001e0fe80024
:10b08800a0c1b30019fe0700804078001e007800b8
:10b09800014878001e0fe800b0c1b30013fe070096
:10b0a800804078001e007800014878000080fa008f
:10b0b80000000600cc00fa0050a798000000eb0042
:10b0c800000f78005ea09000610060000004e000be
:10b0d8002d0032000e80e80075fe07000000fb001e
:10b0e8001e0f70000e80e800104190000e80e800ee
:10b0f800204290000e80e800b04090000e80e800ea
:10b10800404090008241780004417800d80207004e
:10b11800e2d920000089be000e80e800504190006e
:10b128000e80e800604290000e80e800f040900039
:10b138000e80e800004890008241780004417800c1
:10b14800cb020700e2d920002001980031019800c5
:10b158000e80e800104990000e80e800204a900018
:10b168000e80e800b04890000e80e800404890004b
:10b178008241780004417800bd020700e2d920002e
:10b1880040019800510198005ea090004800de0040
:10b19800610060000004e0002e0032000e80e8002c
:10b1a80060fe07000000fb001e0f70000e80e80024
:10b1b800104190000e80e800204290000e80e800c8
:10b1c800b04090000e80e800404090008241780036
:10b1d80004417800a6020700e2d920006001980027
:10b1e800710198000e80e800504190000e80e80040
:10b1f800604290000e80e800f04090000e80e80069
:10b2080000489000824178000441780098020700c5
:10b21800e2d9200000099800110998000e80e80082
:10b22800104990000e80e800204a90000e80e80047
:10b23800b04890000e80e8004048900082417800b5
:10b24800044178008a020700e2d92000200998000a
:10b25800310998005ea090000000d10061006000f4
:10b268000004e0002e0032000e80e8004afe0700cd
:10b278000000fb001e0f70000e80e80010419000d7
:10b288000e80e800204290000e80e800b040900058
:10b298000e80e80040409000824178000441780028
:10b2a80073020700e2d9200040099800510998006c
:10b2b8000e80e800504190000e80e8006042900047
:10b2c8000e80e800f04090000e80e80000489000f2
:10b2d800824178000441780065020700e2d9200025
:10b2e80060099800710998000e80e80010499000e4
:10b2f8000e80e800204a90000e80e800b0489000d8
:10b308000e80e800404890008241780004417800af
:10b3180057020700e2d92000001198001111980087
:10b328005ea090004200de00610060000004e000c2
:10b338002e0032000e80e80038fe07000000fb00f7
:10b348001e0f70000e80e800104190000e80e8008b
:10b35800204290000e80e800b04090000e80e80087
:10b368004040900082417800044178004002070084
:10b37800e2d9200020199800311998000e80e800c1
:10b38800504190000e80e800604290000e80e80076
:10b39800f04090000e80e80000489000824178005c
:10b3a8000441780032020700e2d9200040199800d1
:10b3b800511998000e80e800104990000e80e800ae
:10b3c800204a90000e80e800b04890000e80e80007
:10b3d8004048900082417800044178002402070028
:10b3e800e2d9200060199800711998005ea09000b9
:10b3f8004300de00610060000004e0002e0032001f
:10b408000e80e8009afe07000000fb001e0f700087
:10b418000e80e800104190000e80e8002042900065
:10b428000e80e800b04090000e80e8004040900098
:10b4380082417800044178000d020700e2d920001b
:10b4480040119800511198000e80e800504190007a
:10b458000e80e800604290000e80e800f040900006
:10b468000e80e8000048900082417800044178008e
:10b47800ff010700e2d920006019980071199800af
:10b488000e80e800104990000e80e800204a9000e5
:10b498000e80e800b04890000e80e8004048900018
:10b4a8008241780004417800f1010700e2d92000c8
:10b4b80020099800310998005ea090004400de0041
:10b4c800610060000004e0002e0032000e80e800f9
:10b4d800effd07000000fb001e0f70000e80e80063
:10b4e800104190000e80e800204290000e80e80095
:10b4f800b04090000e80e800404090008241780003
:10b5080004417800da010700e2d9200060219800a0
:10b51800712198000e80e800504190000e80e800ec
:10b52800604290000e80e800f04090000e80e80035
:10b53800004890008241780004417800cc0107005f
:10b54800e2d9200000299800112998000e80e8000f
:10b55800104990000e80e800204a90000e80e80014
:10b56800b04890000e80e800404890008241780082
:10b5780004417800be010700e2d920002029980084
:10b58800312998005ea090004500de00610060004f
:10b598000004e000120032000e80e800f6fd07000b
:10b5a8000000fb001e0f70000e80e80010419000a4
:10b5b8000e80e800204290000e80e800b040900025
:10b5c8000e80e800404090008241780004417800f5
:10b5d800a7010700e2d920004011980051119800f6
:10b5e8005ea090004600de00610060000004e000fc
:10b5f800120032000e80e800c2fd07000000fb00c8
:10b608001e0f70000e80e800104190000e80e800c8
:10b61800204290000e80e800b04090000e80e800c4
:10b628004040900082417800044178009001070072
:10b63800e2d9200040299800512998005ea0900086
:10b648004700de00610060000004e0003c003200ba
:10b658000e80e80023fe07000000fb001e0f7000ac
:10b668000e80e800104190000e80e8002042900013
:10b678000e80e800b04090000e80e8004040900046
:10b68800824178000441780079010700e2d920005e
:10b6980060299800712998000e80e80050419000b8
:10b6a8000e80e800604290000e80e800f0409000b4
:10b6b8000e80e8000048900082417800044178003c
:10b6c8006b010700e2d92000003198001131980081
:10b6d8000e80e800104990000e80e800204a900093
:10b6e8000e80e800b04890000e80e80040489000c6
:10b6f80082417800044178005d010700e2d920000a
:10b7080020319800313198000e80e80050499000af
:10b718000e80e800604a90000e80e800f048900033
:10b728000e80e800005090008241780004417800c3
:10b738004f010700e2d920004031980051319800ac
:10b748001e0078000080fa00000006000e00fa00d3
:10b7580040079800510798004e0090000000e8004c
:10b76800300798000000eb00100798004e0090008a
:10b7780047fd07000000fb00000f78001e00e000f6
:10b788000400320080f32f001e004000600798007c
:10b798002d0037004e00900010407800e14f500017
:10b7a80003003e000000eb00600798002600370009
:10b7b8004e009000104078000080fb000080e900f7
:10b7c8000080d100100798000000eb0020079800c7
:10b7d800170037003e009000104078008081fb0081
:10b7e8003e0090000000e800300798003e009000fe
:10b7f800104078000081fb003e0090000000e80047
:10b80800300798002e00900000004000800078006b
:10b818005e009000808040004810dd00030070004a
:10b82800800878002e0090000000e80020079800ab
:10b83800ae0090001e009000808f5000e5ff390098
:10b848001e009000600798006e0090000080fa00cb
:10b85800000006000000fa00cbc2bf000080fb0019
:10b868000000d100614060008040780010c0b30043
:10b8780001405000614060006140600000414000ac
:10b88800b12c200091407800d0cfb30000c06000f8
:10b8980002407000cbe2b7000080fa00000006000a
:10b8a8000000fa00d07980000000e0000e003200ad
:10b8b80062000700e07980000000e0000300320029
:10b8c800e07980000000e900e0798800e0798000f4
:10b8d8000000e00006003a008000eb0040c52500ab
:10b8e800e517070002003700401f2000430007004b
:10b8f8000080fa00000006000000fa00c07980000d
:10b908000000e0000c003a000000eb00d07988004d
:10b918000000eb00e07988008000eb0040c52500be
:10b928007d1707008000eb00e0c225007a170700aa
:10b9380010002000c07988000080fa00000006008e
:10b948000800fa0040479800310798003e00900030
:10b958000000e000200032004e409000004f7800c8
:10b968001a003700803e20001007980010003700aa
:10b97800cbc2bf00624060000004e00005003a004e
:10b98800cb22a80000f4210001002000cb1d0700f5
:10b9980004003700cb22a90000f421000100200098
:10b9a800c61d07001e0090000000e900100798005f
:10b9b8001e0090000000e000edff3a00009020001b
:10b9c800d1032000bd1d07001e4fe9001e04e00042
:10b9d800e4ff3a0007003700c7ff07004e40900019
:10b9e8000080fb00e0798800419c200040c52500cc
:10b9f800a11707000080fa00000006000200fa0004
:10ba0800000f7800bcff07001e007800000040000f
:10ba18000001780000712200110009000280d8009e
:10ba280080007800e0c2250093170700100020006e
:10ba3800d07988000080fa00000006000000fa00b3
:10ba48008000eb00e0c225008b1707000000eb0028
:10ba5800d0798800cbc2bf000080fa000000060041
:10ba68000200fa00000f78001e0078006101b8009b
:10ba780000c429000012b8006010b900050378005e
:10ba88000003430000c429000098b90000034300e4
:10ba9800860278000400be00881d07000080fa00b6
:10baa800000006000200fa00000f78001e0078006f
:10bab8006101b800800220000012b8006010b900cf
:10bac8000503780000034300800220000098b900b5
:10bad80000034300860278000400be00771d0700bb
:10bae8000080fa00000006000800fa00889fbe00e7
:10baf800d0cc2c00c1dc2300008fbe000000eb007e
:10bb0800fb1b0700f0788800f87880006140b900d6
:10bb18006cd7070020079800310798000800e0005c
:10bb280007003d0002002000037824002e0090004a
:10bb3800be00900005d8070020079800310798003c
:10bb480092282d00e3b523002e009000be0090003f
:10bb5800c9d7070082612200b3fc2300fad7070087
:10bb68000079880011798800207980003179800077
:10bb78006011b80054d807000000e000010035004b
:10bb8800050037000079800011798000207988004d
:10bb98003179880011003700007980001179800020
:10bba8001e01be00b4d707000004be001e01be007f
:10bbb8000000200001f82300e3d707002279800065
:10bbc80033798000acd707000001be000800be0032
:10bbd800ded7070020798800317988004f04be003d
:10bbe8000080fa00000006000200fa0020798000b8
:10bbf80031798000020020008312240030d8070029
:10bc08000000e00001003c0004003700caa2a900bf
:10bc18000000eb00000f7800120037002079800048
:10bc280031798000323323003312240026d80700ec
:10bc38000000e0000100350007003700caa2a80094
:10bc48008000eb0000c0eb003dff07002000200053
:10bc5800000f780003003700caa2a80010002000d7
:10bc6800000f78001e0078000080fa00000006002f
:10bc78000a00fa006047980071479800024f980040
:10bc8800134f98000e8fe8001e0078009e48900021
:10bc9800014878001e00e8008e48900001487800ae
:10bca8001e80e800fe409000014878009e00780061
:10bcb80063804000ee409000014878001e0090002c
:10bcc800ae0090000080fa00000006000400fa00b0
:10bcd800008fbe001e00be00b2fd200093042400a9
:10bce80023d70700020020004333240062d707004f
:10bcf8000080fa00000006000400fa00008fbe0071
:10bd08001e00be00b2fd2000930424005ad707008d
:10bd1800020020004333240015d707000080fa00f2
:10bd2800000006001000fa0020079800310798006c
:10bd38004207980053079800640798007507980011
:10bd48004e019000de0190002e009000be00900091
:10bd5800dbd707000000e00001003c001c003700b2
:10bd68006e019000fe0190002e009000be00900031
:10bd7800d5d707000000e0000100350004003700b7
:10bd88002e009000be009000008fbe002b003700f0
:10bd98004e019000de0190006e009000fe009000c1
:10bda800c7d707000000e00001003c00040037008e
:10bdb8006e009000fe009000008fbe001f0037004c
:10bdc8004e009000de009000008fbe001b00370080
:10bdd8006e019000fe0190002e009000be009000c1
:10bde800b7d707000000e00001003c00040037005e
:10bdf8002e009000be009000008fbe000f0037009c
:10be08004e019000de0190006e009000fe00900050
:10be1800add707000000e00001003500040037003e
:10be28006e009000fe009000008fbe0003003700f7
:10be38004e009000de009000008fbe001e00be0085
:10be48000080fa00000006000800fa0010079800b9
:10be580021079800320798009e0090002e0090005d
:10be6800808f5000110036009e0090003e00900028
:10be7800808f5000030031001e009000000f7800f2
:10be88001a003700be0090002e009000808f5000ee
:10be9800030036003e009000000f780013003700c2
:10bea8002e009000000f7800100037009e009000d0
:10beb8003e009000808f5000030036001e00900066
:10bec800000f780009003700be0090002e00900097
:10bed800808f5000030031003e009000000f780072
:10bee800020037002e009000000f78001e00780036
:10bef8000080fa00000006000c00fa001007980005
:10bf080021079800320798004307980054079800c3
:10bf18009e0090002e009000808f50004800310055
:10bf28009e0090003e009000808f50004400310039
:10bf38009e0090004e009000808f5000400031001d
:10bf48009e0090005e009000808f50003c00310001
:10bf5800de0090004e009000808f50000e003600ea
:10bf6800de0090003e009000808f50000a003600ee
:10bf7800de0090002e009000808f500006003600f2
:10bf88004e019000be0090002e009000aeff07000a
:10bf9800000f780049013700ce0090005e00900045
:10bfa800808f50000e003600ce0090003e009000ba
:10bfb800808f50000a003600ce0090002e009000be
:10bfc800808f5000060036005e019000be00900091
:10bfd8002e0090009cff0700000f78003701370003
:10bfe800be0090005e009000808f50000e0036006a
:10bff800be0090004e009000808f50000a0036006e
:10c00800be0090002e009000808f50000600360081
:10c018005e019000ce0090002e0090008aff07007d
:10c02800000f7800250137005e019000ce009000d7
:10c038003e00900084ff0700000f78001f013700c2
:10c04800ae0090001e009000808f50004800310024
:10c05800ae0090003e009000808f500044003100f8
:10c06800ae0090004e009000808f500040003100dc
:10c07800ae0090005e009000808f50003c003100c0
:10c08800de0090004e009000808f50000e003600b9
:10c09800de0090003e009000808f50000a003600bd
:10c0a800de0090001e009000808f500006003600d1
:10c0b8004e019000be0090001e00900062ff070035
:10c0c800000f7800fd003700ce0090005e00900061
:10c0d800808f50000e003600ce0090003e00900089
:10c0e800808f50000a003600ce0090001e0090009d
:10c0f800808f5000060036005e019000be00900060
:10c108001e00900050ff0700000f7800eb0037007a
:10c11800be0090005e009000808f50000e00360038
:10c12800be0090004e009000808f50000a0036003c
:10c13800be0090001e009000808f50000600360060
:10c148005e019000ce0090001e0090003eff0700a8
:10c15800000f7800d90037005e019000ce009000f3
:10c168003e00900038ff0700000f7800d30037002a
:10c17800be0090001e009000808f500048003100e3
:10c18800be0090002e009000808f500044003100c7
:10c19800be0090004e009000808f5000400031009b
:10c1a800be0090005e009000808f50003c0031007f
:10c1b800de0090004e009000808f50000e00360088
:10c1c800de0090002e009000808f50000a0036009c
:10c1d800de0090001e009000808f500006003600a0
:10c1e8004e019000ae0090001e00900016ff070060
:10c1f800000f7800b1003700ce0090005e0090007c
:10c20800808f50000e003600ce0090002e00900067
:10c21800808f50000a003600ce0090001e0090006b
:10c22800808f5000060036005e019000ae0090003e
:10c238001e00900004ff0700000f78009f003700e1
:10c24800ae0090005e009000808f50000e00360017
:10c25800ae0090004e009000808f50000a0036001b
:10c26800ae0090001e009000808f5000060036003f
:10c278005e019000ce0090001e009000f2fe0700c4
:10c28800000f78008d0037005e019000ce0090000e
:10c298002e009000ecfe0700000f780087003700a2
:10c2a800ce0090001e009000808f500048003100a2
:10c2b800ce0090002e009000808f50004400310086
:10c2c800ce0090003e009000808f5000400031006a
:10c2d800ce0090005e009000808f50003c0031003e
:10c2e800de0090003e009000808f50000e00360067
:10c2f800de0090002e009000808f50000a0036006b
:10c30800de0090001e009000808f5000060036006e
:10c318003e019000ae0090001e009000cafe07008b
:10c32800000f780065003700be0090005e009000a6
:10c33800808f50000e003600be0090002e00900046
:10c34800808f50000a003600be0090001e0090004a
:10c35800808f5000060036005e019000ae0090000d
:10c368001e009000b8fe0700000f78005300370049
:10c37800ae0090005e009000808f50000e003600e6
:10c38800ae0090003e009000808f50000a003600fa
:10c39800ae0090001e009000808f5000060036000e
:10c3a8005e019000be0090001e009000a6fe0700ef
:10c3b800000f7800410037005e019000be00900039
:10c3c8002e009000a0fe0700000f78003b00370009
:10c3d800ce0090003e009000808f50000e00360086
:10c3e800ce0090002e009000808f50000a0036008a
:10c3f800ce0090001e009000808f5000060036008e
:10c408003e019000ae0090001e0090008efe0700d6
:10c41800000f780029003700be0090004e00900001
:10c42800808f50000e003600be0090002e00900055
:10c43800808f50000a003600be0090001e00900059
:10c44800808f5000060036004e019000ae0090002c
:10c458001e0090007cfe0700000f780017003700d0
:10c46800ae0090004e009000808f50000e00360005
:10c47800ae0090003e009000808f50000a00360009
:10c48800ae0090001e009000808f5000060036001d
:10c498004e019000be0090001e0090006afe07004a
:10c4a800000f7800050037004e019000be00900094
:10c4b8002e00900064fe0700000f78001e00780030
:10c4c8000080fa00000006000800fa002007980023
:10c4d800310798006011b8002e009000be0090004f
:10c4e800f9d507000000e00001003500050037001d
:10c4f8002e009000be00900001f0a200008fbe0048
:10c50800030037002e009000be009000008fbe0090
:10c518001e00be000080fa00000006000600fa00b7
:10c52800200798002e009000100798000e8fe80052
:10c538001e007800104078000080fb000080fa00a0
:10c54800000006000600fa00200798002e00900060
:10c55800100798000e8fe8001e00e80010407800d1
:10c568000080fb000080fa00000006000c00fa00c2
:10c5780010079800210798000000eb00000f7800d2
:10c588002e0090000000e00003003a00e0ff2f00ba
:10c59800500798001c003700100020003007980052
:10c5a8000a0037003e009000800078001e009000ce
:10c5b80000804000104078000080fb001e0f400003
:10c5c8003e0090000000e80030079800be00900090
:10c5d8002e009000808f5000f2ff3900f00f2000ed
:10c5e8001e0f60001e00e000030032000080eb0018
:10c5f80040079800020037000000eb004007980051
:10c608004e009000500798005e0090000080fa00ed
:10c61800000006000a00fa00100798002107980099
:10c62800320798000040eb00004f78003e00900071
:10c63800804178002e0090008040780000c8b30048
:10c6480000c04000004178009e00900000c1b30087
:10c658004b150700004f78001e04e000050032006b
:10c6680000c8b3001e4070000000fb00400798009f
:10c678000d003700be0090001e009000bbff0700b1
:10c68800004f78001e04e0000500320000c4b3002b
:10c698001e4070000000fb004007980002003700b1
:10c6a8000000eb00400798004e0090000080fa0060
:10c6b800000006000600fa00200798002e009000ef
:10c6c80063004000104078000080fb00010020005b
:10c6d800008fbe001e00be004809dd00c801de0054
:10c6e800830171004801dd002e0090000080e80001
:10c6f800104078000080fb0001002000001f41006e
:10c70800019749001e00be004809dd00c801de008f
:10c71800830171004801dd002e0090000000e80050
:10c72800104078000080fb0001002000001f41003d
:10c73800019749001e00be004809dd00c801de005f
:10c74800830171004801dd002e0090001040780040
:10c758000080fb0001002000001f410001974900f4
:10c768001e00be000080fa00000006001000fa005b
:10c77800881f780050079800610798000040eb0078
:10c78800004f78006e0090000000e00006003200c4
:10c798000e00e800820020008000eb009dff0700eb
:10c7a800004f7800050037000e00e80082002000e6
:10c7b8008100200097ff0700004f78001e04e0006a
:10c7c800030032001e00fb0070079800310037009c
:10c7d8000e00e800204090000080fb00c800dd004b
:10c7e8000e00e800104090000080fb000080700000
:10c7f800cf80de0033d407000200200043bb2300b3
:10c808009dd407005e0190000089be005e00900084
:10c81800640440000e00e800404090000080fb00e7
:10c82800c800dd000e00e800304090000080fb00ea
:10c8380000807000cf80de0022d4070002002000b4
:10c8480043bb23008cd40700008cbe005e00900020
:10c85800680440000e00e800604090000080fb0083
:10c86800c800dd000e00e800504090000080fb008a
:10c8780000807000cf80de0012d407000200200084
:10c8880043bb23007cd40700008cbe000000eb00f3
:10c89800700798007e0090004f0478000080fa002e
:10c8a800000006000e00fa00881f78005007980064
:10c8b8000040eb00004f78000e00e80082002000e6
:10c8c8000101200053ff0700004f78001e04e0001c
:10c8d800030032001e00fb0060079800310037009b
:10c8e8000e00e800204090000080fb00c800dd003a
:10c8f8000e00e800104090000080fb0000807000ef
:10c90800cf80de00efd307000200200003202400c0
:10c9180017d407005e0190000089be005e009000f9
:10c92800640440000e00e800404090000080fb00d6
:10c93800c800dd000e00e800304090000080fb00d9
:10c9480000807000cf80de00ded3070002002000e8
:10c958000320240006d40700008cbe005e0090006f
:10c96800680440000e00e800604090000080fb0072
:10c97800c800dd000e00e800504090000080fb0079
:10c9880000807000cf80de00ced3070002002000b8
:10c9980003202400f6d30700008cbe000000eb0043
:10c9a800600798006e0090004f0478000080fa003d
:10c9b800000006000e00fa00881f78005007980053
:10c9c8000040eb00004f78000e00e80082002000d5
:10c9d800810120000fff0700004f78001e04e000cf
:10c9e800030032001e00fb0060079800310037008a
:10c9f8000e00e800204090000080fb00c800dd0029
:10ca08000e00e800104090000080fb0000807000dd
:10ca1800cf80de00abd307000200200043cb230009
:10ca280015d407005e0190000089be005e009000ea
:10ca3800640440000e00e800404090000080fb00c5
:10ca4800c800dd000e00e800304090000080fb00c8
:10ca580000807000cf80de009ad30700020020001b
:10ca680043cb230004d40700008cbe005e00900076
:10ca7800680440000e00e800604090000080fb0061
:10ca8800c800dd000e00e800504090000080fb0068
:10ca980000807000cf80de008ad3070002002000eb
:10caa80043cb2300f4d30700008cbe000000eb004a
:10cab800600798006e0090004f0478000080fa002c
:10cac800000006000e00fa00881f78005007980042
:10cad8000040eb00004f78000e00e80082002000c4
:10cae80001022000cbfe0700004f78001e04e00082
:10caf800030032001e00fb00600798003100370079
:10cb08000e00e800204090000080fb00c800dd0017
:10cb18000e00e800104090000080fb0000807000cc
:10cb2800cf80de0067d307000200200003702400d6
:10cb38008fd307005e0190000089be005e00900060
:10cb4800640440000e00e800404090000080fb00b4
:10cb5800c800dd000e00e800304090000080fb00b7
:10cb680000807000cf80de0056d30700020020004e
:10cb7800037024007ed30700008cbe005e00900086
:10cb8800680440000e00e800604090000080fb0050
:10cb9800c800dd000e00e800504090000080fb0057
:10cba80000807000cf80de0046d30700020020001e
:10cbb800037024006ed30700008cbe000000eb0059
:10cbc800600798006e0090004f0478000080fa001b
:10cbd800000006001800fa00881f7800200f98004f
:10cbe8000040eb00004f78000e00e8002201200012
:10cbf800c103200087fe0700004f78001e04e000f4
:10cc0800030032001e00fb00300f98002900370097
:10cc18000e00e8000000e800a6fe070029d3070080
:10cc2800020020000370240051d307002e09900051
:10cc38000089be002e089000640440000e00e80041
:10cc4800650040009bfe07001ed30700020020007d
:10cc58000370240046d30700008cbe002e08900005
:10cc6800680440000e00e8006900400091fe0700db
:10cc780014d3070002002000037024003cd30700ef
:10cc8800008cbe002e0890006c0440000e00e800e6
:10cc98006d00400087fe07000ad30700020020004d
:10cca8000370240032d30700008cbe000000eb00a4
:10ccb800300f98003e0890004f0478000080fa007a
:10ccc800000006001400fa00881f7800000f980082
:10ccd8000040eb00004f78000e00e800e200200062
:10cce800e10420004bfe0700004f78001e04e0001e
:10ccf800030032001e00fb00100f980031003700bf
:10cd08000e00e8000000e8006afe0700edd2070008
:10cd1800020020004333240057d3070002002000fc
:10cd28000370240012d307000200200003682400c7
:10cd38000fd307000e0990000089be000e0890006e
:10cd4800640440000e00e8006500400059fe07003a
:10cd5800dcd20700020020004333240046d307003a
:10cd6800020020000370240001d307000200200005
:10cd780003682400fed20700008cbe000e08900055
:10cd8800680440000e00e8006900400049fe070002
:10cd9800ccd20700020020004333240036d307001a
:10cda8000200200003702400f1d2070002002000d6
:10cdb80003682400eed20700008cbe000000eb00e0
:10cdc800100f98001e0890004f0478000080fa00a9
:10cdd800000006000a00fa00300798000040eb0047
:10cde800004f78000e00e800420020008102200079
:10cdf80008fe0700004f78001e04e0000300320020
:10ce08001e00fb00400798000e0037000e00e800e7
:10ce1800204090000080fb00c800dd000e00e80004
:10ce2800104090000080fb0000807000cf80de0082
:10ce3800a4d207003e0190000089be000000eb006c
:10ce4800400798004e0090000080fa00000006009d
:10ce58000e00fa00881f7800500798000040eb0089
:10ce6800004f78000e00e80082002000c102200078
:10ce7800e8fd0700004f78001e04e00003003200c0
:10ce88001e00fb0060079800310037000e00e80024
:10ce9800204090000080fb00c800dd000e00e80084
:10cea800104090000080fb0000807000cf80de0002
:10ceb80084d207000200200003482400acd20700f7
:10cec8005e0190000089be005e009000640440008e
:10ced8000e00e800404090000080fb00c800dd0024
:10cee8000e00e800304090000080fb0000807000d9
:10cef800cf80de0073d20700020020000348240020
:10cf08009bd20700008cbe005e00900068044000c1
:10cf18000e00e800604090000080fb00c800dd00c3
:10cf28000e00e800504090000080fb000080700078
:10cf3800cf80de0063d207000200200003482400ef
:10cf48008bd20700008cbe000000eb006007980041
:10cf58006e0090004f0478000080fa000000060080
:10cf68001200fa00500798006107980072079800ad
:10cf78000040eb00004f78000e00e800820020001f
:10cf880041032000a3fd0700004f78001e04e000c5
:10cf9800030032001e00fb00000f98002f0037002e
:10cfa8000e00e800204090000080fb00c800dd0073
:10cfb8000e00e800104090000080fb000080700028
:10cfc800cf80de003fd20700020020000348240083
:10cfd80067d207005e0190000089be000e00e800dd
:10cfe800404090000080fb00c800dd000e00e80013
:10cff800304090000080fb0000807000cf80de0091
:10d0080030d207000200200043cb23009ad2070049
:10d018006e0190000089be000e00e800604090009c
:10d028000080fb00c800dd000e00e80050409000c2
:10d038000080fb0000807000cf80de0021d2070056
:10d04800020020000348240049d207007e01900016
:10d058000089be000000eb00000f98000e08900049
:10d068000080fa00000006001000fa00700798001f
:10d078000000eb00000f78007e0090006100600067
:10d088000004e000050032008000eb00e0d9200039
:10d09800b6fd07000000fb001e0f70007e00900028
:10d0a8004800de00610060000004e0000500320076
:10d0b80011002000a0da2000acfd07000000fb00f2
:10d0c8001e0f70007e0090000000d100610060001b
:10d0d8000004e0000400320060db2000f1fd0700de
:10d0e8000000fb001e0f70007e0090004200de0072
:10d0f800610060000004e0000400320020dd200030
:10d108002cfe07000000fb001e0f70007e00900040
:10d118004300de00610060000004e0000600320009
:10d12800a1dd2000a2dc200060dc20008cff0700cd
:10d138000000fb001e0f70007e0090004400de001f
:10d14800610060000004e00004003200a0de20005e
:10d158005cfe07000000fb001e0f70007e009000c0
:10d168004500de00610060000004e00015003200a8
:10d178000e80e80036ff07000000fb001e0f70005d
:10d188000e80e8001000be00e2d92000401198008f
:10d19800511198000e80e800b00090002000900027
:10d1a800e2d9200060119800711198000e80e80003
:10d1b800d000900040009000e2d9200000199800ab
:10d1c800111998007e0090004600de0061006000a2
:10d1d8000004e0000400320060df2000fdfe0700cc
:10d1e8000000fb001e0f70007e0090004900de006a
:10d1f800610060000004e00004003200a0e02000ac
:10d2080074fe07000000fb001e0f70007e009000f7
:10d218004a00de00610060000004e0000400320003
:10d22800a0e12000a7fe07000000fb001e0f700011
:10d238001e0078000080fa00000006001000fa00c6
:10d24800881f78000001780001047800f00f500072
:10d258005200320005003e00e10f50006e0032001f
:10d26800e20f5000ae003a008c00370000082000a2
:10d27800800f510026003200f00f2000800f51006f
:10d28800a7003a00f166800061409000e14f40003d
:10d298001a00320061099000f1099000829fbe00d7
:10d2a800c3fb2900831f780078805700e2cc070071
:10d2b800f1668000e88140006140900062c0b300e0
:10d2c8000440bc000280410042062000f88057005c
:10d2d800d8150700f1668000e881400061409000a1
:10d2e80062c0b3000440bc00028041004206200036
:10d2f80088007800cf150700e6875700caa2a80063
:10d308008000eb0000c0eb008df9070084003700b7
:10d31800f166800061409000e14f40001a00320041
:10d3280061099000f1099000829fbe00c3fb2900ab
:10d33800831f780078805700bfcc0700f166800013
:10d34800e88140006140900062c0b3000440bc0026
:10d358000280410042062000f8805700b5150700fa
:10d36800f1668000e88140006140900062c0b3002f
:10d378000440bc000280410042062000880078007a
:10d38800ac150700e6875700caa2a8008000eb008a
:10d3980010c0b3006af9070061003700f166800029
:10d3a80061409000e14f40005d003200610990004b
:10d3b800f1099000829fbe00c3fb2900831f7800fb
:10d3c800788057009ccc0700f1668000e881400017
:10d3d8006140900062c0b3000440bc00028041007c
:10d3e80042062000f880570092150700f166800079
:10d3f800e88140006140900062c0b3000440bc0076
:10d408000280410042062000880078008915070044
:10d41800e687570042003700f16680001100e000ff
:10d428003f00320061409000e14f40003c00320074
:10d4380061099000f1099000829fbe00c3fb29009a
:10d44800831f7800788057007bcc0700f166800046
:10d45800e88140006140900062c0b3000440bc0015
:10d468000280410042062000f8805700711507002d
:10d47800f1668000e88140006140900062c0b3001e
:10d488000440bc0002804100420620008800780069
:10d4980068150700e687570021003700f16680000d
:10d4a80012002000910f11001d003600614090000d
:10d4b800e14f40001a00320061099000f109900024
:10d4c800829fbe00c3fb2900831f78007880570025
:10d4d80059cc0700f1668000e88140006140900067
:10d4e80062c0b3000440bc00028041004206200034
:10d4f800f88057004f150700f1668000e88140006a
:10d508006140900062c0b3000440bc00028041004a
:10d51800420620008800780046150700e687570075
:10d528004f0478000080fa00000006000000fe00aa
:10d5380000000600889fbe00810478000000e0001b
:10d548004b003200110490006140b900ddd00700a3
:10d558000800e00003003d000200200003782400da
:10d568007ad1070002002000a347240000d1070059
:10d578005068880061688800190478006140b90023
:10d58800d0d007000800e00003003d0002002000a2
:10d59800037824006dd1070002002000a34724006f
:10d5a800f3d00700106888002168880059009000af
:10d5b800cf80de00c3d0070002002000a34724006c
:10d5c800ebd00700406a8800516a88006900900023
:10d5d800cf80de00bbd0070002002000a347240054
:10d5e800e3d00700606a8800716a880079009000bb
:10d5f800cf80de00b3d0070002002000a34724003c
:10d60800dbd00700806a8800916a880029009000b2
:10d61800cf80de00abd0070002002000a347240023
:10d62800d3d00700606b8800716b880039009000c8
:10d63800cf80de00a3d0070002002000a34724000b
:10d64800cbd00700806b8800916b88004900900060
:10d65800cf80de009bd0070002002000a3472400f3
:10d66800c3d00700a06b8800b16b88003800370072
:10d6780002002000a34724005068800061688000f1
:10d68800fdd0070092d10700900498000200200006
:10d69800a34724001068800021688000f6d00700a6
:10d6a8008bd10700800c780002002000a3472400db
:10d6b800606b8000716b8000efd0070084d1070099
:10d6c800a004980002002000a3472400806b80007b
:10d6d800916b8000e8d007007dd10700b004980066
:10d6e80002002000a3472400a06b8000b16b8000db
:10d6f800e1d0070076d10700c0049800020020009e
:10d70800a3472400406a8000516a8000dad00700ed
:10d718006fd10700d004980002002000a34724001e
:10d72800606a8000716a8000d3d0070068d1070062
:10d73800e004980002002000a3472400806a8000cb
:10d74800916a8000ccd0070061d10700f0049800ee
:10d758000000eb004f04be0000000600889fbe00da
:10d768008a1f7800010578000000e00012003200ee
:10d7780021009000cf80de0052d007000200240074
:10d78800c36124007ad007000004be001a0090008c
:10d79800cf80de004bd0070002002400c3612400c4
:10d7a80073d007000001be001a80fb000802be000b
:10d7b800030d070010003700090d0700004d780021
:10d7c8000080fb00080d070002002400c36124004c
:10d7d800a9d007003ed10700100598001a80fb0069
:10d7e8000e0d070002002400c3612400a2d0070028
:10d7f80037d10700200598000000eb004f0578009e
:10d808004f04be0000000600881f7800010478005d
:10d81800caa2a800c51207000004e00005003200f3
:10d8280011fc29000008200084fe07000080eb009e
:10d838000b003700080078000b1307000004e00015
:10d848000500320061fd2900000820007bfe07006a
:10d85800e0ff2f0002003700caa2a9000000eb0079
:10d868004f047800000006005a00fa00889fbe00a6
:10d87800c0fe290008000900305f78009e00b10052
:10d888009000b1004713070000482800e10120007c
:10d898000a160700f9150700531107006011b800b0
:10d8a8000200be00771107006011b8000200be0038
:10d8b800b51107006e140700fc1107003e110700a0
:10d8c8004111070000482800e1012000fb1507006e
:10d8d8000040eb00030b070040752900b4ea07007d
:10d8e8001100200010c0b30015f80700e7e9070091
:10d8f8001000200086ea0700ca22a800caa2a900d0
:10d9080000202100a1072000ec150700d5c2bf00a8
:10d918000038a30004003a00c2150700d5c2bf00b2
:10d928000038a300fcff32000e00780031f4070035
:10d938000040eb00004f98000e007800ae1407007e
:10d948001100200030c0b300fdf70700ca22a9006b
:10d95800caa2a800f0678000016880006d13070064
:10d96800580f07000110200000ac200010db070052
:10d9780080322800a0568800e0572800705a880096
:10d9880020922600805a8800a0a92600905a880074
:10d9980080c02600c05a8800e0a92600a05a880046
:10d9a80020bb2600b05a88000004eb000856880007
:10d9b800c6eaef00b8568800400b2000c056880021
:10d9c80050002000d056880020ac2000ef0a070045
:10d9d800a1002000808829004f0f070088007800e8
:10d9e800204f28004c0f070088007800805328003b
:10d9f800490f0700d86c8800c0622800c06c8800f6
:10da080080ac2000c613070080ac2000e913070093
:10da1800421f200051ff290080ac20000514070098
:10da2800e0ac2000c9130700e0ac2000e1130700b8
:10da3800421f2000c1012a00e0ac2000fd130700ae
:10da4800f166800061409000e14f40001b00320009
:10da58006904470061099000f1099000829fbe00a7
:10da6800c3fb2900831f780008007800f2ca07006a
:10da7800f1668000e88140006140900062c0b30018
:10da88000440bc0002804100420620008800780063
:10da9800e8130700f1668000e881400061409000cb
:10daa80062c0b3000440bc0002804100420620006e
:10dab80021042a00df130700e68757001e04e00050
:10dac80004003a00f1062a00f00f2000dbfd0700f1
:10dad80026003700f90447008e1f780031082a0015
:10dae800811f780009007800d3ca0700f16680001a
:10daf800e487570061409000e14f40001b0032006e
:10db08006904470061099000f1099000829fbe00f6
:10db1800c3fb2900831f780008007800c6ca0700e5
:10db2800f1668000e88140006140900062c0b30067
:10db38000440bc00028041004206200088007800b2
:10db4800bc130700f1668000e88140006140900046
:10db580062c0b3000440bc000280410042062000bd
:10db680089007800b3130700e6875700caa2a90006
:10db7800a1b5200000ac2000b0da070080ac20007e
:10db88007d130700e0ac20007b1307000000eb00ca
:10db98004f04be000080fa00000006003600f800be
:10dba800809fbe00829fbe00849fbe00869fbe00ed
:10dbb8003400f80000c0b300a00188001000fa008b
:10dbc8008020a900f166800061409000e14f40008c
:10dbd8001a00320061099000f1099000829fbe008e
:10dbe800c3fb2900831f78007680570092ca07007c
:10dbf800f1668000e88140006140900062c0b30097
:10dc08000440bc000280410042062000f680570014
:10dc180088130700f1668000e881400061409000a9
:10dc280062c0b3000440bc000280410042062000ec
:10dc380091092a007f130700e68757000000fe00bd
:10dc48000080fa003400f9004f03be004f02be0006
:10dc58004f01be004f00be003600f900004006002c
:10dc68003600f800809fbe00829fbe00849fbe00e1
:10dc7800869fbe003400f80000c0b300a0018800f1
:10dc88001000fa008060a900f166800061409000f1
:10dc9800e14f40001a00320061099000f10990003c
:10dca800829fbe00c3fb2900831f7800768057003f
:10dcb80061ca0700f1668000e88140006140900079
:10dcc80062c0b3000440bc0002804100420620004c
:10dcd800f680570057130700f1668000e88140007e
:10dce8006140900062c0b3000440bc000280410063
:10dcf80042062000d10a2a004e130700e687570083
:10dd08000000fe000080fa003400f9004f03be0056
:10dd18004f02be004f01be004f00be003600f900a2
:10dd2800004006003600f800809fbe00829fbe00bb
:10dd3800849fbe00869fbe003400f80000c0b30078
:10dd4800a00188001000fa008040a900f166800058
:10dd580061409000e14f40001a00320061099000d4
:10dd6800f1099000829fbe00c3fb2900831f780041
:10dd78007680570030ca0700f1668000e8814000cd
:10dd88006140900062c0b3000440bc0002804100c2
:10dd980042062000f680570026130700f16680002f
:10dda800e88140006140900062c0b3000440bc00bc
:10ddb8000280410042062000e10b2a001d130700e3
:10ddc800e68757000000fe000080fa003400f900e2
:10ddd8004f03be004f02be004f01be004f00be0001
:10dde8003600f900004006003600f800809fbe00ab
:10ddf800829fbe00849fbe00869fbe003400f8004c
:10de080000c0b300a00188001000fa008080a900bb
:10de1800f166800061409000e14f40001a00320036
:10de280061099000f1099000829fbe00c3fb2900a0
:10de3800831f780076805700ffc90700f1668000cd
:10de4800e88140006140900062c0b3000440bc001b
:10de58000280410042062000f6805700f5120700b4
:10de6800f1668000e88140006140900062c0b30024
:10de78000440bc000280410042062000d10c2a0068
:10de8800ec120700e68757000000fe000080fa0049
:10de98003400f9004f03be004f02be004f01be0020
:10dea8004f00be003600f90000400600000178006f
:10deb8006e08b900800078006400400003802000ec
:10dec800608079001200600005003a00668040001a
:10ded80092009000608079000080600001003200ac
:10dee80010002000000006006e09b90082017800c9
:10def800e400410002802000e10079009080700079
:10df080001187800e6804100e1007900108870006f
:10df1800000005001082fb00b001900082717a00b9
:10df28001082fb00b0019000848141004811de009e
:10df38009241980010c8e8000080e800eaff370026
:10df48009082fb003002900002f27a009082fb007f
:10df580030029000050242004811de00124298008b
:10df68001082fb0030019000040141002341980019
:10df78001082fb003001900004014100c819de0046
:10df88003341980010417800644841000080e8005f
:10df9800d5ff37001083fb00b002900082727b002f
:10dfa8001083fb00b0029000868242004811de0018
:10dfb800924298009082fb003001900005014100d8
:10dfc800234198009082fb00300190000501410038
:10dfd800c819de00334198009081fb0030019000a1
:10dfe80003014100444198009081fb0030019000fa
:10dff800030141004822de00544198001041780096
:10e00800664841000080e800b7ff37000800fa00c2
:10e01800889fbe008a1f78000005780002047800f7
:10e0280040c0b300a0f79f008004eb00a9bf9f0089
:10e03800b9bf9f00c9bf9f000141780081c8b300e4
:10e048000a00780017ee070066004500c0bf9f0071
:10e0580018487800c8409000114098005841900036
:10e0680022409800a8409000314098009800900005
:10e07800224080000100610077003a0028009000eb
:10e088000608b60074003a00924080000100610062
:10e098009e003a00280090001408b6009b003a0041
:10e0a8000241800001006100a3003a0028009000ae
:10e0b8002208b600a0003a00724180000100610009
:10e0c80084003a00280090003008b60081003a0029
:10e0d800e241800001006100a1003a0028009000a0
:10e0e8003e08b6009e003a005242800001006100de
:10e0f800a5003a00280090004c08b600a2003a009b
:10e10800c242800001006100ab003a002800900084
:10e118005a08b600a8003a003243800001006100a6
:10e12800ad003a00280090006808b600aa003a003e
:10e13800a243800001006100b0003a00280090006e
:10e148007608b600ad003a00124480000100610074
:10e15800b2003a00280090008408b600af003a00e8
:10e168008244800001006100e5003a002800900028
:10e178009208b600e2003a00f24480000100610013
:10e18800e8003a0028009000a008b600e5003a0030
:10e198006245800001006100ea003a002800900012
:10e1a800ae08b600e7003a00d245800001006100e1
:10e1b800ed003a0028009000bc08b600ea003a00da
:10e1c8004246800001006100f1003a0028009000fa
:10e1d800ca08b600ee003a00b246800001006100ad
:10e1e800f3003a0028009000d808b600f0003a0082
:10e1f8002247800001006100f5003a0028009000e5
:10e20800e608b600f2003a0092478000010061007b
:10e21800f8003a0028009000f408b600f5003a002b
:10e228000248800001006100fb003a0028009000cd
:10e238000209b600f8003a002ff19700224598002d
:10e248000a0078009ced07004f0578004f04be00d7
:10e258000080fa0000000600b8519000e7816100d4
:10e2680048509000670060004300dd008081710025
:10e2780058509000670060004600dd008081710002
:10e28800e8509000e7806000c908dd000851900060
:10e298006f01610018509000610060004400dd00cb
:10e2a8000001710028509000630060004500dd0007
:10e2b8000001710081817100890078006e8057002b
:10e2c8001fff07000000e0000a003a0098009000d5
:10e2d8006dff370058199000781a9000e8199000df
:10e2e800310020006e8057002aff07000000e00080
:10e2f8002f0032000080eb004f0578004f04be006d
:10e308000080fa0000000600d3ff370038009000b4
:10e31800c8009000810178000001780011002000f9
:10e328006e80570006ff07000000e000f1ff3a008a
:10e33800980090005aff370028199000481a90005a
:10e34800b8199000210020006e80570011ff0700c7
:10e358000000e000e7ff3a009800900056ff370001
:10e368000821900028229000982190004100200068
:10e378006e80570007ff07000000e000ddff3a004d
:10e388009800900058ff37003821900058229000dc
:10e39800c8219000510020006e805700fdfe070044
:10e3a8000000e000d3ff3a009800900054ff3700c7
:10e3b8009800900046ff3700682190006100200017
:10e3c8006e805700d3fe07000000e000c9ff3a0046
:10e3d8009800900050ff3700082990009829900075
:10e3e800710020006e805700d5fe07000000e00095
:10e3f800c0ff3a00980090004dff37007821900048
:10e40800810020006e805700c2fe07000000e00077
:10e41800b8ff3a00980090004bff3700d82a9000c8
:10e42800482a9000b8299000a82890002ff097005b
:10e438000081fb004fb89700017079002ff097001a
:10e448000081fb004fb8970002004000c808de00ba
:10e45800114098002ff197008280fb004fb8970079
:10e4680001004000234098002ff097008080fb00b7
:10e478004fb8970001004000c819de0033409800eb
:10e488002ff197008280fb004fb8970001004000f1
:10e49800444098002ff097008080fb004fb8970009
:10e4a800010040004822de00544098002ff19700f8
:10e4b8008280fb004fb8970001004000654098003b
:10e4c8002ff097008080fb004fb8970001004000b4
:10e4d800c82ade0075409800aff09700e8c04000f9
:10e4e800a1f79f00910020006c8057007efe070076
:10e4f8000000e0007fff3a009800900018ff370006
:10e5080068299000f8299000a10020006e8057002b
:10e518008bfe07000000e00076ff3a0098009000ac
:10e5280015ff370008319000b10020006e805700b9
:10e5380078fe07000000e0006eff3a0098009000a7
:10e5480013ff370058019000e8019000c100200037
:10e558006e8057007afe07000000e00065ff3a0071
:10e568009800900010ff3700183190003832900062
:10e57800a8319000d10020006e80570085fe07006a
:10e588000000e0005bff3a00980090000cff3700a5
:10e5980048319000e10020006e8057005dfe0700c2
:10e5a8000000e00053ff3a00980090000aff37008f
:10e5b80058319000f10020006e80570055fe07008a
:10e5c8000000e0004bff3a009800900008ff370079
:10e5d80068319000f8319000010120006e805700ea
:10e5e80057fe07000000e00042ff3a009800900044
:10e5f80005ff370008399000983990001101200074
:10e608006e8057004efe07000000e00039ff3a0018
:10e618009800900002ff37004207200008014100df
:10e628002ff097008080fb004fb897008080400053
:10e638008300200092487800320078004880de008d
:10e64800904098008180e8008301e900f9ff3a00d2
:10e65800aff09700f0c04000a1f79f002101200013
:10e668006c80570020fe07000000e00021ff3a0000
:10e678002ff19700224598000a0078008eec0700d9
:10e68800f1fe37000080fb000038a3000e003200c6
:10e6980067006000c1102a00e20f50000800320035
:10e6a8001600340001102a00e30f50000400320065
:10e6b800c10d2a00e40f5000010032008000eb0079
:10e6c80001007800000006006700600081142a003d
:10e6d800e20f5000faff320010003400c1132a0084
:10e6e800e30f5000f6ff320081112a00e40f5000ba
:10e6f800f3ff32008000eb00f1ff3700810e2a00a3
:10e708000000e000eeff3200e10f5000ebff3a009e
:10e71800400f2a0000000600ebff370041122a00d4
:10e728000000e000e6ff3200e10f5000e3ff3a008e
:10e7380000132a0000000600e3ff370061006000b4
:10e74800f1152a000400320041152a00e10f50009b
:10e75800010032008000eb00010078000000060094
:10e7680063006000c1182a00e10f50000800320061
:10e778000900340031182a00e20f5000040032006a
:10e78800a1162a00e30f5000010032008000eb00c0
:10e798000100780000000600e1172a000000e000f0
:10e7a800faff3a000100780000000600faff37007f
:10e7b80067006000911c2a00e30f50000600320039
:10e7c80007003400411d2a00e50f50000200320006
:10e7d800e11c2a000e003d00010078000000060040
:10e7e800b11b2a00e10f5000fbff3200011c2a0078
:10e7f800f9ff3c00611b2a000000e000f6ff320030
:10e80800311a2a000100780000000600f4ff3700e2
:10e81800f11d2a00e60f5000efff320071192a009f
:10e82800e70f5000ecff3200311a2a00f5ff3700dd
:020000040000fa
:10e83800c20c00000a000000000000005a0b000093
:10e848008600000000000000dc0c00000200000050
:10e858000200000000000000de0c000002000000c2
:10e8680002000000c00a0000c00a00009a00000070
:10e8780000000000e00c00000200000002000000a0
:10e88800ffff000000080000c001000002000000b7
:10e89800000000000000000001000000000000006f
:10e8a800020001000000000000000200000000005b
:10e8b8000100020000020000000000000004000047
:10e8c8000000030000030000030000000000000037
:10e8d800080000000007000003000400000000001a
:10e8e80000001000000000000f00030000050000f9
:10e8f800000000000020000000001f0000030000ce
:10e90800060000000000000040000000003f00007a
:10e918000100070000000000000080000000000067
:10e928007f00020000080000000000000000010055
:10e938000000ff00000100000900000000000000c6
:10e948000002000000ff010004000a0000000000af
:10e958000000000004000000ff030200000b00009c
:10e9680000000000000008000000ff000701000090
:10e978000c000000000000000010000000ff0f0065
:10e9880002000d0000000000000000002000000050
:10e99800ff1f0300000e0000000000000000400000
:10e9a8000000ff003f0100000f0000000000000011
:10e9b8000080000000ff7f0001001000000100003f
:10e9c8000100000000000000ffff0200001100002d
:10e9d80001000200000000000100ff00ff0200002b
:10e9e80012000100000400000000030000ffff0007
:10e9f80008001300000100000800000000070000e4
:10ea0800ffff0000001400000100100000000000db
:10ea18000f00ff00ff0000001500010000200000ab
:10ea280000001f0000ffff000000160000010000aa
:10ea380040000000003f0000ffff0000001700003a
:10ea480001008000000000007f00ff00ff000000c0
:10ea580018000100000000000000ff00ffffff0099
:10ea680000001900000100000000000000ffff0086
:10ea7800ffff0000001a0000010000000000000075
:10ea8800ffffff00ff0000001b0000000007000060
:10ea9800ffffff00ffffff0000001c000000000058
:10eaa80000007c0000ffff00ffff0000001d0000c9
:10eab8000000000000800200ffffff00ff000000d0
:10eac8001e000000000000008001ff00ffffff00a3
:10ead80000001f000000000003000000e0ffff002e
:10eae800ffff0000000000006c0c00002c0000007c
:10eaf8000200000002010000000000000000000009
:10eb080000000000000000000000000000000000fd
:10eb180000000000000000000000000000000000ed
:10eb28000000000000000000000000008600000057
:10eb3800c0090000000100000200000042000000bf
:10eb480000000000000000000000000000000000bd
:10eb580000000000000000000000000000000000ad
:10eb6800000000000000000000000000000000009d
:10eb7800000000000000000000000000000000008d
:10eb8800000000000000000000000000000000007d
:10eb9800000000000000000000000000000000006d
:10eba800000000000000000000000000000000005d
:10ebb800000000000000000000000000000000004d
:10ebc800000000000000000000000000000000003d
:10ebd800000000000000000000000000000000002d
:10ebe800000000000000000000000000000000001d
:10ebf800000000000000000000000000000000000d
:10ec080000000000000000000000000000000000fc
:10ec180000000000000000000000000000000000ec
:10ec280000000000000000000000000000000000dc
:10ec380000000000000000000000000000000000cc
:10ec480000000000000000000000000000000000bc
:10ec580000000000000000000000000000000000ac
:10ec6800000000000000000000000000000000009c
:10ec7800000000000000000000000000000000008c
:10ec8800000000000000000000000000000000007c
:10ec980000000000980c00002a000000020000009c
:10eca8009a0ce00088dc8800de8824008a2c8a0020
:10ecb8004c8aa6008a188b00588bae000ce088009e
:10ecc800dc88de0088e28800ea880a008964890016
:10ecd800d68916008a010000e20c0000020000003c
:10ece80000000000260e000068000000020000007e
:10ecf800000000000000000000000000000000000c
:10ed080000000000000000000000000000000000fb
:10ed180000000000000000000000000000000000eb
:10ed280000000000000000000000000000000000db
:10ed380000000000000000000000000000000000cb
:10ed48000000000000000000ffffff0000000000be
:10ed580000000000000000000000000000000000ab
:10ed6800000000000000000000000000000000009b
:10ed78000000000000000000000000004a0f000032
:10ed88000400000000000000520f00000200000014
:10ed98000200000001000000e60c0000b8000000be
:10eda800000000009e0d0000880000000000000028
:10edb800f40e000018000000000000001e0f000004
:10edc8000a0000000200000000000000000000002f
:10edd80000008000bf000000380f0000060000009f
:10ede80000000000540f00000200000000000000b6
:10edf800cc0c000008000000020000000000000029
:10ee08000000000000000000e00b000046000000c9
:10ee180002000000000000000000000000000000e8
:10ee280000000000000000000000000000000000da
:10ee380000000000000000000000000000000000ca
:10ee480000000000000000000000000000000000ba
:10ee580000000000000000000000000000000000aa
:10ee6800000000000000000000000000000000009a
:10ee780000000000560f0000020000000000000023
:10ee8800280f00000800000000000000d40c00005b
:10ee98000800000002000000000000000000000060
:10eea80000000000260c00004600000002000000e0
:10eeb800000000000000000000000000000000004a
:10eec800000000000000000000000000000000003a
:10eed800000000000000000000000000000000002a
:10eee800000000000000000000000000000000001a
:10eef800000000000000000000000000000000000a
:10ef080000000000000000000000000000000000f9
:10ef18004e0f00000400000002000000020009007b
:10ef280000000000580f000002000000020000006e
:10ef3800000000003e0f0000060000000200000074
:10ef48000400000000000000440f0000060000005c
:10ef58000200000022008e000e2200008e0e00002b
:10ef680044000000000000000c0f00001200000028
:10ef78000200000001000200000400000800100068
:10ef880000000000202b2d0023300000300f00006f
:10ef98000800000002000000686a6c00747a4c00e7
:10efa80000000000d20e0000220000000200000055
:10efb8003031320033343500363738003961620079
:10efc8006364650066003000313233003435360042
:10efd80037383900414243004445460000000000ec
:10efe800e40c000002000000000000000000000027
:020000040000fa
:10eff800889fbe008a9fbe008c9fbe0040002000f4
:10f00800bb0e07000004780050788800cf80de002f
:10f018002cca07000005be000800e0006a003500a1
:10f0280002002400c34124000a00be0024cb0700cc
:10f038000000e0003b003400020020006349240087
:10f048000a00be00c0ca070002002000a34724002f
:10f0580047ca07000004be000001be0086ca0700b8
:10f068000006be000001be000800be0082ca0700fc
:10f07800c21a240043fc23007fca07000005be0013
:10f0880062e9290093c32b000c00be007aca07006e
:10f098000001be000a00be00acca07000005be00a1
:10f0a800e2d92b0063fe23000800be0072ca0700e5
:10f0b8000001be000a00be00a4ca0700e2942000b6
:10f0c800a3012400a1ca07000001be00000020001f
:10f0d80001f8230026ca07000004be006011b8002a
:10f0e800f9ca07000000e0002f00350002002000e8
:10f0f800030024000800be00f1ca07000000e00079
:10f108000200340008002000090024000878880064
:10f11800197888004f06be004f05be004f04be0098
:10f128000000060002002000634924000a00be0017
:10f1380085ca070002002000a34724000cca070064
:10f148000004be000001be004bca070002402200b6
:10f1580043f7230048ca07000005be0002c021008b
:10f16800230224000800be0043ca07000001be00b5
:10f178000a00be0075ca070032732d00d3002400b0
:10f1880072ca07000001be000000200001f8230039
:10f19800f7c907000004be006011b800caca07001a
:10f1a8000000e000d1ff3d006044b8000878880006
:10f1b800197888004f06be004f05be004f04be00f8
:10f1c80000000600d7ff3700020020000378240063
:10f1d8005eca07000005be0091ff3700889fbe0089
:10f1e8008a9fbe008c9fbe00c0002000400e070012
:10f1f8000004780020788800cf80de00b1c90700bd
:10f208000005be000800e0006a0035000200240086
:10f21800c34124000a00be00a9ca07000000e0009c
:10f228003b00340002002000634924000a00be00ad
:10f2380045ca070002002000a3472400ccc90700e4
:10f248000004be000001be000bca07000006be0095
:10f258000001be000800be0007ca0700c21a240049
:10f2680043fc230004ca07000005be0062e9290028
:10f2780093c32b000c00be00ffc907000001be00ad
:10f288000a00be0031ca07000005be00e2d92b0003
:10f2980063fe23000800be00f7c907000001be0096
:10f2a8000a00be0029ca0700e2942000a301240036
:10f2b80026ca07000001be000000200001f8230054
:10f2c800abc907000004be006011b8007eca070081
:10f2d8000000e0002f003500020020000300240099
:10f2e8000800be0076ca07000000e00002003400f3
:10f2f8000800200009002400a8778800b977880052
:10f308004f06be004f05be004f04be0000000600b9
:10f3180002002000634924000a00be000aca070050
:10f3280002002000a347240091c907000004be0082
:10f338000001be00d0c907000240220043f72300a5
:10f34800cdc907000005be0002c021002302240029
:10f358000800be00c8c907000001be000a00be00c0
:10f36800fac9070032732d00d3002400f7c907003b
:10f378000001be000000200001f823007cc907003e
:10f388000004be006011b8004fca07000000e0008a
:10f39800d1ff3d006044b800a8778800b97788009d
:10f3a8004f06be004f05be004f04be000000060019
:10f3b800d7ff37000200200003782400e3c90700c4
:10f3c8000005be0091ff3700889fbe008a9fbe00df
:10f3d8008c9fbe00b0002000c50d07000004780017
:10f3e80030788800cf80de0036c907000005be00ef
:10f3f8000800e0006a00350002002400c341240030
:10f408000a00be002eca07000000e0003b003400de
:10f4180002002000634924000a00be00cac9070090
:10f4280002002000a347240051c907000004be00c1
:10f438000001be0090c907000006be000001be0022
:10f448000800be008cc90700c21a240043fc230030
:10f4580089c907000005be0062e9290093c32b0093
:10f468000c00be0084c907000001be000a00be00ef
:10f47800b6c907000005be00e2d92b0063fe2300d1
:10f488000800be007cc907000001be000a00be00db
:10f49800aec90700e2942000a3012400abc907000d
:10f4a8000001be000000200001f8230030c9070059
:10f4b8000004be006011b80003ca07000000e000a5
:10f4c8002f00350002002000030024000800be00c1
:10f4d800fbc907000000e00002003400080020001b
:10f4e80009002400c8778800d97788004f06be0035
:10f4f8004f05be004f04be000000060002002000b9
:10f50800634924000a00be008fc9070002002000da
:10f51800a347240016c907000004be000001be006e
:10f5280055c907000240220043f7230052c90700cb
:10f538000005be0002c02100230224000800be000e
:10f548004dc907000001be000a00be007fc90700c0
:10f5580032732d00d30024007cc907000001be00cf
:10f568000000200001f8230001c907000004be00c4
:10f578006011b800d4c907000000e000d1ff3d00c9
:10f588006044b800c8778800d97788004f06be0065
:10f598004f05be004f04be0000000600d7ff37002d
:10f5a800020020000378240068c907000005be0097
:10f5b80091ff3700889fbe008a9fbe008c9fbe00c7
:10f5c800a00020004a0d0700000478004078880059
:10f5d800cf80de00bbc807000005be000800e000c1
:10f5e8006a00350002002400c34124000a00be005e
:10f5f800b3c907000000e0003b003400020020000f
:10f60800634924000a00be004fc907000200200019
:10f61800a3472400d6c807000004be000001be00ae
:10f6280015c907000006be000001be000800be00a4
:10f6380011c90700c21a240043fc23000ec90700a1
:10f648000005be0062e9290093c32b000c00be0030
:10f6580009c907000001be000a00be003bc9070037
:10f668000005be00e2d92b0063fe23000800be009f
:10f6780001c907000001be000a00be0033c9070027
:10f68800e2942000a301240030c907000001be0055
:10f698000000200001f82300b5c807000004be00e0
:10f6a8006011b80088c907000000e0002f0035008d
:10f6b80002002000030024000800be0080c90700e3
:10f6c8000000e000020034000800200009002400c7
:10f6d800e8778800f97788004f06be004f05be001e
:10f6e8004f04be0000000600020020006349240009
:10f6f8000a00be0014c9070002002000a347240026
:10f708009bc807000004be000001be00dac807005d
:10f718000240220043f72300d7c807000005be00b7
:10f7280002c02100230224000800be00d2c807003e
:10f738000001be000a00be0004c9070032732d0094
:10f74800d300240001c907000001be00000020000a
:10f7580001f8230086c807000004be006011b80045
:10f7680059c907000000e000d1ff3d006044b8001f
:10f77800e8778800f97788004f06be004f05be007d
:10f788004f04be0000000600d7ff3700020020002b
:10f7980003782400edc807000005be0091ff37007c
:10f7a8001400fa00889fbe002007980031079800cf
:10f7b8004207980053079800640798007507980057
:10f7c800060f9800170f98006e019000fe01900038
:10f7d8000e0890009e089000dcc807000001be00db
:10f7e8006e009000fe00900061c80700008fbe0008
:10f7f8002e019000be0190001e00be009ec80700aa
:10f808000004be001e01be000000200001f8230015
:10f81800cdc807004e019000de01900096c8070091
:10f828000001be000800be00c8c8070020079800f5
:10f83800310798002e009000be0090004f04be00d3
:10f848000080fa00000006000600fa00889fbe004b
:10f85800000f780012079800230798001e00780010
:10f86800400a9000d00a90001e0078001001be00e7
:10f878000400be0080c807001e01780060019800df
:10f88800710198001e007800000c9000900c900008
:10f898001e0078001002be001e007800600990006b
:10f8a800f00990000400be0073c807000001be0004
:10f8b8000800be00a5c807001e01780000099800ce
:10f8c800110998001e0078001002be001e00780082
:10f8d80020019000b00190000400be009ac8070003
:10f8e8001e019000ae01900021c807000002be0072
:10f8f8001e00780000119000901190000400be00d6
:10f908005dc807001e017800200998003109980099
:10f918001e00780060029000f00290001e0078003f
:10f9280000099000900990000400be0087c80700f5
:10f938000002be001e00780020099000b009900067
:10f948000400be0081c807001e017800400198002d
:10f95800510198001e0078001000be001e017800ba
:10f9680020019800310198004f04be000080fa0081
:10f97800000006000600fa00889fbe00000f78000d
:10f9880012079800230798001e007800400a90008c
:10f99800d00a90001e0078001001be000400be00ce
:10f9a80035c807001e0178006001980071019800b1
:10f9b800707a80000000e900707a8800807a800000
:10f9c8000000e900807a8800707a80000000e0007a
:10f9d80027003c001e0078001000be006011b8002f
:10f9e800b7c807000000e00001003c002000370015
:10f9f8001e0078001000be006011b800b0c80700f3
:10fa08000000e00001003c00110037001e007800f3
:10fa1800000c9000900c90001e0078001002be00b0
:10fa28001e00780060099000f00990000400be00f4
:10fa380011c807000001be000800be0043c8070047
:10fa48001e01780000099800110998000600370087
:10fa58001e00780090089000000890001e017800b1
:10fa6800000998001109980020002000707a880089
:10fa7800807a80000000e00027003c001e0078002b
:10fa88001000be006011b8008fc807000000e00039
:10fa980001003500200037001e0078001000be006d
:10faa8006011b80088c807000000e00001003500b8
:10fab800110037001e007800000c9000900c900098
:10fac8001e0078001002be001e0078006009900039
:10fad800f00990000400be00e7c707000001be005f
:10fae8000800be0019c807001e0178000009980028
:10faf80011099800060037001e0078009008900051
:10fb0800000890001e01780000099800110998006b
:10fb180090002000807a88001e0078001002be0045
:10fb28001e00780020019000b00190000400be0083
:10fb380005c807001e019000ae0190008cc70700a1
:10fb48000002be001e007800001190009011900085
:10fb58000400be00c8c707001e01780020099800ed
:10fb6800310998001e00780060029000f0029000b1
:10fb78001e00780000099000900990000400be0063
:10fb8800f2c707000002be001e007800200990009e
:10fb9800b00990000400be00ecc707001e01780001
:10fba80040019800510198001e0078001000be0026
:10fbb8001e01780020019800310198004f04be0012
:10fbc8000080fa00000006000600fa00889fbe00c8
:10fbd800000f780012079800230798001e0078008d
:10fbe800000c9000900c90001e0078001002be00df
:10fbf8001e00780060099000f00990000400be0023
:10fc08009dc707000001be000800be00cfc707005f
:10fc18001e01780000099800110998001e0078005c
:10fc2800400a9000d00a90001e0078001001be0023
:10fc38000400be0090c707001e0178002009980044
:10fc4800310998001e007800000a9000900a900080
:10fc58001e00780020099000b00990000400be0042
:10fc6800bac707001e0178004001980051019800aa
:10fc78001e0078001000be001e01780020019800c8
:10fc8800310198004f04be000080fa000000060011
:10fc98001200fa00889fbe0040079800520798009b
:10fca8006307980074079800050f98005e0090009d
:10fcb800ee00900020079800310798007e01900020
:10fcc8008e099000028fbe004e009000d000900078
:10fcd800400090001e01be00f9c707000000e000c8
:10fce80001003c00120037004e009000000c90000c
:10fcf800900c90004e00900040019000d0019000c0
:10fd08001e00be0090c707000001be000800be002c
:10fd18008ec707004e01900000099800110998004d
:10fd28004e0090001e01be0042009800530098004b
:10fd38004e009000d0009000400090002e019000ee
:10fd4800be019000e0c707000000e0000100350098
:10fd5800140037004e009000000c9000900c9000aa
:10fd68004e00900040019000d00190002e009000bd
:10fd7800be00900074c707000001be000800be0066
:10fd880072c707004e0190000009980011099800f9
:10fd98004e0090002e019000be0190004200980095
:10fda800530098004f04be000080fa0000000600cf
:10fdb8000a00fa00000f780012079800230798003d
:10fdc80034079800450798001e00780090089000b6
:10fdd800000890003e019000ce019000b8c70700cf
:10fde8000000e00001003c00050037001e0078001c
:10fdf8003e019000ce019000020898001308980078
:10fe08001e00780090089000000890001e019000e5
:10fe1800ae019000acc707000000e000010035000b
:10fe2800050037001e0078001e019000ae0190000a
:10fe380002089800130898000080fa0000000600e5
:10fe48000600fa00000f78001207980023079800b0
:10fe58001e0078001000be001e019000ae01900048
:10fe680097c707000000e00001003c0005003700cc
:10fe78001e0078001e019000ae0190000288be00ae
:10fe8800100037001e0078001002be001e0090000f
:10fe9800ae0090000001be0003f0a2000400be0006
:10fea80089c707000000e0000100350005003700a1
:10feb8001e009000ae00900001f0a2001e01780024
:10fec8000089be000080fa00000006000000fa0069
:10fed8000000370006c2bf00614060000004e00077
:10fee800fcff3a0006c2bf00644060000004e00066
:10fef800f8ff3a0006c2bf00684060000004e00056
:10ff0800f4ff3a0006c2bf00704060000004e00041
:10ff1800f0ff3a0009c2bf000044b2000004e0004c
:10ff2800ecff3a000080fa00000006000000fa002a
:10ff380007e2a90007a2a9000782a8000762a90092
:10ff48000742a9000722a8000702a90006e2a900a3
:10ff580006c2a90006a2a9000682a9000662a90095
:10ff68000642a9000622a9000602a900f005200001
:10ff780020108800c10a200091407800f0c8b30022
:10ff880000c0600001c5b30001407000ace0b700dc
:10ff980008c2a9009600a90007e2a80000a821004d
:10ffa80061002000450c0700100020000080fa00c6
:10ffb800000006000000fa0007e2a9008620a90058
:10ffc8008600a9009600a900d8ff070006000700d0
:10ffd80000fa200001002000380c07001000200063
:10ffe8000080fa00000006000000fa008620a90040
:10fff8009620a80000322000010020002f0c0700e6
:020000040001f9
:10000800100020000080fa00000006000000fa003e
:100018008620a9009620a900100020000080fa0080
:10002800000006000600fa000000370016c2bf00f4
:10003800614060000004e000fcff3a0016c2bf0007
:10004800644060000004e000f8ff3a0016c2bf00f8
:10005800684060000004e000f4ff3a0016c2bf00e8
:10006800704060000004e000f0ff3a0016c2bf00d4
:10007800624060000004e000ecff3a0061f52000f7
:1000880010c0b3008048780008c2bf00704060000c
:100098000004e000170032000602a80000712200e8
:1000a80001002000008fbe000b00370060f5200023
:1000b800104078000004e00003003a00100020001f
:1000c800200798000d0037000080eb008080eb00cf
:1000d8001e0f40005e9748001e00be00e00f500053
:1000e800e08f5800f1ff3a008000eb0021079800ec
:1000f800020037000000eb00200798002e00900057
:100108000080fa00000006000600fa0061f52000f1
:1001180060c0b3008048780008c2bf006840600033
:100128000004e000170032000622a8000071220037
:1001380001002000008fbe000b00370060f5200092
:10014800104078000004e00003003a00100020008e
:10015800200798000d0037000080eb008080eb003e
:100168001e0f40005e9748001e00be00e00f5000c2
:10017800e08f5800f1ff3a008000eb00210798005b
:10018800020037000000eb00200798002e009000c6
:100198000080fa00000006000200fa0061f5200065
:1001a80030c0b3008048780006c2bf0061406000dc
:1001b8000004e00010003a0006c2bf00644060007e
:1001c8000004e0000c003a0006c2bf00684060006e
:1001d8000004e00008003a0006c2bf00704060005a
:1001e8000004e00004003a0006c2bf00624060005c
:1001f8000004e000030032000000eb00000f78006c
:100208000b00370006a2a9000682a80060f52000ae
:10021800104078000004e00003003a0010002000bd
:10022800000f7800020037000000eb00000f780094
:100238001e0078000080fa00000006000600fa00a0
:1002480061f5200030c0b3008048780006c2bf00c6
:10025800614060000004e00010003a0006c2bf00e0
:10026800644060000004e0000c003a0006c2bf00d1
:10027800684060000004e00008003a0006c2bf00c1
:10028800704060000004e00004003a0006c2bf00ad
:10029800624060000004e000030032000000eb0050
:1002a800200798001700370006a2a8000682a800b9
:1002b8000071220001002000008fbe000b003700f3
:1002c80060f52000104078000004e00003003a00c8
:1002d80011002000210798000a0037000080eb0079
:1002e8008080eb001e0f40005e9748001e00be0095
:1002f800e00f5000e08f5800f1ff3a008000eb005b
:10030800210798002e0090000080fa0000000600e7
:100318000a00fa003007980000712200010020004e
:1003280010079800210798000040eb00004f780064
:1003380061f5200040c0b3008048780000712200b9
:100348000100200010079800210798001d003700c1
:1003580006c2bf00614060000004e00013003a00dc
:1003680006c2bf00644060000004e0000f003a00cd
:1003780006c2bf00684060000004e0000b003a00bd
:1003880006c2bf00704060000004e00007003a00a9
:1003980009c2bf000044b2000004e00003003a00b4
:1003a80010c0b300004f78000b0037001e0090000b
:1003b800ae00900061005000e080580010079800df
:1003c800210798001e009000ae009000e00f50003a
:1003d800e08f5800deff3a001e04e00003003a00f8
:1003e8000000eb00400798001e0037000662a800d6
:1003f800006a2800110020001007980021079800c3
:100408001100370060f52000104078000004e0007b
:1004180007003a0000108000804078003e009000fd
:100428000148780010002000400798000d003700b0
:100438001e009000ae00900061005000e08058005f
:1004480010079800210798001e009000ae00900049
:10045800e00f5000e08f5800eaff3a000000eb0080
:10046800400798004e0090000080fa000000060047
:100478000600fa0061f5200050c0b30080487800fb
:100488000642a8000071220001002000008fbe0073
:100498000b00370060f52000104078000004e000f1
:1004a80003003a0010002000200798000a003700d7
:1004b8000080eb008080eb001e0f40005e97480034
:1004c8001e00be00e00f5000e08f5800f1ff3a0018
:1004d8008000eb00210798002e0090000080fa00b1
:1004e800000006000800fa004047980061f5200067
:1004f80020c0b300804878004e4090000000fb0008
:10050800101088000602a8000071220001002000d7
:10051800008fbe000b00370060f520001040780007
:100528000004e00003003a001000200030079800a3
:100538000a0037000080eb008080eb001e0f4000af
:100548005e9748001e00be00e00f5000e08f580084
:10055800f1ff3a008000eb00310798003e00900060
:100568000080fa0000000600809fbe000000fa002c
:100578008620a90061f520000040eb008048780043
:100588000080fa004f00be0000400600881f780077
:10059800000478008000eb00010878001100980042
:1005a80051f6070011002000080078004ef60700f9
:1005b80021002000080078004bf6070031002000d9
:1005c8000800780048f6070041002000080078007d
:1005d80045f60700510020000800780042f60700a1
:1005e80081002000080078003ff60700c1002000c5
:1005f800080078003cf60700710020000800780029
:1006080039f60700910020000800780036f6070048
:10061800b10020000800780033f60700210120000f
:100628000800780030f60700d100200008007800a4
:100638002df60700e1002000080078002af60700e0
:100648004f04780000000600c067800000404000aa
:10065800f64cb7005aebb700e0568000f156800020
:10066800005b8800115b880021578000215b8800af
:1006780010578000305b880002002000031224001d
:10068800506d8000616d8000fbc4070090c50700b5
:10069800705c88000200200003122400706d800046
:1006a800816d8000f4c4070089c50700805c88005c
:1006b8000200200003122400906d8000a16d8000cc
:1006c800edc4070082c50700905c88000200200086
:1006d80003122400906e8000a16e8000e6c407001b
:1006e8007bc50700a05c88000200200003122400dc
:1006f800b06e8000c16e8000dfc4070074c50700bb
:10070800b05c88000200200003122400d06e800034
:10071800e16e8000d8c407006dc50700c05c880082
:1007280002002000a3472400b06d8000c16d800046
:10073800d1c4070066c50700d05c8800020020000d
:10074800a3472400d06d8000e16d8000cac4070073
:100758005fc50700e05c880002002000a347240072
:10076800f06d8000016e8000c3c4070058c5070003
:10077800f05c880002002000a3472400506f80002e
:10078800616f8000bcc4070051c50700005d880088
:1007980002002000a3472400706f8000816f800052
:1007a800b5c407004ac50700105d88000200200094
:1007b800a3472400906f8000a16f8000aec407009b
:1007c80043c50700205d8800a62bef00020020002b
:1007d800a3472400306e8000416e8000a6c4070045
:1007e8003bc50700505d880002002000a347240095
:1007f800506e8000616e80009fc4070034c50700fa
:10080800605d8800b06f8000c16f800030c5070050
:10081800405d880071fa070021788000715d8800ca
:10082800e9fa070030788000805d880061fb0700e6
:1008380041788000915d8800edf9070050788000cc
:10084800a05d8800a8ec070002002000a347240050
:10085800207980003179800087c407001cc5070013
:10086800d05d880002002000a3472400e06b8000d0
:10087800f16b800080c4070015c50700e05d8800a3
:1008880002002000a3472400206c8000316c800007
:1008980079c407000ec50700f05d88000069800074
:1008a8001169800002002000a347240072c40700d9
:1008b80007c50700005e8800206980003169800054
:1008c80002002000a34724006bc4070000c50700ee
:1008d800105e8800d0ea2d00b05d8800c05d8800f9
:1008e800205e8800305e8800405e8800505e880088
:1008f80040232100605e880002002000a3472400f6
:10090800b0738000c17380005bc40700f0c40700a7
:10091800705e880002002000a34724003074800025
:100928004174800054c40700e9c40700805e880051
:1009380002002000a3472400d0738000e1738000e8
:100948004dc40700e2c40700905e88000200200042
:10095800a3472400507480006174800046c40700d7
:10096800dbc40700a05e880002002000a347240023
:1009780090738000a17380003fc40700d4c40700af
:10098800b05e880002002000a34724001074800095
:100998002174800038c40700cdc40700c05e8800f9
:1009a80002002000a3472400707380008173800038
:1009b80031c40700c6c40700d05e880002002000ca
:1009c800a3472400f0738000017480002ac4070044
:1009d800bfc40700e05e880000000600460be20086
:1009e80020003a00480be20003003200100020000b
:1009f800305a88001b003700a2b520008040eb0069
:100a0800a0ae200081f507000000e00008003200d9
:100a1800f0668000008990000200e00011003200ba
:100a2800811e2a0000082000020001000d00370086
:100a3800cac2bf000000d10000c0ea0061406000e7
:100a480000404000a12c2000914078000114a10032
:100a580080c0700001007800cae2b70010002000d2
:100a6800305a880000000600480be20020003a00d7
:100a7800460be2000300320010002000405a8800b4
:100a88001b003700a2b520008040eb00a0ae20007c
:100a98005ef507000000e00008003200f066800004
:100aa800008990000200e0001100320071202a0045
:100ab80000082000020001000d003700cac2bf0074
:100ac8000000d10000c0ea00614060000040400022
:100ad800a12c2000914078000114a10080c0700072
:100ae80001007800cae2b70010002000405a8800d0
:100af80000000600889fbe008a9fbe008004780020
:100b080001047800fa6780000b6880006108b9006a
:100b18006cc307000800e00003003d00020020004d
:100b28000378240009c407000a01be0066c4070050
:100b38000000e00003003d000a00be0046c30700b5
:100b4800000478000900e00003003200e18f54003f
:100b580011003a00080037006a40b90080007800a8
:100b6800204f2800440307000800e00011003a0065
:100b7800ca22a9000f0037006a40b9008000780037
:100b8800805328003c0307000800e00009003a00f1
:100b9800ca22a90007003700f0668000008990008b
:100ba8000200e0000300320061222a000008200051
:100bb800020001004f05be004f04be000000060001
:100bc80010668800e10f500004003a002266880091
:100bd8003366880044668800556688000000060071
:100be8001066800000000600000178000000e000a8
:100bf800040032006000b800e10f510006003a001e
:100c08000300370010748000217480000200370050
:100c18002066800031668000000006000001780030
:100c28000000e000040032006000b800e10f51004d
:100c380006003a0003003700f0738000017480005a
:100c48000200370040668000516680000000060000
:100c5800889fbe008a1f7800d15d8000e16c880003
:100c6800802c2300808f500002003600e06c880042
:100c78000500370030c22200808f500002003e007d
:100c88000000e800e06c8800f067800001688000e0
:100c9800f1c2070000017800a1b5200000ac2000d7
:100ca800b0d70700a1b5200000ac200076d6070019
:100cb8006acbbf00e14f50001b003200170039001b
:100cc800e74f50001b003a00800020008cdf07002f
:100cd800005c8000cf80de00fac207000004be007e
:100ce800f05b8000cf80de00f6c207000801be007e
:100cf80064040700205c8000cf80de00f1c207009a
:100d08000004be00105c8000cf80de00edc207004a
:100d18000801be009c0407001401370010002000e1
:100d280077df0700110137002000200074df07007b
:100d38000e0137004000200071df07000000eb00c3
:100d4800005c8800f05b8800205c8800105c8800ec
:100d58006dcbbf000038a300030032001000200054
:100d6800d06b88001a00370067006000e10f500060
:100d780013003a007a2def00305c8000cf80de004f
:100d8800d0c2070002002000a3472400f8c20700d1
:100d98000004be001066800093ff0700d2cc2c0030
:100da800c3e4230034c307000001be000800be00ee
:100db80066c30700e06b8800f16b88000400370009
:100dc80010002000d06b88007c2def007e2def00f6
:100dd8006ecbbf000038a3000300320010002000d3
:100de800106c88001b00370067006000e10f50009e
:100df80014003a00822def00405c8000cf80de00b6
:100e0800b0c2070002002000a3472400d8c2070090
:100e18000004be001066800080ff0700d2cc2c00c2
:100e2800c3e4230014c307000001be000800be008d
:100e380046c3070001f0a200206c8800316c8800ce
:100e48000400370010002000106c8800842def008b
:100e5800862def006fcbbf000038a30003003200df
:100e680010002000506c88006b003700670060009d
:100e7800e10f50000f003200e30f500060003a000d
:100e88008a2def00505c8000cf80de008dc2070005
:100e9800b2fd200093042400f7c2070002002000de
:100ea800134e2400b2c20700606c8800716c880081
:100eb800590037008a2def00905c80008a0bb5003e
:100ec800cf80de007fc2070002002000031224004a
:100ed800a7c207000004be00160037000200200069
:100ee800433324000800be0075c307000000e0007b
:100ef8000500340002002000433b24000800be0027
:100f080011c307000004be000200200043332c0078
:100f18000800be006cc307000000e00005003d00ab
:100f280002002000433b24000800be0007c307005e
:100f38000004be006011b8000800be0062c30700cc
:100f48000000e00009003d000045eb000200200021
:100f580043332c000800be005bc307000000e0001c
:100f68000a003d001ac0b300080037000045eb0036
:100f780002002000433324000800be0050c30700cd
:100f88000000e000010034001ac0b3000a04e000c9
:100f9800d2ff3a0002002000031224000800be001d
:100fa80047c307000000e0000300340008002000e9
:100fb80009122400080037000200200003122c0048
:100fc8000800be0040c307000000e00002003d002a
:100fd8000800200009122c00d2cc2c00c3dc23000e
:100fe8000800be00a4c2070002002000031224006b
:100ff8005fc20700606c8800716c880006003700cb
:101008008a2def00905c8000cf80de002dc20700a3
:10101800606c8800716c880001b7200091407800ee
:101028000180fb000038a300100032006700600058
:10103800e40f500004003a0010002000a067880068
:10104800906c880049003700f42cef001000200055
:10105800906c8800505d8000cf80de0019c20700c8
:10106800a06c8800b16c8800400037006780600081
:10107800e20f50002800320003003c00e10f50004e
:1010880032003a0016003700e30f50000e0032001d
:10109800e40f50002d003a0010002000a0678800df
:1010a800922def00605c8000cf80de0005c2070053
:1010b80002002000a34724002dc20700a06c88006e
:1010c800b16c8800290037000000eb00a067880099
:1010d800906c8800942def00962def0023003700c8
:1010e8008000eb00a167880010002000806788005e
:1010f800916c8800605c8000cf80de00f1c1070041
:1011080002002000a347240019c20700a06c880031
:10111800b16c8800150037000000eb00806788007c
:10112800a0678800906c8800605c8000cf80de003b
:10113800e4c1070002002000a34724000cc20700f6
:10114800a06c8800b16c8800080037000000eb0034
:10115800a0678800906c8800505d8000cf80de001a
:10116800d8c10700a06c8800b16c88004f057800d2
:101178004f04be0000000600e22cec000000060050
:10118800c00ce20002003a00c02cef00000006008c
:101198008000eb00008c28005f010700890507002c
:1011a8008c050700c02cef0000000600f8ff370090
:1011b800000005000000050000000500010078009f
:1011c80082007800f706070000000500889fbe002f
:1011d800010478008004eb0008007800830707000a
:1011e8000000e000060032000804e8008904e80076
:1011f800080078007d0707000000e000faff3a00c9
:10120800090078004f04be0000000600889fbe0059
:101218008a1f7800010578000204be000300e00080
:1012280009003a00820078000a007800dd0607000d
:10123800e80607000000e000fdff3a004f057800cf
:101248004f04be0000000600e22cef00a1002000c1
:10125800008c280088010700880078000a007800c0
:10126800d0060700db060700000478000000e00055
:101278000b00320010678000808f5400f9ff3100a6
:101288008000eb00008c28007b0107000080eb0049
:101298004f0578004f04be0000000600eaff370043
:1012a80080007800008c280073010700080078008f
:1012b8004f0578004f04be0000000600e2ff37002b
:1012c800889fbe008a9fbe0001047800020578004e
:1012d800830478000300e0000e003a000200e000fa
:1012e8000800320008007800400707000000e0000e
:1012f800fcff32000804e8008904e800890f550063
:10130800f8ff3a000000eb004f05be004f04be0096
:1013180000000600e22cef00a1002000008c28004d
:10132800550107000a00e0000b003a008a05780022
:101338008000eb00008c28004f0107000080eb00c4
:101348008a8f5500efff32004f05be004f04be00e4
:1013580000000600efff37008005eb00080078006a
:10136800220707000000e000020032000804e8003d
:101378008b05e80010678000808f5400ecff39006f
:101388008a8f5500f5ff39008000eb00008c28009b
:10139800390107000080eb008a8f5500eaff3a0008
:1013a800d8ff3700881f7800010478000100e000aa
:1013b80006003a00090707000000e000fdff3200c0
:1013c8000000eb004f04780000000600e22cef005c
:1013d800a1002000008c280027010700106780006a
:1013e800800f540008003600fc0607000000e000eb
:1013f800faff32008000eb00008c28001e01070075
:101408000000eb00efff37008000eb00008c2800a5
:10141800190107000080eb004f0478000000060067
:10142800eaff37000200fa000f80e900ef06070024
:101438000000e000fcff3a000080fa00000006000f
:1014480001007800820078002506070000000500ea
:10145800889fbe00010478008004eb000800780033
:10146800c30607000000e000060032000804e80098
:101478008904e80008007800bd0607000000e000c5
:10148800faff3a00090078004f04be000000060089
:10149800889fbe008a1f7800010578000204be00fc
:1014a8000300e00009003a00820078000a00780092
:1014b8000b060700160607000000e000fdff3a00d3
:1014c8004f0578004f04be0000000600e22cef0034
:1014d800a1002000008c2800e700070088007800a1
:1014e8000a007800fe0507000906070000047800d6
:1014f8000000e0000b00320010678000808f54006d
:10150800f9ff31008000eb00008c2800da000700aa
:101518000080eb004f0578004f04be000000060075
:10152800eaff370080007800008c2800d20007000e
:10153800080078004f0578004f04be000000060040
:10154800e2ff3700889fbe008a9fbe000104780032
:1015580002057800830478000300e0000e003a00da
:101568000200e0000800320008007800800607004a
:101578000000e000fcff32000804e8008904e800ed
:10158800890f5500f8ff3a000000eb004f05be0038
:101598004f04be0000000600e22cef00a10020006e
:1015a800008c2800b40007000a00e0000b003a0095
:1015b8008a0578008000eb00008c2800ae00070048
:1015c8000080eb008a8f5500efff32004f05be0008
:1015d8004f04be0000000600efff37008005eb0057
:1015e80008007800620607000000e00002003200f0
:1015f8000804e8008b05e80010678000808f54001d
:10160800ecff39008a8f5500f5ff39008000eb00a8
:10161800008c2800980007000080eb008a8f550096
:10162800eaff3a00d8ff3700881f780001047800e5
:101638000100e00006003a00490607000000e0004b
:10164800fdff32000000eb004f04780000000600a8
:10165800e22cef00a1002000008c28008600070083
:1016680010678000800f5400080036003c06070011
:101678000000e000faff32008000eb00008c280038
:101688007d0007000000eb00efff37008000eb0053
:10169800008c2800780007000080eb004f047800d9
:1016a80000000600eaff37000200fa000f80e90098
:1016b8002f0607000000e000fcff3a000080fa0057
:1016c800000006000000fa000000eb008008880017
:1016d8000111200091407800f0ccb30000c06000f8
:1016e80010e1b7000000eb003008880000fa200085
:1016f8006008880084e0a90094e0a80011e1a8002f
:101708000080fa00000006000000fa0011e1a900bc
:101718000080fa00000006000800fa001007980090
:1017280021079800a07a8000000f78000b0037008e
:101738001e007800b00090001e009000808f5000be
:1017480003003a0011002000310798001f003700fd
:101758001e007800c0009000010f78001e00e00015
:10176800f3ff3a00a0002000d2bb0700000f78006a
:101778001e00e00002003a00100020001fbc070015
:10178800ae0090001e007800010878009e007800e6
:101798000000eb00900098009e00780010c0b30095
:1017a800c04098001e0078009e009000310098000c
:1017b800a17a80001e007800410098001e00780081
:1017c800a07a880011002000310798003e009000a0
:1017d8000080fa00000006000800fa0020079800c0
:1017e8000000eb0010079800a07a8000000f780036
:1017f8001a0037001e007800b00090002e009000fc
:10180800808f500010003a001e0090000000e00099
:10181800050032001e007800c00090001e009000f5
:1018280041009800030037001e0078004000900037
:10183800a07a88001e00780002bc07001100200072
:1018480031079800090037001e007800100798003b
:101858001e007800c0009000010f78001e00e00014
:10186800e4ff3a0020002000300798003e00900076
:101878000080fa00000006000800fa00100798002f
:1018880021079800a07a8000000f78000e0037002a
:101898001e007800b00090001e009000808f50005d
:1018a80006003a00ae0090001e007800010878009b
:1018b8001100200031079800070037001e0078004b
:1018c800c0009000010f78001e00e000f0ff3a0011
:1018d80020002000300798003e0090000080fa00a9
:1018e800000006000600fa0010079800a07a8000a1
:1018f800000f78000e0037001e007800b00090003e
:101908001e009000808f500006003a009e0078006c
:101918000000eb00900098001100200021079800bb
:10192800070037001e007800c0009000010f780003
:101938001e00e000f0ff3a00200020002007980079
:101948002e0090000080fa00000006000600fa0051
:1019580010079800a07a8000000f78000e0037006a
:101968001e007800b00090001e009000808f50008c
:1019780006003a009e0078000040eb00c040980046
:101988001100200021079800070037001e0078008a
:10199800c0009000010f78001e00e000f0ff3a0040
:1019a80020002000200798002e0090000080fa00f8
:1019b800000006000600fa0010079800a07a8000d0
:1019c800000f78000e0037001e007800b00090006d
:1019d8001e009000808f500006003a009e0078009c
:1019e80010c0b300c04098001100200021079800e3
:1019f800070037001e007800c0009000010f780033
:101a08001e00e000f0ff3a002000200020079800a8
:101a18002e0090000080fa00000006003600f80052
:101a2800809fbe00829fbe00849fbe00869fbe002e
:101a38003400f80000c0b300a00188000200fa00da
:101a4800a07a8000000f780084e0a9001e0037000b
:101a58001e00780040409000e14f500017003a0007
:101a68001e007800100078000000e000130032002b
:101a78001e007800100090008000e8001e0078002a
:101a8800110098001e007800100090008000780077
:101a98001e007800100078000000e900808f5000d8
:101aa800060036001e00780030009000000001009b
:101ab8009e0078000000eb00900098001e0078005f
:101ac800c0009000010f78001e00e000e0ff3a001f
:101ad8000080fa003400f9004f03be004f02be0038
:101ae8004f01be004f00be003600f900004006005e
:101af8000400fa0020479800314798000040eb00a6
:101b0800004f78001800370010c0b300004f78006d
:101b180044f907001e4f60002e40900071fa07003c
:101b28001e4f60003e4090006efa07001e4f600096
:101b380075f907001e4f60002e4090000040e80035
:101b480068fa07001e4f60000e00e800f0f9070071
:101b58001e4f6000b9f9070045fa07001e04e000af
